:020000040800F2
:10000000F8FF012075B00A0811B10A08F544050887
:1000100011B10A0811B10A0811B10A080000000064
:1000200000000000000000000000000011B10A08FC
:1000300011B10A080000000011B10A089D68040807
:1000400011B10A0811B10A0811B10A0811B10A0860
:1000500011B10A0811B10A08591E0408811E0408CA
:10006000A91E0408D11E0408F91E0408BD030000DF
:10007000D1030000E5030000F90300000D040000B7
:10008000210400003504000011B10A0811B10A086A
:1000900011B10A0811B10A0811B10A08211F040898
:1000A00011B10A08CD49040811B10A08BD49040874
:1000B000DD490408ED490408FD490408FD10040861
:1000C000F1100408311104082511040811B10A08BF
:1000D00011B10A08F93D0000493F0000B540000099
:1000E000611F040811B10A0800000000B94A0408A1
:1000F000914A0408C94A0408814A040849040000D6
:1001000011B10A086D2F04080D4A040811B10A083C
:1001100025420000954300001D4A040899D70908AC
:100120005D040000710400008504000099040000D3
:10013000AD04000011B10A0811B10A0811B10A0892
:1001400000000000000000000000000000000000AF
:10015000C1040000D5040000E904000005450000CA
:10016000651104085911040811B10A0811B10A08EF
:1001700011B10A0811B10A0811B10A080000000003
:1001800011B10A0811B10A0875460000E5470000E0
:1001900011B10A0811B10A0811B10A0811B10A080F
:1001A00011B10A0811B10A0811B10A0811B10A08FF
:1001B00011B10A0811B10A0811B10A08991104080D
:1001C0008D11040811B10A0811B10A0811B10A0809
:1001D00011B10A08E9CD090811B10A0811B10A08DC
:1001E00011B10A0811B10A0811B10A0811B10A08BF
:1001F00011B10A0811B10A0811B10A0811B10A08AF
:1002000011B10A0811B10A0811B10A0811B10A089E
:10021000D94A0408E94A0408F94A040811B10A084D
:1002200011B10A0811B10A0811B10A080000000052
:10023000712F040811B10A080000000011B10A086A
:1002400011B10A0811B10A0811B10A0811B10A085E
:1002500011B10A0811B10A0811B10A0811B10A084E
:1002600011B10A0811B10A0811B10A0811B10A083E
:1002700011B10A0811B10A08554900000000000038
:1002800011B10A080000000011B10A0800000000C6
:080290000000000011B10A0892
:020000040804EE
:10000000114A037A0168D35C10B4CC58CA1824F0A2
:100010000104CC501368DB07FCD4037D1F2B09D9E6
:10002000203B20225DF8044B02FA03F343F018034F
:10003000CB60704720225DF8044B02FA03F343F0D3
:1000400018038B60704700BFF0720B084368426D65
:1000500030B49A61EFF31182502383F31288416820
:10006000D2B2856C0B68046D23EA050323430B6051
:1000700082F31188436981681A68096822F00102D5
:10008000D0E908541A60826A1D605C615A60D0E948
:100090000B429C60DA600023B0F86C2030BCCA626E
:1000A00003777047002A4FEA014C034630B508BF7A
:1000B000E64600F1C00514BF8E468C460024196840
:1000C0000C3353F8042C43F8084C41EA0C0142EA83
:1000D0000E02AB4243F80C1C43F8042CEFD1D0F8CD
:1000E000C03043EA0E03C0E93144C0F8C03030BD2F
:1000F00010B40C4C6368002B11DD002004F1080CD7
:100100000146DCF8AC3003F1C00259600C33934275
:10011000FBD1013063680CF5867C8342F1DC5DF82D
:10012000044B704704000020F0B5404C04EB401332
:1001300093F8543403B9F0BD3D4B42011D7893F858
:1001400001C065450CD00CEB4C0E03EBCE0E9EF8B7
:1001500004604FEA4C0E771E012F5AD9032E52D05D
:100160002244A2F83814EFF31181902383F312880C
:1001700092F83A34C9B2B2F8380443EA4003002096
:100180009BB282F83A0481F311881909207881EA38
:1001900013215940D8B1C9431B01D2F8505401244E
:1001A000D2F83C049BB201F00F01D5F8AC2084409A
:1001B0000B4302F1C000590013F4004F8BB202D17F
:1001C0005168214351600C329042F4D1F0BDD2F815
:1001D0003C041B01D2F8502401F00F0110309BB2F7
:1001E0000124D2F8AC200B43844002F1C000590036
:1001F00013F4004F8BB202D15168214351600C328D
:100200009042F4D1F0BD0CF1010606F00306AE42B7
:10021000A6D0E64403EBCE030344597C00299FD0CB
:10022000A318012083F83A049AE700BF04000020D5
:10023000501D0024704700BF024B03EB401393F89E
:100240005504704704000020D0E90920131A5842D1
:100250005841704790F8573830B53BB990F8551869
:10026000012490F85638DAB2914200D830BD04FA31
:1002700003F2B0F85E5801332A43A0F85E28F2E793
:100280000379024613F0010006D0D2E90731D268A3
:100290005B1A013A03EA0200704710B5037904467D
:1002A00013F001030ED0FFF7EBFF034650B1226AB3
:1002B0006369E1689B5C0132B2FBF1F0DBB201FBE8
:1002C00010222262184610BD03799B070AD5436AA3
:1002D0008269D154436A02690133B3FBF2F102FB34
:1002E00011334362704770470171704703790146CB
:1002F00013F0020007D00B69D1E90921013B521A22
:100300001A40D2B2981A70470C4B4FF0E02C10B440
:100310005A6EDCF81800596E8A42F9D1996E8842FB
:10032000F6D8DC6E4FF47A7101FB04F31B1AB3FBB1
:10033000F4F35DF8044B01FB02307047501D0024BC
:1003400010B584464FEA810E102312F4004F4FEA95
:10035000420214BF0E240724013B92B2CCF80040A5
:10036000F444F2D100EB81128C010351122042F8C7
:10037000213010BD10B584464FEA810E0424130BC2
:10038000013C4FEA021203EB430392B203F118035C
:10039000CCF80030F444F2D100EB01130A01845090
:1003A000062043F8214010BD704700BF704700BFD2
:1003B00000EB4000024B03EBC00393F84905704784
:1003C00004000020064B93F8F825824206D900EB82
:1003D000400003EBC003D3F84C0570470020704782
:1003E000040000201D4B93F8FC25AAB3D3F8381560
:1003F00009B100200860012A2ED0D3F8501509B1A8
:1004000000200860022A27D0D3F8681509B100201F
:100410000860032A20D0D3F8801509B100200860B5
:10042000042A19D0D3F8981509B100200860052ACC
:1004300012D0D3F8B01509B100200860062A0BD0FD
:10044000D3F8C81509B100200860072A04D0D3F8F2
:10045000E0350BB100221A60704700BF0400002095
:100460001D4B93F8FC25AAB3D3F8381509B1002029
:100470000860012A2ED0D3F8501509B10020086079
:10048000022A27D0D3F8681509B100200860032A92
:1004900020D0D3F8801509B100200860042A19D0B3
:1004A000D3F8981509B100200860052A12D0D3F8B6
:1004B000B01509B100200860062A0BD0D3F8C81582
:1004C00009B100200860072A04D0D3F8E0350BB149
:1004D00000221A60704700BF04000020C34B1B7845
:1004E000002B40F04D81C24B93F8FC25002A00F010
:1004F000478193F8481530B500294ED1D3F8381507
:100500000020012A086047D993F86015002966D1B8
:10051000D3F850150020022A08603DD993F87815C9
:10052000002940F0C980D3F868150020032A08602C
:1005300032D993F89015002940F0E080D3F8801567
:100540000020042A086027D993F8A815002940F054
:10055000F680D3F898150020052A08601CD993F876
:10056000C015002940F00D81D3F8B0150020062AEF
:10057000086011D993F8D815002959D1D3F8C815B6
:100580000020072A086007D993F8F025002A72D1C5
:10059000D3F8E03500221A6030BDD3F83C25910A2B
:1005A000A1F58011522940F20D814FF0FE0CEFF3BE
:1005B0001181502080F312888E4C4FF02C0E556A1A
:1005C000C9B250690EFB0C4C013540F00100CCF86B
:1005D0009850506181F3118893F8FC258EE7D3F889
:1005E0005425910AA1F58011522940F2EF804FF075
:1005F000FE0CEFF31181502080F312884FF02C0E87
:10060000556A7C4CC9B2506901350EFB0C4440F070
:100610000100C4F89850506181F3118893F8FC25CB
:100620000020D3F85015022A08603FF677AFB3E7F1
:10063000D3F8CC25910AA1F58011522900F2E2806D
:100640006D4810F801C0EFF31181502080F312883B
:100650004FF02C0E556A674CC9B2506901350EFB3C
:100660000C4440F00100C4F89850506181F31188A7
:1006700093F8FC2582E7D3F8E425910AA1F58011CF
:10068000522900F2C2805C4810F801C0EFF31181DA
:10069000502080F312884FF02C0E556A554CC9B289
:1006A000506901350EFB0C4440F00100C4F898502D
:1006B000506181F311886BE7D3F86C25910AA1F59D
:1006C0008011522940F286804FF0FE0EEFF3118127
:1006D000502080F312884FF02C0C556A454CC9B25B
:1006E000506901350CFB0E4440F00100C4F89850ED
:1006F000506181F3118893F8FC2514E7D3F8842521
:10070000910AA1F58011522968D94FF0FE0CEFF340
:100710001181502080F312884FF02C0E556A354C11
:10072000C9B2506901350EFB0C4440F00100C4F819
:100730009850506181F3118893F8FC25FEE6D3F8B8
:100740009C25910AA1F5801152294BD94FF0FE0C3E
:10075000EFF31181502080F312884FF02C0E556A70
:10076000244CC9B2506901350EFB0C4440F0010025
:10077000C4F89850506181F3118893F8FC25E8E69D
:100780007047D3F8B425910AA1F58011522935D9C3
:100790004FF0FE0CEFF31181502080F312884FF0E0
:1007A0002C0E556A134CC9B2506901350EFB0C442E
:1007B00040F00100C4F89850506181F3118893F81B
:1007C000FC25D1E60C4810F801C0F0E60A4810F804
:1007D00001C00EE7084810F801E077E7064810F876
:1007E00001C094E7044810F801C0B1E700000024FC
:1007F00004000020501D002478DD0A08044810F889
:1008000001C0C7E74FF0FE0C1DE74FF0FE0C3DE7BF
:1008100078DD0A0800EE100AB8EE400A704700BF03
:10082000BCEEC00A10EE103A98B2704707280AD8FA
:100830004FF4B472054B02FB0033B3F80006B0FA74
:1008400080F0400970470020704700BF040000207E
:10085000072807D8044B4FF4B471012201FB003381
:1008600083F80226704700BF04000020072808D83C
:10087000044B03EB401393F8542412B1012283F884
:100880003A24704704000020072808D8054B03EBE2
:100890004013B3F83804B0FA80F0400970470020E4
:1008A000704700BF04000020054B93F8F8258242F2
:1008B00004D903EB4013D3F8440470470020704779
:1008C0000400002038B5074B14460D46D3F8043316
:1008D0001B6A984702464FF40073002012682A6092
:1008E000238038BD501D002408B5064BD3F80433CF
:1008F00023B15B699847013840B208BD4FF0FF3023
:1009000008BD00BF501D0024002070472DE9F041B4
:100910000BB316460F4603EB0208124CD4F80453EF
:10092000002339463046AD681A46A8470028F5D05E
:10093000D4F80433002BFBD05B6998470028F7D02C
:10094000013607F50077B045E8D1636E0020C4F8A2
:100950000833BDE8F081034C0020636EC4F808330F
:10096000BDE8F081501D00242DE9F0413BB316464F
:100970000F4603EB0208154C04E0D4F8041319B138
:100980004B699847D4F8041300230D693046394663
:100990001A46A8470028F0D1D4F80433002BFBD026
:1009A0005B6998470028F7D0013607F50077B04516
:1009B000E8D1636E0020C4F80833BDE8F081034C31
:1009C0000020636EC4F80833BDE8F081501D002498
:1009D000002070470020704700207047034B93F8B9
:1009E0003003003818BF0120704700BF501D00249D
:1009F000816D03460A6A52681278FF2A09D090F87E
:100A0000F020013A52B2002A80F8F02006DD0120E1
:100A100070470822002083F8F02070470B6A0022FC
:100A200002205B681A707047836D1B6A5B681B78D5
:100A3000FF2B0AD190F9F030002B03F1FF3280F840
:100A4000F020D4BF0220012070470020704700BF73
:100A5000836D1B6A5B681B78FE2B0CD0FF2B08D1C3
:100A600090F9F0305A1E002B80F8F02001DD0120B3
:100A70007047022070470020704700BF10B5044641
:100A80006BF06CFD0146204689B2BDE81040FFF7CF
:100A90004BBB00BF38B50B4D00EB400005F5A7631D
:100AA000C40003EBC003254493ED027AD3ED037A2F
:100AB000E7EE007AB0EE670A6BF050FDD5F83835F6
:100AC000186038BD0400002002692DE9F843C368AE
:100AD00012EA030828D005460E464FF00047B8FA40
:100AE00088F327FA03F21B3BD24308EA02082A6183
:100AF000042B16D8DFE803F03B30251A0300B36A55
:100B0000002B3FD003F1FF3900231FFA89F9B362AC
:100B1000746A34B123682046494698476468002CBB
:100B2000F8D1B8F1000FDAD1BDE8F8837068002879
:100B3000F7D0696B036889B29847B8F1000FCED13E
:100B4000F2E7B0680028ECD0A96B036889B2984737
:100B5000B8F1000FC3D1E7E7F0680028E1D0E96BF6
:100B6000036889B29847B8F1000FB8D1DCE7306963
:100B70000028D6D0296C036889B29847B8F1000FD5
:100B8000ADD1D1E7EB6A1FFA83F9C1E78069B430D0
:100B900057F050BA10B590F83DE0BEF1020F76D094
:100BA000144690F83D208446012A02D1022280F8A2
:100BB0003D200C2921D8DFE801F007202020222049
:100BC00020203A2020205200DCF824003449DCF8B0
:100BD0000020C1633349C16490F8341001290CD05E
:100BE000012180F8341090F83510012952D00022EC
:100BF0004FF4006380F834204365002010BDDCF81A
:100C000028002749DCF80020C1632649C16490F818
:100C100034100129F1D0012180F8341090F83510FA
:100C20000129E4D13832214657F0F0FEE5E7DCF83F
:100C30002C001B49DCF80020C1631A49C16490F8FC
:100C400034100129D9D0012180F8341090F83510E2
:100C50000129CCD13C32214657F0D8FECDE7DCF853
:100C600030000F49DCF80020C1630E49C16490F8E0
:100C700034100129C1D0012180F8341090F83510CA
:100C80000129B4D14032214657F0C0FEB5E75FFAE2
:100C90008EF010BD3432214657F0B8FEADE700BFEC
:100CA0000D970908B5960908F8B5A0F507642379EA
:100CB000DB0725D5657994F8543805F001073D46E2
:100CC000FBB1D4F848341A68D36A5B08536294F8CD
:100CD000583823B1B4F862380133A4F8623885F08B
:100CE0000101606C60F09EFF012384F857380023F7
:100CF00084F8553884F85638A4F85E3884F85438A7
:100D0000F8BD94F85768012E03D194F8553884F84B
:100D100056382046FFF79EFA4EB9012385EA0301B3
:100D200084F85738606CBDE8F84060F07BBF002362
:100D3000394684F85738F5E738B5A0F5076400223E
:100D4000344D606C03685A62A1F12903302B31D80D
:100D500095F89F3495F8A0140133DBB2012B85F888
:100D60009F3409D9B4F85E3885F89F245B08A4F84D
:100D70005E384B1C85F8A03495F8A0240023082A7F
:100D8000A4F8603815D185F8A034B5F8A234013341
:100D90009BB2032BA5F8A23408D92379DB0705D52C
:100DA000E36A94F85E0843B3216B98470023A4F8E4
:100DB0005E3838BD5B396C290CD8B4F85E3885F8DC
:100DC0009F245B0843F08003A4F85E3895F8A034B4
:100DD0000133CFE794F85938002BCDD1012185F8A4
:100DE0009F34A5F8A234802384F85918A4F85E38FB
:100DF00085F8A01460F016FFBEE7E3696269D0547D
:100E0000E369E2680133B3FBF2F102FB1133E36102
:100E1000CCE700BF501D002438B55BF05FF80D49EA
:100E20000D4CD1F8FC20A4FB00400C4D42F0807228
:100E30000B4B800CC1F8FC204FF060420949E8667A
:100E4000C2F8B01F00225A601A6842F001021A600C
:100E500038BD00BF00ED00E083DE1B43501D0024C1
:100E6000001000E055CEACC570B505460A26084C0A
:100E7000013E00D170BD94F9000019F09FFB031EE4
:100E800004DB6178EA185172A278EA540434EFE77F
:100E9000CBDD0A0810B50E4CD4F8A4344BB194F84D
:100EA000B0249988186802F001031B0101FA03F3CA
:100EB00083615FF0A7FED4F80433002BFBD05B699D
:100EC00098470028F7D0636E0020C4F8083310BD9F
:100ED000501D00242DE9F041274D084611461A46C1
:100EE000D5F860433CB12668A3883469234095F85F
:100EF0005D4384B38BBBC3062FD10123C5F8E40443
:100F0000C5F8EC24C5F8D4344FF40073C5F8E834C0
:100F100061F0A4FB08BBD5F8D434002BFBD1D5F885
:100F2000346541F20D17D5F8F044DFF850803604EF
:100F3000A66041F28832E3680D21204603EA0803E7
:100F40003B43E3605BF064FE58B1D5F824350343BE
:100F5000C5F82435ECE7002BCDD14FF0FF30BDE8CC
:100F6000F081636903F4F053B3F5006FE0D16B6E69
:100F7000C5F80833BDE8F081501D0024C0E0FEFF35
:100F80002DE9F041214D10460A46D5F860433CB1A9
:100F90002668A1883469214095F85D437CB381BB04
:100FA000002161F0D7FB60BBD5F8D834002BFBD112
:100FB000D5F8346541F20D17D5F8F044DFF85080CC
:100FC0003604A66041F28832E3680D21204603EA28
:100FD00008033B43E3605BF01BFE28B1D5F82435E2
:100FE0000343C5F82435ECE7636903F4F053B3F524
:100FF000006FE6D16B6EC5F80833BDE8F0810029BB
:10100000CED14FF0FF30BDE8F08100BF501D00246D
:10101000C0E0FEFF30B597B000231F4C0DF1070272
:101020000890084608218DF8143007938DF8283071
:101030000B938DF83C301593184D84F8FC136944DC
:10104000099004F5597006959FED117BCDE90232A8
:10105000CDE910330122CDE91233022304928DF839
:1010600050200E938DED0C7B55F010FFD4F86433B7
:10107000186A0028FCD19DF80730FE2B03D0FF2B07
:101080000CBF0120022017B030BD00BFAFF30080BD
:101090000000000000000000501D0024510A040858
:1010A00030B40D4CBFF34F8F0C4BC3F85C42BFF311
:1010B0004F8FBFF36F8F0A4B0A4D03F13000DA797F
:1010C0002AB1597934F8112092B225F811200C3345
:1010D0008342F4D130BC7047A006012400ED00E04B
:1010E000BC22002460F0002400207047704700BF3D
:1010F000014858F02DBA00BF28230024084810B436
:10110000D0F8D835D0F80C4699691A682CB1234626
:1011100000F5BB605DF8044B18475DF8044B704761
:10112000501D0024014858F013BA00BF8C2300243E
:10113000084810B4D0F83C36D0F8704699691A685F
:101140002CB1234600F23C605DF8044B18475DF873
:10115000044B7047501D0024014858F0F9B900BFF6
:10116000F0230024084810B4D0F8A036D0F8D446B4
:1011700099691A682CB1234600F5D4605DF8044BD8
:1011800018475DF8044B7047501D0024014858F083
:10119000DFB900BF54240024084810B4D0F8043745
:1011A000D0F8384799691A682CB1234600F20470C8
:1011B0005DF8044B18475DF8044B7047501D002440
:1011C0002DE9F04784B08DF80F30431C00F09F806C
:1011D0000328044600F39B80824E642303FB0063D4
:1011E000D3F8D805002800F0928093F81956202DE6
:1011F00040F0878093F81856012D00F08280012579
:10120000D6F8507783F8185604E0D6F85037DB1B31
:10121000192B66D8856915F40045F6D14FF0640A9C
:10122000714B00974FEA41080AFB04FA41460AEB6A
:101230000309B24421234846CAF80C568AF81936E5
:1012400040238AF81A360DF10F03CAF81C56CAF863
:10125000FC350123AAF802360A2361F0FFFF0028BB
:1012600073D1BAF802369BB2FF2B40F29180DAF8C4
:10127000D815FF235D48AAF800364B685C4A034046
:1012800043EA08031A434A60642505FB046505E048
:10129000B5F802369BB2002B00F08C803A460A214A
:1012A00048465AF015FB60BBD5F8FC35D5F8D81583
:1012B00013F8010BB5F800268862C5F8FC35013A31
:1012C000B5F8023692B2013BA5F800269BB2A5F80C
:1012D0000236B5F802369BB2002BD9D0002AD7D1FE
:1012E0001EE064232020002103FB0463D3F81C26A6
:1012F00083F818160243C3F81C2683F8190683F8EE
:101300001A16B6F8543701339BB2A6F854370020AA
:1013100004B0BDE8F087D6F85037DB1B0A2B27D87E
:101320008A6912F08002F6D0B5F802369BB2FF2B24
:101330000ED94B682D4A13402D4A43EA08031A433D
:10134000FF23A5F800364A60A2E78AF81856D8E7C6
:10135000B5F8023625489BB24A68A5F80036DBB2DC
:10136000024048EA0343134343F000734B608FE7A6
:101370006423202103FB0464D4F81C3684F8182667
:101380000B43C4F81C3684F8191684F81A26B8E7FB
:10139000BAF80236DAF8D8159BB214484A68AAF8A7
:1013A0000036DBB2024048EA0343134343F00073C4
:1013B0004B6069E73946484661F0FCFE0346002869
:1013C0009FD1D5F8D82520240A48D461516801401E
:1013D0000120516085F8194685F8183685F81A36C7
:1013E00096E700BF501D002428230024009C00FC29
:1013F0000000FF0100E800FEB0F1FF3F00F0E680D2
:1014000003282DE9F047064682B000F39A808D4C00
:10141000642000FB0640D0F8D875002F00F09180C2
:1014200090F81956202D40F0868090F81856012D1E
:1014300000F08180012580F81856D4F8505704E058
:10144000D4F85007401B19287FD8B86910F4004819
:10145000F6D14FF064097C4F2220009509FB06F974
:101460004FEA410A0A994F44A14489F819064020DD
:10147000C9F8FC15514689F81A063846C9F81C8681
:10148000C9F80C86A9F802360A2361F05BFE002831
:101490006CD1B9F802369BB2FF2B40F2C080D9F86C
:1014A000D805FF236949A9F800364368684A0B400C
:1014B00043EA0A031A4342604FF0640808FB0648F7
:1014C00004E0D4F850375B1B0A2B25D8826912F050
:1014D0000402F6D0426AD8F8FC351A70B8F8023621
:1014E000D8F8FC25013B01329BB2C8F8FC25A8F8CE
:1014F0000236B8F80036B8F80226013B92B29BB229
:10150000A8F8003603B9A2BBB8F802369BB2002B8C
:101510006ED0D8F8D805D9E76423202003FB064312
:10152000D3F81C1683F818260143C3F81C1683F859
:10153000190683F81A26B4F8543701339BB2A4F87D
:101540005437002002B0BDE8F0876423202000213A
:1015500003FB0643D3F81C2683F818160243C3F88E
:101560001C2683F8190683F81A16E4E789F818860A
:10157000E1E7D8F8D80504E0D4F850375B1B0A2B14
:1015800026D8826912F08002F6D0B8F802369BB2F3
:10159000FF2B0BD943682F4A13402F4A43EA0A0313
:1015A0001A43FF23A8F800364260ADE7B8F80236C8
:1015B00028499BB24268A8F80036DBB20A404AEAE2
:1015C0000343134343F0007343609DE700207047DB
:1015D0006423202103FB0646D6F81C3686F818261D
:1015E0000B43C6F81C3686F8191686F81A26A2E7A9
:1015F0002946384661F0DEFD034600289BD1D8F825
:10160000D82520241548D46151680140012051603B
:1016100088F8194688F8183688F81A3692E7B9F823
:101620000236D9F8D8059BB208494268A9F80036B5
:10163000DBB20A404AEA03431343094A1A434260B1
:101640003AE700BF501D002428230024009800FC26
:101650000024FF81009C00FC0000FF0100E800FE68
:10166000002400822DE9F0410468D4E90435A86122
:101670001A7D1F681F2A49D9203A20212E6801FAB5
:1016800002F242F01802FA602A7D1F2A48D9203A55
:10169000202101FA02F242F01802F2606A68002189
:1016A0005868016038461160116841F010011160FE
:1016B00093F80880A269414665F078FC2D7AE269CA
:1016C0003046294665F072FC226A63689468184ABD
:1016D00012F80800515D5A686FF30F0222435A60F6
:1016E0003A5842F001023A50725842F001027250E8
:1016F0009A6842F440429A601A6842F001021A6005
:101700001A6842F400721A60BDE8F08120212E6848
:1017100001FA02F242F01802BA602A7D1F2AB6D8F6
:10172000202101FA02F242F01802B260B6E700BFCF
:10173000F0720B08D3B20F2B1FD8114B00B503F179
:101740007E0E02E00333734514D093F800C0844545
:10175000F8D193F801C08C45F4D102EB420209485C
:10176000997800EB82030430D96000EB8200197194
:101770005DF804FB00205DF804FB0020704700BF0B
:10178000F0DD0A080000002410B40C4C002304F51E
:10179000EB6C01E0152B0CD003EB430201331CF87A
:1017A00002108142F6D1144494F95A075DF8044BB3
:1017B00070474FF0FF305DF8044B7047501D002418
:1017C00030B5114D002305F1F80C02E001331A2B5E
:1017D00018D05CF833408442F8D10CEBC30EDC0027
:1017E0009EF804E08E45F1D102EB4202074B2544FE
:1017F00003EB8201043395F8FD4003EB8200CC60DB
:101800000C7130BD002030BD78DD0A0800000024D6
:10181000F0B1002310B504460E4894F804E000F53A
:10182000EB6C01E0152B11D003EB430201331CF8E4
:1018300002107145F6D183186179206893F95A270F
:10184000D3B20F2B02D8BDE81040B9E7002010BD7D
:1018500000207047501D002401380E4B0E4A00EB4B
:10186000C000D2F8D81003EB800310B4D3F8C43012
:1018700083B00A4CA34214BF022301231943C2F8C8
:10188000D810D2F8D82013400193019B03B05DF823
:10189000044B70470000002400440258000002403E
:1018A0000138F8B500EBC000124C1D46124B04EB9A
:1018B000800417460E46D4F8C400984214BFA120F5
:1018C000A02061F003FDB4F9DA00B909C4F8D460CE
:1018D000C4F8DC5061F00AFCB4F9DA30002B07DB05
:1018E00003F01F0001225B090449824041F82320D4
:1018F000F8BD00BF000000240000024000E100E04D
:10190000234B5B68C3F3080310B4DBB9EFF3118317
:10191000C3B9204B4FF0E02C5A6EDCF81800596E1A
:101920008A42F9D1996E8842F6D8DC6E4FF47A710A
:1019300001FB04F3181AB0FBF4F05DF8044B01FB53
:1019400002007047EFF31181102383F312884FF0E8
:10195000E0229469136913F4803F0E4B03D00120F9
:10196000C3F898079469586EC9B2D3F8982781F3E1
:101970001188D96E4FF47A73024403FB01F0001B07
:101980005DF8044BB0FBF1F003FB0200704700BFB1
:1019900000ED00E0501D0024BE4803780BB9012083
:1019A000704743682DE9F04F002BDFF8109387B0A4
:1019B000D9F8646018DD00F108050024B649D5F8AF
:1019C000F430BFF34F8F03F59072C1F85C322033CF
:1019D0009342FAD1BFF34F8FBFF36F8F0134436847
:1019E00005F586759C42EADB90F8F815AB4A049140
:1019F000A2FB0612AA4BAB4E5209DFF8C4A2A3FB0E
:101A00000213DB0803EB8303A2EB4303DAB206EB1A
:101A1000830B06F538730592009300239846049BC8
:101A2000984500F01481DAF81830DAF80470D3E938
:101A30003D45FFF765FF9C4999F89DE7012269182C
:101A40000190BEF1540F99F89C0702FA07F204EBDB
:101A5000410104EB400301D1A9F8A607994240F2E5
:101A60006A811F88174200F05F815F88174200F08B
:101A700070819F88174200F06E81DF88083317421B
:101A8000ECD11C1B99424FEA640440F25481281B9C
:101A9000452828BF452003EB4000834280F04F815A
:101AA00000251F46AC462946CDE9028EB3F800E07A
:101AB0000EEA020E8E451CD1B3F802E00EEA020EC9
:101AC000714540F01A81B3F804E00EEA020E714548
:101AD00040F01581B3F80680083308EA0208414552
:101AE00008D1984209D9B3F800E00EEA020E8E45FB
:101AF000E2D00233984200F2E580BCF1110FDDE93B
:101B0000028E40F21C81DCF1150200F11881674958
:101B1000D9F8B007D1F804339C4238BFC1F8044368
:101B2000019C231A002B14DB614B03449C4201D916
:101B300023460533C9F8B037D1F80433052B40F2FA
:101B40000C81053BDBB289F89C374FF0FF33C1F8BD
:101B500004333AB105FA02F2CCF1140C012505FA6E
:101B60000CF51543534BC5F3C43203EB8202D2F894
:101B7000C80105F01F0203EB8202D2F8C811C5F3B9
:101B80004412C5F3842503EB820241EA0031D2F806
:101B9000C82103EB850341EA0211D3F8C83141EAB9
:101BA0000321454B81EA1122D3F81C3A82EA121232
:101BB000013302F00F020F2A40F0A380B1F5803FFD
:101BC00080F09F80BEF1540F4FEA111147D03A4A7E
:101BD000B1F5606FC2F81C3A4DD0009B998196F820
:101BE00058300598834210D0DBF8082033689B1AE0
:101BF00033607368DBF830209B1A73600023CBF8E6
:101C00000830CBF8303086F8580033680133336041
:101C1000DBF808300133CBF808304FF6FF739942F8
:101C200007D1736801337360DBF830300133CBF8D0
:101C30003030009B08F101085C360BF15C0B14336B
:101C4000B8F1080F0AF1200A00937FF4E8AE0123EF
:101C5000194A012082F8183B07B0BDE8F08FB9F8A7
:101C6000A027B1F5606F02F10102A9F8A027124A7E
:101C7000C2F81C3AB1D199F8013003EB430309EBE8
:101C8000C30343445B7C0D2BA7D18023009A937739
:101C9000A5E700BF0400002000ED00E01F85EB5128
:101CA000CDCCCCCC30180020C7FFFF7F0000002433
:101CB00020A1070078DD0A08FC100020501D002438
:101CC0003C040020A3EB070E254F33F8021C4FEA1B
:101CD0006E0E11400EF1010E87FB0E87A7EBEE771B
:101CE0004FF0010E012FB8BF0127BD40BC44013F9A
:101CF0000EFA07F73D431F46D8E60433FAE60633EB
:101D0000F8E6BEF1540F04D1B9F8A0270132A9F8C2
:101D1000A027144A4FF6FF71C2F81C3AD2F8183ABD
:101D20000133C2F8183A5AE702331C1B99424FEAB2
:101D300064043FF6ACAE10B1013889F89C07BEF1DF
:101D4000540F7FF476AFB9F8A2370133A9F8A23760
:101D50006FE7043395E6063393E60023F3E600BF0E
:101D600056555555FC100020264B70B51A785B78F7
:101D70009A4242D1244E7368002B22DD06F10800FE
:101D80000025224CD0F8AC30BFF34F8F03F1E002B6
:101D9000C4F8683220339342FAD1BFF34F8FBFF3B8
:101DA0006F8F337813B1037F012B20D04269013547
:101DB000716800F586701368A94243F0010313604F
:101DC000E0DCFFF79DFD124BD3F81C4B002C0DDD22
:101DD00003F5326303EBC4041968083333F8042CA9
:101DE000C8689C4242EA0002CA60F5D170BD002377
:101DF00080F8FC30FEF72AF9D8E767F0DFFA002810
:101E0000B8D170BD501D00240400002000ED00E09A
:101E1000FC100020800AA0F58010522806D8044B40
:101E20001B5C0D2B02D8034AD05670470020704728
:101E300078DD0A08E0720B0860B182884FF0B0418B
:101E40004FF00043B2FA82F2D1F88000D34003434E
:101E5000C1F88030704700BF4FF0B042D2F88030F8
:101E6000D2F888100B4003F00103C2F8883023B188
:101E7000024BD3F8B407036818477047501D00247D
:101E80004FF0B042D2F88030D2F888100B4003F007
:101E90000203C2F8883023B1024BD3F8B8070368B5
:101EA00018477047501D00244FF0B042D2F88030E0
:101EB000D2F888100B4003F00403C2F8883023B135
:101EC000024BD3F8BC07036818477047501D002425
:101ED0004FF0B042D2F88030D2F888100B4003F0B7
:101EE0000803C2F8883023B1024BD3F8C007036857
:101EF00018477047501D00244FF0B042D2F8803090
:101F0000D2F888100B4003F01003C2F8883023B1D8
:101F1000024BD3F8C407036818477047501D0024CC
:101F2000F8B54FF0B043D3F88050D3F8882015406F
:101F300005F47875C3F888507DB1084F0126B5FACD
:101F400085F4C4F11F0407EB840306FA04F4D3F804
:101F5000B40703689847A543F1D1F8BD501D00248C
:101F6000F8B54FF0B043D3F88050D3F8882015402F
:101F700005F47C45C3F888507DB1084F0126B5FAB9
:101F800085F4C4F11F0407EB840306FA04F4D3F8C4
:101F9000B40703689847A543F1D1F8BD501D00244C
:101FA00030B1036882881B691A4214BF01200020E7
:101FB000704700BF10B1036882889A61704700BF04
:101FC00018B1838802681B049361704770B50D4691
:101FD00082B00446164640B101680C4B0C4A0B44D3
:101FE0009B0A02EB4303B3F8480261F06FF9C5F3B3
:101FF0008101C5F3411305F01302CDE90016A18854
:10200000206866F011F802B070BD00BF0000FEA7A6
:1020100078DD0A0800B1D9E770472DE9F84FC44FC1
:102020006423044603FB0073D3F8C065002E00F060
:102030006981D3F8C885B8F1000F04D098F906304B
:10204000002B40F05F81642303FB0473D3F8CC556D
:1020500025B195F90630002B40F05481631CDBB2AA
:10206000B8F1000F04D0152288F8073088F8062050
:1020700015B11622EB71AA714FF0640A308D61F030
:1020800025F929460AFB04FA404667F017F940464D
:1020900007EB0A09DFF8BC8299F8D23599F8D02508
:1020A000002B0CBF4FF01E0B4FF03E0B5946FFF7B5
:1020B000B1FF28469F4D594699F8D1255544FFF761
:1020C000A9FF4C22002128466BF0DEFAD9F8C03572
:1020D000994A5B689342C9F8D835DFF87C9240F0A2
:1020E000138159F01DFFD9F82030C3F30213434484
:1020F00093F85C3203F01F039FED907A9FED905AA6
:10210000B0EE084AD8406423F7EE003A4FF0000CD6
:1021100007EE900A03FB047340F21458F8EE677A56
:10212000B3F8D4A5C7EE275A07EE90AA9FED857A9B
:10213000F8EEE77AC7EE274ADFED837AB0EE007A51
:10214000E5EE877AA5EE875A25EE844A37EE856A52
:1021500074EEE72ABAF5C87F0CF1010ED5BF4FF433
:10216000967278226423322307EE90EAD8BF4FF4A8
:1021700016791344A2F13202F8EEE76AC8BF4FF4B1
:10218000827907EE903AD4BF41464FF4FA7166EE79
:10219000A56AB8EEE77AC7EE267A07EE102A01EBB9
:1021A0000902B8EEC77A37EE447A77EEE37AFCEEAE
:1021B000E77A17EE903AC7EE267AFCEEE77A17EE4A
:1021C000900A07EE909AB8EEE73A07EE902AF8EEFA
:1021D000E77A23EE243A83EE277A37EE453A32EE59
:1021E000C77AC3EE267A77EEE37AFCEEE77A17EE4B
:1021F000901AC7EE267A77EEE37AFCEEE77A17EECE
:10220000902A02F1020909EB010BB0EE467A07EEC3
:1022100090BAF8EE677AA6EEA77AF4EEC74AF1EE26
:1022200010FA7DDC43EA00095FFA89F9B9F10F0F72
:1022300078D841EA02091FFA89F9B9F1FF0F71D87C
:102240001B05000403F07F6392B200F47F00034398
:102250003E4843EA0C7300EA01210B431343642216
:10226000284602FB04740027C4F8DC350123C4F8B7
:10227000E075C4F8E435C4F8E875C4F8EC75C4F842
:10228000F475C4F8F87565F081FE94F81936202BC2
:10229000D9B21AD194F81836012B16D0242384F819
:1022A0001936D4F8D8351A6822F001021A601A6873
:1022B00022F480521A601A681A601A6842F0010209
:1022C0001A6084F8191684F81876002196F82B0005
:1022D00060F00CFF96F82B3001241D4D5A0903F0D5
:1022E0001F03002104FA03F345F8223096F82A0070
:1022F00060F0FCFE96F82A305A0903F01F039C4058
:1023000045F82240BDE8F88F59F00AFED9F81C3094
:10231000C3F30213984498F85C32EBE6F44619E7ED
:10232000013170E7BEF10F0FF8D1002397E700BF2E
:10233000501D002428230024001C0058286B6E4EDA
:1023400000001643002474490000704200FFFF00A3
:1023500000E100E078DD0A080044025808B10022DC
:1023600034E6704770B50E4C94F8F865AEB104F5DC
:102370008764002503E001352034B5420DD0237F6A
:10238000002BF8D0E06800220028F4D00135217D30
:10239000FFF71CFE2034B542F1D1012070BD00BF13
:1023A0000400002070B590F8EE311C09013C082CA7
:1023B0000FD81A4E054603F00F0306EB4402B2F89D
:1023C0006C0240FA03F2D20703D595F8F121012AF5
:1023D00001D0012070BD9A402644013A10406BF0B4
:1023E00003FB96F880320E4A034402EBC30452F812
:1023F0003320A38810691840ECD0002395F8EF2112
:102400000221204685F8F131FFF7E0FDD5F8502193
:10241000136843F008031360DBE700BF78DD0A08A8
:102420004425002470B5154BBFF34F8F144903F5B5
:102430008652C1F8683220339342FAD1BFF34F8FEE
:10244000BFF36F8F0F4C40F22A430C4AB4F84C5440
:1024500004F580602946FEF79DFB034618B1002372
:1024600084F84E3470BDD4F80064294604F58060C9
:1024700001227362BDE8704068F056B8E05B012449
:1024800000ED00E0501D0024014B43F82010704780
:102490005040005819481A4B01681A4A41F480719B
:1024A00030B482B00160D3F8F410FF24CA2041F4A4
:1024B0008031C3F8F410D3F8F41001F480310191A5
:1024C0005321019D546250625162D3F8D030DB0138
:1024D0000CD40C4B00220C495A659A65DA651A66D1
:1024E0005A669A66196502B030BC7047126D064B89
:1024F0009A42EED102B030BC704700BF004802588B
:102500000044025800400058316665422DE9F84FFA
:10251000D0F85C710446534B00F59676FDB227F077
:10252000FF09826800F1E00A103D4846D2F80080B9
:10253000A3FB05352D09294664F094FDD4F81C2130
:102540000023B2F5807F84F820317FD00DD8102A87
:1025500000F084805DD8012A46D0042A16BF6FF4AB
:1025600000616FF008013C230EE0B2F5805F71D08E
:10257000B2F5803F3BD0B2F5806F15BF6FF40061BC
:102580006FF008013C230423324608F11806404648
:1025900056F803C001EA0C01F150D4F81CB15946B9
:1025A00064F00EFABBF5807F2ED024D8BBF1100F5B
:1025B0003FD037D8BBF1010F02D0BBF1040F34D1AB
:1025C0004FF0080C336852462946484643EA0C034C
:1025D00033604023C4F8E83064F0E8FC3B6843F023
:1025E00010033B60BDE8F88F6FF00801CCE76FF097
:1025F00008013C23C8E7BBF5805F22D0BBF5803FD4
:102600001AD0BBF5806F10D108F11C064FF0080CF2
:10261000D8E7402A15BF6FF400616FF008013C2332
:102620000023B1E7BBF1400FCAD03C364FF4006C39
:10263000C8E74FF4006CC5E708F154064FF0080CEA
:10264000C0E708F11C064FF4006CBBE76FF008010F
:10265000042399E76FF40061042395E76FF40061A8
:1026600092E700BFABAAAAAA2DE9F04F474D85B06B
:102670002B781BB9012005B0BDE8F08F444B5C6E90
:10268000FFF73EF995F8F8350193002B00F0C7816C
:10269000404B05F5C065404E0027A3FB0423009581
:1026A0005B09A6FB03263D4AF60802F2347806EBE6
:1026B0008606A3EB4606D2F8483BC11A1346F2B28F
:1026C00003F6142A08EB860689460392B9F1000F37
:1026D00005DB009BD3F824314B4500F387814FF491
:1026E000B4732A4A03FB072393F82037002B00F02A
:1026F000BF80009D2A48D5F85C11AB681A68CBB240
:1027000021F0FF01103BA0FB030326481B09C35C1B
:102710000B44A9895C68D368A4B223EA0103C4F11D
:102720001604D360072C40F2A3801C4A0121D5F87F
:102730006451D2F81C3A8B46AE4602970133C2F878
:102740001C3A00222868944614E0BCF1140F2BDCDC
:1027500013F1080748BF03F117073B110CEB271CC7
:102760005F1E013102FA03F30BFA07F78C4247EAC6
:10277000030219D303468C425EF8040FA0EB030357
:10278000E3D8CCF115034FF0150CE9E70400002065
:10279000501D00241F85EB51CDCCCCCCFC1000206B
:1027A000ABAAAAAAF0720B08BCF1150F029F40F069
:1027B00013819F48C2F38423C2F3441100EB8303C7
:1027C00000EB8101D3F88C32D1F88C121B0243EA62
:1027D000011302F01F01C2F3C43200EB810100EBD0
:1027E0008202D1F88C12D2F88C220B4343EA0233D6
:1027F00083EA132282EA121202F00F020F2A40F03B
:10280000EB80C3F30F134FF6FF72934200F0E480A6
:10281000B3F5606F00F0EE80AAF80C3098F85820FD
:102820000398824210D0B168D8F80020521AC8F834
:102830000020D8F80420316B521AC8F80420002276
:10284000B260326388F85800D8F800200132C8F826
:102850000020B2680132B2604FF6FF72934207D196
:10286000D8F804300133C8F80430336B01333363D4
:10287000009C013708F15C085C3620460AF1140A16
:10288000FFF744FE04F5B4730093019BBB427FF451
:102890001DAF68490122002381F8182BC1F8483B7D
:1028A0006549D1F8083691F8D8261B6812F0020F56
:1028B000D1F81C171A6A0CBF0A4342EA81021A6255
:1028C000019B012B3FF4D6AE5B49D1F8703791F8EC
:1028D00040281B6812F0020FD1F884181A6A0CBF46
:1028E0000A4342EA81021A62019B022B3FF4C2AE04
:1028F0005149D1F8D83891F8A8291B6812F0020F75
:10290000D1F8EC191A6A0CBF0A4342EA81021A6232
:10291000019B032B3FF4AEAE4749D1F8403A91F802
:10292000102B1B6812F0020FD1F8541B1A6A0CBF4F
:102930000A4342EA81021A62019B042B3FF49AAED9
:102940003D49D1F8A83B91F8782C1B6812F0020F92
:10295000D1F8BC1C1A6A0CBF0A4342EA81021A620F
:10296000019B052B3FF486AE3349D1F8103D91F819
:10297000E02D1B6812F0020FD1F8241E1A6A0CBF5A
:102980000A4342EA81021A62019B062B3FF472AEAF
:102990002949D1F8783E91F8482F1B6812F0020FB0
:1029A000D1F88C1F1A6A0CBF0A4342EA81021A62EC
:1029B000019B082B7FF45EAE204A52F8203C92F82F
:1029C000B0001B68D2F8F41080071A6A4CBF42EAC4
:1029D00081020A431A624DE6164AD2F8183A0133C8
:1029E000C2F8183AAFB14FF6FF7317E7002005B0F1
:1029F000BDE8F08F12494A7802EB420201EBC202B5
:102A00003A44527C0D2A7FF407AF80228AF81E20B8
:102A100004E7294658220B486AF0D8FDE3E7194637
:102A20000122044BC3F8481B83F8182B22E600BF91
:102A300078DD0A08FC1000200400002004100020AB
:102A4000501D0024BC1B0020464A92F8781C013916
:102A500049B24B1C00F08480434B480103EB411109
:102A600000B5C2F87C1C811D13F801E003EB010CDA
:102A700092F8801C8E455BD09CF802E08E4555D0C4
:102A800000F10A0113F801E003EB010C92F8811C3C
:102A90008E4546D09CF802E08E4540D000F10E01F4
:102AA00013F801E003EB010C92F8821C8E4531D043
:102AB0009CF802E08E452BD092F8761C31B300F1E1
:102AC000120113F801E003EB010C92F8831C8E4510
:102AD00035D09CF802E08E452FD000F1160113F896
:102AE00001E003EB010C92F8841C8E4533D09CF876
:102AF00002E08E452DD01A3092F8851C13F800C0E4
:102B000003448C4521D0987888421DD05DF804FBA1
:102B10000CF1020CBCF80010A2F8881CCCE70CF1F8
:102B2000020CBCF80010A2F8921CB7E70CF1020CE2
:102B3000BCF80010A2F8901CA2E70CF1020CBCF843
:102B40000010A2F88A1CC8E702331B88A2F88E3C4A
:102B5000DCE70CF1020CBCF80010A2F88C1CCAE7F0
:102B6000704700BF501D002484E00A080120704710
:102B700038B5134D41F20D13124941F28832D5F8A0
:102B80003405D5F8F0440004A060E0680140204618
:102B90000B430D21E3605AF03BF838B1D5F82425FA
:102BA000034600201343C5F8243538BD606900F49E
:102BB000F050A0F50060B0FA80F0400938BD00BFC9
:102BC000501D0024C0E0FEFF08B5FFF7D1FFA0B103
:102BD0000B4BD3F8600358B1026893F85D338088DB
:102BE000126910402BB9003818BF0120013840B2DB
:102BF00008BDB0FA80F04009F8E74FF0FF3008BD9B
:102C0000501D0024C74BD3F8B414D3F8B82470B5C2
:102C10008C0F93F8F05C100EC2F3072C83F8984CDD
:102C2000C1F383640001012D83F8994CC1F3016461
:102C300083F89A4CC1F3074483F89B4CC1F30724F3
:102C4000C9B283F89C4CC2F3035483F89D1CA3F8CB
:102C50009E0CC2F3C030B3F89E1C89B241EA040155
:102C6000C2F30344A3F89E1CC2F3403183F8A04C86
:102C7000C2F3803483F8A10C4FF0000083F8A24C1B
:102C800083F8A31CC2F3003183F8A41CD3F8BC144E
:102C900083F8A50C40F2EF80022D00F0C3802A20BB
:102CA0004FEA4C0C83F8B14CC1F3C01201F07F0124
:102CB0000CF07E0C83F8B2CC4FF0010C93F8B24CC0
:102CC0001443D3F8C02483F8B24CD40F83F8B31C58
:102CD000910D83F8B44CC2F3417401F00C01C2F3BE
:102CE000815583F8B54CC2F3826483F8B64C83F8FF
:102CF000B71C93F8B71CD3F8C444294383F8B71C16
:102D0000C2F3405183F8B81C002183F8B91CC2F308
:102D1000004183F8BA1CC2F3C03183F8BB1CC2F374
:102D2000803183F8BC1CC2F3403183F8BD1CC2F370
:102D3000003183F8BE1CC2F3812183F8BF1CC2F3AB
:102D40000121C2F3460283F8C01CC4F3074183F893
:102D5000C12C220E090283F8C2CC83F8C42CC4F320
:102D60000722A3F8C61C2406B3F8C61C89B2114377
:102D7000A3F8C61CD3F8C814C3F8C84C0C0ED3F87B
:102D8000C82C42EA0442C3F8C82C0A0AD3F8C84C3B
:102D900002F47F422243C1F30724C9B2C3F8C82C0E
:102DA000D3F8C85CD3F8CC242C43C3F8C84C83F8C0
:102DB000CC1C110E83F8CD1C110C0906C3F8D01CD5
:102DC0001102D3F8D04C0A4601F47F01214392B29C
:102DD000D3F8D044C3F8D01CD3F8D01C0A43C3F8AE
:102DE000D02CC4F30352D3F8D01C41EA1461C3F8C9
:102DF000D01C93F8D41C1143C4F3072283F8D41CCD
:102E0000210A01F47061A3F8D61CB3F8D61C89B26C
:102E10001143C4F34602A3F8D61C83F8D82C83F8D8
:102E2000D9CC70BD1204C1F3072C0D0E02F47C1234
:102E3000C3F8A82CC1F30742D3F8A84C44EA0524F0
:102E4000C3F8A84CD3F8A84C22434FF40074C3F83D
:102E5000A82CD3F8A82CC3F8E84C013240F10004A8
:102E6000A40244EA92549202C3F8E44CC1F38034C1
:102E7000C3F8E02C14E74FEA8C2CC1F3C265940030
:102E80000CF44062C1F3072C04F47F74C3F8A82C3F
:102E9000D3F8A82C1443CA0BC3F8A84C02F00602BE
:102EA000D3F8A84C44EA9174C3F8A84CC1F3026467
:102EB00083F8AC5C012583F8AD4CC1F3425483F830
:102EC000AE4CC1F3824483F8AF4CC1F3C03483F8F5
:102ED000B02C93F8B02C224383F8B02CD3F8A84C34
:102EE00093F8B02C93F8A06C023205FA02F2B540C8
:102EF000D617A2FB052EC3F8E85C05FB06EE04FB23
:102F00000EEE0134A2FB0424A644520AC1F380341D
:102F100042EACE52C3F8E02C4FEA5E22C3F8E42C1A
:102F2000BEE600BF501D00240E4838B5D0F860330F
:102F30000D4614463BB1196890F85D239B880969DA
:102F40000B4052B15BB9FFF75DFE074A4FF40073C7
:102F50000020126C2A60238038BD002BF3D14FF083
:102F6000FF3038BD501D0024F02900245FF098B9CF
:102F70005FF096B92DE9F8432422D0F85051002390
:102F80008168C0F8D02104462A6800F5A87622F0AE
:102F900001022A602B606B60AB604279C0F8D831C7
:102FA00080F8CC31C0F8D031C0F86831C0F8D431E5
:102FB000C0F870319302C0F8541103F48053BC4937
:102FC000C0F8583113038D4203F40053C0F85C314C
:102FD0004FEA022303F48063C0F8603100F0AB8154
:102FE0002379D80703F0020100F14081002940F065
:102FF0007181C4F8641194F8F0314BB1D4F8783190
:1030000043F00803C4F878314FF40043C4F8883122
:1030100012F00802D4F8D03100F06E81002B00F0DD
:10302000AD8124233046C4F8D0312B6823F001034E
:103030002B6059F09DFB012817D0D4F87831002B74
:1030400040F09F816B68304623F490436B60AB681F
:1030500023F02203AB60AB6843F00803AB602B683E
:1030600043F001032B6064F0BFF894F8048018F07B
:10307000010F6FD0D4F82C71002F00F06C81002369
:103080004FF4807C04F13C09E7632366E36648461D
:10309000C4E91133C4E91433C4E91933D4F8343121
:1030A000C4F8B8304FF48063E3644FF48033C4E96C
:1030B00016C365F005F9484655F008FBD4F8D4313D
:1030C000C4F8C891202B666741D1E368626998B261
:1030D000EAB3B0FA80F14909C8B394F8CCC1BCF1A5
:1030E000010F34D04FF0220CC4F8D811A4F8AC0171
:1030F0000120C4F8D4C1DFF8D0C1C4F8A821C4F8B5
:1031000078C0DFF8C8C1C4F88C10C4F87CC0DFF800
:10311000C0C184F8CC01C4F888C094F870C084455C
:103120000CD084F8700094F87100012800F031810F
:103130004FF4006384F87010C4F890301023C4F882
:10314000D831002384F8CC312023C4F8D0317B68F7
:10315000C4F8443118F0020F00F08680D4F83051E2
:10316000002D00F0EC80D4F83821002304F1B407DE
:10317000C4F8C0303846C4F8C830C4E92D524022E3
:10318000C4F8BC204FF48062C4F8C4204FF48032ED
:10319000C4E93333C4E93633C4E93833C4F8D4203E
:1031A00065F08EF8384655F091FA002840F0A3807B
:1031B000404B4149414A8D4218BF9D42404801F170
:1031C0006001C4F8C4710CBF01230023C4F8EC6093
:1031D000954208BF43F001033032854208BF43F0F7
:1031E00001036030954208BF43F0010330328D4245
:1031F00008BF43F0010301F56871954208BF43F031
:10320000010302F55C72854208BF43F0010300F53B
:103210006870954208BF43F0010330328D4208BF09
:1032200043F001036031954208BF43F0010330329F
:10323000854208BF43F00103954208BF43F00103F4
:1032400030328D4208BF43F00103954208BF43F07E
:1032500001033BB91B4BEB1AB3FA83F35B09002B59
:1032600000F0AF8000236B60BDE8F8830423C4F84E
:10327000643171B10C23C4F86431D3077FF5BBAE60
:10328000D4F878314FF4803143F00203C4F8801150
:1032900028E0D3077FF5AFAED4F8783143F00203CE
:1032A000C4F878314FF48033C4F88031A3E600BF0E
:1032B000000C00581000024028000240400002406C
:1032C00058000240B804024095970908C9970908B8
:1032D000CD9709080823D107C4F864317FF58BAE78
:1032E000D4F8783143F00103C4F878314FF4003357
:1032F000C4F87C317FE6FEE70BB194F8CC2124239F
:1033000084F8CC213046C4F8D0312B6823F0010377
:103310002B6059F02DFA01283FF4A7AED4F878318C
:10332000002B32D16B68304623F490436B60AB685E
:1033300023F02A0392E60423C0F8743150E6D4F84F
:10334000DC311A6842F080021A601A6842F04002CA
:103350001A60BDE8F883D4F8DC311A6842F4807250
:103360001A609A6842F001029A601A6842F02002DC
:103370001A601A6842F010021A60EBE684F8CC3149
:103380004FE6304659F0ECFB5CE6304659F0E8FB7E
:10339000C8E79BB2484605F1240155F037FB0028E9
:1033A0007FF4CCAE84F8CC012B6843F480732B609F
:1033B000AB6843F00103AB60AB6843F04003AB6024
:1033C000C5E66B6050E700BF38B50409013C082C26
:1033D0001AD80F4D00F00F0305EB4402B2F86C024F
:1033E00040FA03F212F0010210D00122254402FA41
:1033F00003F3013B18406AF0F7FA95F88032054A6A
:10340000034402EBC30038BD002038BD104638BD70
:1034100078DD0A08442500242DE9F047984D05EB96
:103420000013D3F8F44C002C00F08F80B3F8FE7C2E
:1034300006464FEA001938465FF048FF01227B0933
:1034400007F01F07023BBA40082B0FD8DFE813F044
:10345000BF00C700CF00D700DF000900E700EF0082
:10346000B7008849CB6F23EA0203CB6705EB09035A
:10347000013693F8F80CF6B2FFF7A6FF074610B135
:103480001223C671837105EB090393F8F90CFFF75A
:103490009BFF824610B11323C671837105EB0903AC
:1034A00093F8FA0CFFF790FF804610B11423C67111
:1034B00083714D4450462E2195F8FC2CFEF7AAFD51
:1034C00095F8FD2C40460E21FEF7A4FD95F8FB2C47
:1034D0002E213846FEF79EFD23686B4A23F0010338
:1034E0009442236033D0694B9C423ED1654BD3F864
:1034F000902042F48042C3F89020D3F8902022F428
:103500008042C3F89020E36843F00043E360A3687F
:1035100023F4F073A3602368DA0716D4A1685C4A29
:103520005C4B0A401343A360E368DB0042D5E268CA
:10353000594B134043F0E863E360236823F40063CE
:103540002360236D23F001032365BDE8F0874D4B15
:10355000D3F8982042F48052C3F89820D3F89820EA
:1035600022F48052C3F89820CDE74C4B9C4213D0F4
:103570004B4B9C4263D04B4B9C426ED1414BD3F89A
:10358000982042F48012C3F89820D3F8982022F4AF
:103590008012C3F89820B6E73A4BD3F8902042F453
:1035A0000042C3F89020D3F8902022F40042C3F8E0
:1035B0009020A8E7236843F480532360B7E731499C
:1035C000D1F89C3023EA0203C1F89C304EE72D4924
:1035D000D1F8983023EA0203C1F8983046E7294928
:1035E000D1F8903023EA0203C1F890303EE7254934
:1035F000D1F8943023EA0203C1F8943036E7214928
:10360000D1F8803023EA0203C1F880302EE71D494B
:10361000D1F8843023EA0203C1F8843026E719493F
:10362000D1F88C3023EA0203C1F88C301EE715492B
:10363000D1F8883023EA0203C1F8883016E7114B2D
:10364000D3F8982042F40052C3F89820D3F8982079
:1036500022F40052C3F8982055E7134B9C427FF4A4
:1036600052AF03F50C33D3F89C2042F02002C3F88C
:103670009C20D3F89C2022F02002C3F89C2042E733
:10368000501D002400440258003001400038004022
:10369000E0FFBF8F07000020FFFF39D8003C00404B
:1036A00000340140005001400014005808B51D20AE
:1036B000FFF78AFE10B190F9063053B11E20FFF7D4
:1036C00083FE10B190F9063003B108BD5523C380C5
:1036D00008BD5523C380F1E72DE9F04FDFF8CCA2F8
:1036E0009BB09AF8541D31B1A74B93F8084320467C
:1036F0001BB0BDE8F08F01200AF59E657C228AF898
:10370000540D284669F0C0FFDAF87C6C4FF4805203
:103710009AF8767C3468CAF8F824CAF8F0441FB1E5
:103720004FF48042CAF8FC2401224FF4003CC5E962
:1037300004C29AF82025002A00F095810322934FB5
:103740008AF82025FA6CD60340F132810AA858F095
:1037500021FC0C988E4A010AA2FB012109094D00A7
:103760006668A8428B4A02EA060242EA01026260E7
:10377000226842F00302226080F0F880DAF85017E5
:10378000DAF85027521A022AFAD9002282497E4ECC
:103790000492A260E2681140D6F80C2341F48051F3
:1037A000E1607E49A1FB021B41F288324FEA5B2BAC
:1037B00002FB0BFB5A46002A00F0BE80616B013A07
:1037C0000806F8D5764A7449A2634FF4D572A26010
:1037D000E268114041F208120A43E260BBF1000FB7
:1037E00009D05A46616B11F0450F02D0890440F1AF
:1037F0008681013AF6D10022CAF82C25A260664AD9
:10380000E1680A4042F48052E2605A46002A00F021
:103810009380616B013A0D06F8D5614A0025A263D9
:1038200004994FF6FE72914200F2B281DFF868917E
:103830005C4FDFF86C8100222046A26041F2371213
:10384000E16801EA09010A433721E26041F2883266
:1038500059F0DEF9002871D1A76041F22912E16820
:1038600001EA09010A43E260BBF1000F08D05A46A1
:10387000616B11F0450F01D0880404D5013AF7D1EE
:103880004FF080505AE0626B510700F10D83C4F88D
:1038900038806169049A002902F101020492049AB5
:1038A00003DB4FF6FE708242C5D904984FF6FE72D4
:1038B000904200F28F834A0040F16E812268012716
:1038C0009307CAF8287500F0F7820022DFF8C88055
:1038D0002046A26041F20232E16801EA08010A438F
:1038E000E26059F037FA48BB626904F1180304F149
:1038F0001C09CAF85C25A2690193CAF86025E2692F
:10390000CAF86425226ACAF8682541F20312A06049
:10391000E16801EA080104F120080A43E260BBF112
:10392000000F09D0626B12F0450F02D0910440F1F4
:103930005483BBF1010BF5D14FF0004001228AF80E
:103940002025DAF824250243CAF824252A24204613
:1039500086F808431BB0BDE8F08F616805460D4A44
:103960000A406260226842F0030222600E49B0FB06
:10397000F5F5B1FBF5F1DAF850070231DAF8502726
:10398000121A9142FAD800E70000002400440258BD
:10399000598B4F01002CC0FFC0E0FEFFD34D6210D9
:1039A000C5002000000010C110210100501D00249E
:1039B000BD6AB96AFE6A11F47C7F7A6BC1F30510A7
:1039C000CBD0C2F3CC0206F0010605F0030507EEEA
:1039D000900A06FB02F2012DF8EEE76A07EE102AC4
:1039E000BAEEE97A00F08982022D00F0AD80002D58
:1039F00040F083823A68950640F1F9843968B7EE61
:103A0000006A3A6BC1F3C101C2F30803584A07EEDA
:103A1000903ACA40F8EEE77A77EE867A37EE877A00
:103A200007EE902AB8EEE76AC6EE267A67EE877A46
:103A30005049F7EE006A504D0A6B0A6B096BC2F3EE
:103A4000064307EE103AB8EEC77A37EE267AC7EE8D
:103A5000876AFCEEE67A17EE900A010AA5FB01518F
:103A600009094D007CE6454A944200F06982444AC7
:103A7000944200F081829AF8900CFFF7A5FC8346EF
:103A80009AF8920CFFF7A0FC05469AF8880CFFF70D
:103A90009BFC9AF88A3C04469AF88C9C9AF88E8C87
:103AA0000193BBF1000F05D058469AF8912C0E21D6
:103AB000FEF78CFA2DB128469AF8932C0E21FEF7CA
:103AC00085FA2CB120469AF8892C0E21FEF77EFA51
:103AD000002F40F0F4810021B6F904005FF006FBEE
:103AE000B6F90420002A07DB02F01F040121520965
:103AF0002448A14040F82210DAF8F0441EE6626B38
:103B0000520700F1AA82626BD3071AD4626B570680
:103B100001D54022A263002201251B492046CAF894
:103B20002C55A260E268114041F237120A43372156
:103B3000E26041F2883259F06BF800283FF470AE31
:103B40009EE60122A26356E6DFED107A87EEA66AB2
:103B50003A6BC2F3080307EE903AF7EE005AF8EE1C
:103B6000E77A77EEA57A77EE877A67EE867A5FE76F
:103B70000090D00300440258598B4F01007000524E
:103B80000024024800E100E0C0E0FEFF0024F44A07
:103B90000499914200F21E822268900700F08C8105
:103BA000DAF82875032F7FF490AEDAF84C15DAF8BE
:103BB0005025A069000DCAF83005880F8DF828003F
:103BC000C1F383608DF82900C1F301608DF82A00EC
:103BD000C1F307408DF82B00C1F30720C9B28DF85F
:103BE0002C008DF82D10110DADF82E10C2F30341ED
:103BF0008DF83010C2F3C0318DF83110C2F380312E
:103C00008DF83210C2F340318DF83310C2F3003119
:103C10008DF8341000218DF83510002F40F07A8196
:103C200040F6FC7101EA8202DAF8541542EA917218
:103C30000E92C1F3C2628DF83C20C1F302628DF88E
:103C40003D20C1F342528DF83E20C1F382428DF8EF
:103C50003F20C1F3C2328DF8402001220E989DF81A
:103C600040C010440CF0070C0CF1020C00FA0CF0F0
:103C70009DF830C00CF00F0CCAF8380502FA0CF2AF
:103C8000CAF83C25520A00FB02F2CAF84025DAF8CD
:103C900034054FF4007BDAF858254FF001094FEA5C
:103CA0000048C1F38030CAF844B58DF84100C1F333
:103CB000C61001F07F018DF8420020468DF84310B8
:103CC000D10F8DF84410C2F341718DF84510C2F345
:103CD00082618DF84610C2F383518DF84710C2F30C
:103CE00040518DF8481000218DF84910C2F3004171
:103CF0008DF84A10C2F3C0318DF84B10C2F38031F9
:103D00008DF84C10C2F340318DF84D10C2F30031E4
:103D10008DF84E10C2F381218DF84F10C2F30121AE
:103D2000C2F346028DF850108DF8512041F207126F
:103D30008DF85290C4F80880E16821F48F3121F4A5
:103D40009F7121F001010A430721E26041F28832AC
:103D500058F05EFF00287FF4F1ADC4F808B041F2DE
:103D6000101BE2681021204622F48F3222F49F7249
:103D700022F0010242EA0B02E26041F2883258F07E
:103D800047FF002840F0BC80DAF850976269910143
:103D900000F18F80402310212046A360E26822F4C6
:103DA0008F3222F49F7222F0010242EA0B02E2609B
:103DB00041F2883258F02CFF00284CD1C4F808801A
:103DC00041F23712E168204621F48F3121F49F71CE
:103DD00021F001010A433721E26041F2883258F0B4
:103DE00017FF002837D14FF0FF3240236262A362F1
:103DF00001301F28FCD9E26A2046A14922F0FF02C7
:103E000042F06302E2620022A260E268114041F2E5
:103E10000D120A430D21E26041F2883258F0F8FE9B
:103E2000C8B90AA806E0DAF85027A2EB0902013265
:103E300000F01781626B12F4957F626B40F0148181
:103E40001204F0D500F12001D4F8802040F8042BB2
:103E50008142F9D1E7E7DAF82425CAF82425894A0E
:103E60000121A263DAF8242502432046CAF824255A
:103E70008AF820154FF40071814AA160E1680A4078
:103E800041F21011114341F28832E160102158F0E3
:103E9000BFFE00283FF45AAD7A4AA2630122CAF855
:103EA00024058AF8202551E504224FF08050A263B2
:103EB00044E54FF40060D2E74FF080603EE50198A2
:103EC000FFF782FA20B19AF88B2C0E21FEF77EF8CC
:103ED0004846FFF779FA20B19AF88D2C0E21FEF7AB
:103EE00075F84046FFF770FA9AF88F2C00283FF4D7
:103EF000F2AD0E21FEF76AF8EDE5DFED637A25E617
:103F0000604AA263DAF824250243CAF824258AF815
:103F100020951BE5012F4FD11204DAF8541502F455
:103F20007C1242EA11420E924FF40072CAF83C250C
:103F30000E9A01329202CAF83825CAF84025A6E640
:103F4000524AD2F8D41021F48031C2F8D410D16F83
:103F500041F48031D167D16F21F48031D167D2F83B
:103F6000D41041F48031C2F8D410D2F8D42002F435
:103F700080320392039A7EE5444AD2F8DC1021F4A1
:103F80000071C2F8DC10D2F8841041F40071C2F85C
:103F90008410D2F8841021F40071C2F88410D2F891
:103FA000DC1041F40071C2F8DC10D2F8DC2002F41D
:103FB00000720292029A5EE5324A01214FF080506F
:103FC000A263DAF8242542F08052CAF824258AF840
:103FD0002015B3E44FF08070B0E4626B520700F13B
:103FE0000F82626BD30700F106822269D2B2032AE4
:103FF00040F00382264AA263626912F4604F0AD03D
:10400000540400F10B8212F4004F14BF4FF480509F
:104010004FF4803092E4120C19492046CAF8342536
:104020001204A260E268114041F209320A43E260E0
:1040300058F090FE00287FF481AC6169019BCAF8BA
:104040004C151A68CAF85025D9F80000CAF854056A
:10405000D8F80000CAF85805ABE50422A263FFF7C0
:10406000CABB4FF00040FAE6130700F1D581626B3E
:10407000910700F1CF81626B920615D5C8E100BFB0
:10408000C0E0FEFFFF0FE01F0024744A0044025806
:10409000C5002000D4F88010DAF8502740F8041B3F
:1040A000A2EB09020132DCD0626BD304F2D4DDE969
:1040B0000C120A984FF4007B4FEA11490B9B5FFAF0
:1040C00082FE4FEA102C29F0FF091BBA49EA0E09BB
:1040D0002CF0FF0CDFF860E34CEA106CC4F838E019
:1040E000C0F3811EC0F340101FFA8CFC8DF814E061
:1040F0008DF81500C8B2ADF816C006938DF81C00F7
:10410000C1F30720C1F303518DF81D0020468DF83F
:104110001E10C2F38521ADF820908DF82210C2F355
:1041200001218DF82310C2F3031102F00F028DF864
:1041300024108DF825209DF83B20BA498DF82620C3
:10414000C4F808B0E268114041F210120A4310218D
:10415000E26041F2883258F05BFD00287FF49CAEAB
:104160009DF82420012F9DF82510D2B2DAF8FC9496
:10417000C9B200F0B5800322CAF848058AF82025A4
:10418000B9F5004F00F0C580B9F5804F00F005810A
:10419000B9F1000F00F0C480DAF8242542F0006283
:1041A000CAF82425DAF8242502B39F494FF4007297
:1041B0002046A163A2609B4AE1680A4041F21011C7
:1041C000114341F28832E160102158F021FD0028AE
:1041D00000F0DE80944AA2630122DAF82415084335
:1041E000CAF824058AF82025FFF7B0BBDAF80405E1
:1041F000DAF8F4240328DAF8F834DAF8001509D8E4
:10420000DAF848E5BEF5007F04D0BEF5807F14BF24
:10421000042002201A4363680A43844919400A4370
:1042200042EA0902DFF8FC910243204662604FF443
:104230000072A26041F21012E16801EA09010A432A
:104240001021E26041F2883258F0E2FC0028C1D12E
:10425000012241F20D1B8AF82025DAF8503701932C
:104260000AE0DAF824250243CAF82425DAF85027B0
:10427000019BD21A013243D0C4F808800D21E268B4
:10428000204602EA090242EA0B02E26041F2883269
:1042900058F0BEFC0028E4D1626902F4F052B2F595
:1042A000006FE3D1002F624F4FF00101CAF82405DF
:1042B00007F1980218BF0225CAF81C05044607F149
:1042C000A80C8AF820158AF8F05C07F110050FCACF
:1042D00087E80F009CE80F0085E80F00FFF737BB69
:1042E0000A4305D00322CAF848B58AF8202547E7D3
:1042F0004FF48072CAF8482503228AF820253FE748
:104300004FF000410122CAF824158AF82025FFF752
:104310001DBBDAF8242542F08052CAF8242541E773
:104320006269002000219201CDE90A015CD40AA84B
:104330005EF0A6FA024628BB0B9AD30365D5C4F8F3
:10434000088041F23712E1682046DFF8D8B001EA70
:104350000B010A433721E26041F2883258F058FCE1
:10436000024678B9C4F80890E16841F20612204686
:1043700001EA0B010A430621E26041F2883258F05B
:1043800047FC0246DAF824150A43CAF8242509E74F
:1043900001228AF82025FFF7D9BA0020626900219E
:1043A000CDE90A0190011FD40AA85EF069FA02461D
:1043B0000028E7D10B9A510327D5C4F8088041F2B1
:1043C0003712E1682046DFF85CB001EA0B010A43CE
:1043D0003721E26041F2883258F01AFC0246002888
:1043E000D0D10222A260BFE74FF40062CAE7DFED3E
:1043F000117AFFF7ABBB0122A2630120FFF79EBA3F
:1044000004221046A263FFF799BA4FF08062B9E721
:10441000202024E5022022E5082020E54FF400506A
:10442000FFF78CBAC0E0FEFFFF0FE01F002CC0FFBB
:10443000042200240024744C3A0F00182DE9F047A0
:10444000344C94F8900CFEF7BFFF064694F8920C9B
:10445000FEF7BAFF054694F8880CFEF7B5FF94F80E
:10446000768C074694F88CAC94F88A0C94F88E4CB1
:104470000EB11823F3800DB11923EB800FB11A236D
:10448000FB80B8F1000F15D138460121FDF792FDF0
:10449000FDF764FF30460121FDF78CFD2846FDF74E
:1044A00089FD3046FDF75AFF28460121BDE8F04757
:1044B000FDF754BFFEF788FF814608B11B23C38078
:1044C0005046FEF781FF804608B11C23C38020467A
:1044D000FEF77AFF044638460CB11D23E380012124
:1044E000FDF768FDFDF73AFF4846FDF763FD4046DE
:1044F000FDF760FD2046FDF75DFD01214846FDF713
:104500002DFF40460121FDF729FF01212046FDF73F
:1045100025FFBFE7501D0024F8B50E4C94F8F87540
:10452000A7B104F5C064C7F109070925013D0FD003
:10453000A6683079FEF748FF94F8DC10F27908B1EC
:10454000FDF744FDAF4204F5B474EFD10120F8BD8E
:10455000AB68FFDE0400002010B51B4C94F8590D29
:10456000FEF732FF28B11F210022C1802021FDF774
:104570002DFDD4F8A4344BB194F8B0249988186870
:1045800002F001031B0101FA03F3836194F9772C14
:1045900000210320FDF7CEF850B1D4F860335BB1B1
:1045A000196894F85D239B8809690B4012B91BB9FF
:1045B000012010BD002BFBD1FFF78EF80028F7D1AA
:1045C000636EC4F8083310BD501D002410B5807808
:1045D000FEF7FAFE90B10A494FF0410C0446002262
:1045E000D1F8603D80F806C00133C1F8603D20215C
:1045F000C371FDF7EBFC2368A2889A6110BD00BF70
:10460000501D0024F8B50446EFF31185502383F3C1
:104610001288D0F830311B6803F001031BB1EDB2F2
:1046200085F31188F8BDD0F8D021D0F8D4110A4311
:1046300002F02102212AF2D0D0E90912914250D091
:1046400090B24BD8194623691B1A9BB2A162002174
:1046500084F8E011D4F8D0112029E0D1A16989189B
:10466000DDD0B3FA83F25209002BD8D094F8CC01F4
:104670000128D4D02120A4F8A6314FF0010CC4F8B1
:10468000D821C4F8D001D4F8C401D4F85061C4F8DA
:10469000A011A4F8A43184F8CCC160B31B4F90F8EA
:1046A00034E0C7631A4FE64502650764194FC764D3
:1046B0000AD090F8357080F834C0674515D04FF4B3
:1046C000006380F834204365102100222023C4F8C1
:1046D000D81184F8CC21C4F8D031A0E7081A83B2ED
:1046E000B4E7012380F8E03199E706F1280254F09D
:1046F0008DF90028E8D100234022326284F8CC31C1
:10470000B36843F08003B36089E700BF6D97090881
:1047100091970908CD970908BFF34F8F0549064BBC
:10472000CA6802F4E0621343CB60BFF34F8F00BF4F
:10473000FDE700BF00ED00E00400FA051C481D4A3B
:10474000C1681D4B10B44FF6FF0485B021401B4CCF
:104750000A43C260D3F8D010D3F8DC20C4F8641D3B
:1047600042F00052C3F8DC20D3F8DC2002F0005203
:104770000192019AD3F8DC2042F08042C3F8DC2099
:10478000D3F8DC2002F080420292029AD3F8DC20B7
:1047900042F00042C3F8DC20D3F8DC3003F00043E1
:1047A0000393039B05B05DF8044BFCF735BB00BFDA
:1047B00000ED00E00005FA0500440258501D0024F9
:1047C00008B51D480023C0F88430BFF34F8F4369FC
:1047D00023F480334361BFF34F8FD0F8803043F62A
:1047E000E074C3F34E3CC3F3C90E4FEA4C1C0CEA11
:1047F0000401734641EA8372013BC0F874225A1CDB
:10480000F8D1ACF1200C1CF1200FF0D1BFF34F8F89
:10481000BFF36F8FBFF34F8FBFF36F8F43690022DA
:1048200023F400334361C0F85022BFF34F8FBFF32E
:104830006F8F72B6FFF770FF00ED00E003689B0A10
:10484000A3F58013522B54D870B5364C14F803C01E
:10485000BCF10D0F4CD843794FF04C0E3248022476
:104860009E080EFB0C0E0CEB8C03B440DEF8685D6A
:104870000CEB4303B6463344EE6800293FD0344383
:1048800000EB83067167C6F88420EC60EFF31185B6
:10489000502383F312882C2202FB0C010B6F4BB3C5
:1048A0001A1DC1F89430214B0CEB8C01204C0CEB01
:1048B000410189000C4410310B4453F8041F09B125
:1048C00011600A1DA342F8D10023EDB2136085F3F5
:1048D00011882C2303FB0C03D3F89430C3B14C2371
:1048E00003FB0C03D3F8682DD36843F00103D360B6
:1048F00070BD70470D4B02FB0C322432D4E726EA20
:104900000404EC6000EB83046167C4F88420BDE715
:104910004C2303FB0C00D0F8682DD36823F001036F
:10492000D36070BD78DD0A08501D0024C01D00242E
:10493000E01D002403689B0AA3F58013522B00D9C5
:1049400070470E4AD35C0D2BFAD84FF04C0C10B4C4
:104950000B4C42790CFB03400223D0F8680DDA407F
:104960009340C26829B922EA03035DF8044BC3608F
:10497000704713435DF8044BC360704778DD0A0845
:10498000501D002403689B0AA3F58013522B10D8F6
:10499000084AD25C0D2A0CD84079022306494FF010
:1049A0004C0CD8400CFB02128340D2F8682DDB433C
:1049B0001361704778DD0A08501D00240149024840
:1049C000FCF782B8C01D00240000014001490248E4
:1049D000FCF77AB8C01D00240000014002494FF0E6
:1049E0008040FCF771B800BFEC1D0024014902486B
:1049F000FCF76AB8181E0024000400400149024870
:104A0000FCF762B8441E0024000800400149024837
:104A1000FCF75AB8701E0024000C0040F8B5164D83
:104A2000164E2A69EB681A404FF00040B2FA82F342
:104A3000EAB120FA03F3012A6FEA030302EA030151
:104A40002B610A46F2D1D6F874718FB1013F002371
:104A5000BFB2C6F87431D6F8704134B1236820462D
:104A6000394698476468002CF8D10022DCE7F8BD8D
:104A7000EF6ABFB2EFE700BF00100040501D0024F6
:104A800001490248FCF720B8F41E0024000401404C
:104A900010B5064C064804F5D271FCF715F804F57C
:104AA000FE710448BDE81040FCF70EB8501D00240C
:104AB00000040140001C004001490248FCF704B812
:104AC000201F00240018004001490248FBF7FCBFEA
:104AD000781F00240020004001490248FBF7F4BF82
:104AE000A41F00240040014001490248FBF7ECBF2D
:104AF000D01F00240044014001490248FBF7E4BFF5
:104B0000FC1F0024004801402DE9F0414FF42572BC
:104B10008EB00021734868F0B7FD734B734D4FF0B2
:104B20000008D3F8F02040F27D27A5F55B7605F666
:104B3000F41442F00102C3F8F020D3F8F02002F0A0
:104B400001020092009AD3F8E82042F00102C3F873
:104B5000E820D3F8E82002F001020192019AD3F88C
:104B6000E82042F00202C3F8E820D3F8E82002F07F
:104B700002020292029AD3F8E82042F00402C3F83B
:104B8000E820D3F8E82002F004020392039AD3F855
:104B9000E82042F00802C3F8E820D3F8E82002F049
:104BA00008020492049AD3F8E82042F01002C3F8F5
:104BB000E820D3F8E82002F010020592059AD3F815
:104BC000E82042F02002C3F8E820D3F8E82002F001
:104BD00020020692069AD3F8F02042F00202C3F8AF
:104BE000F020D3F8F02002F002020792079AD3F8DF
:104BF000E82042F04002C3F8E820D3F8E82002F0B1
:104C000040020892089AD3F8E82042F08002C3F8E4
:104C1000E820D3F8E82002F080020992099AD3F83C
:104C2000E82042F48072C3F8E820D3F8E82002F4C8
:104C300080720A920A9AD3F8F02042F48032C3F8C4
:104C4000F020D3F8F02002F480320B920B9AD3F8C4
:104C5000F02042F40032C3F8F020D3F8F02002F440
:104C600000320C920C9AD3F8F02042F48022C3F860
:104C7000F020D3F8F03003F480230D930D9B55F80A
:104C80002810002354F83320914226D001330E2BF4
:104C9000F8D1002008F107085EF018FBB845EED106
:104CA0004FF0000840F27D2755F82810002354F8F3
:104CB000332091420CD001330E2BF8D1002008F1A3
:104CC00007085EF003FBB845EED10EB0BDE8F081F9
:104CD00006EBC303B3F8640DF1E706EBC303B3F8C7
:104CE000640DD7E7C01D002400440258E4E00A0820
:104CF000800AA0F5801052280DD8074B1A5C0D2AA7
:104D000009D8064B4C2101FB0233D3F8682D1368F8
:104D100043F001031360704778DD0A08501D00243A
:104D20001F4B984210B50ED003F5806398420AD00D
:104D30001C4A03F58043984218BF904203D003F504
:104D4000806398421BD157F0EBF8174B1749DC6989
:104D5000DA69C4F3022CC2F3022201EB0C0393F8CC
:104D60005C3203F01F03D8400F4B11491B69C3F39A
:104D7000C03342EAC303CB5C03FB00F010BD57F025
:104D8000CFF8094B0949DC69DA69C4F30214C2F3AC
:104D900002120B1993F85C3203F01F03D840E3E7CB
:104DA00000000140004001400044025878DD0A083C
:104DB000CC720B082DE9F04F002391B0AD4C00935D
:104DC000AD4BAE4FA3F55D66AB4D4FF00009AC4B5C
:104DD000D5F800A093F8F6204FEA9A23A3F58013A4
:104DE000522B00F2CE80F35C0D2B00F2CA80012A18
:104DF00017F903B000F01081022A02D1BBF1080FAD
:104E00003BD14FF00008414658460EF0D9FC0EF059
:104E10005FFD90F900C0BCF1000F18BFBCF1540F4A
:104E200014BF4FF0010C4FF0000C40F0E98008F186
:104E300004081FFA88F8B8F1100FE4D1009B002B8A
:104E400000F0AA808B4A0AE0F35C0D2B0ED8FB56CB
:104E50005B450ED002F58672944200F0998091680D
:104E60000B689B0AA3F58013522BEDD900235B45F9
:104E7000F0D14B7969799942ECD109F101091C35DE
:104E8000B9F1080FA3D1009B04F586740133042BFC
:104E9000009399D17B4A4FF0010B92F8F83502F557
:104EA000876901330393039B5B4567D0744B99F883
:104EB0001020D9F80C6093F80A310092002E5DD0D2
:104EC000704AD6F800A055686F48B288002D50444B
:104ED00001924FEA902040F3AE80664A002405E03C
:104EE000013402F58672AC4200F0A2801168814262
:104EF000F6D1604B4FF48672019D02FB0434009B97
:104F00000322C9F80C6089F81030019BC9F81840D9
:104F1000B3FA83F7C7F11F035800C9F80430B27120
:104F200086F807B002FA00F6A16C0122D4F854C04A
:104F3000314302FA00F002FA03F3A164216D014348
:104F4000D4F8AC0021654F490E7899B2002E00F0DC
:104F50004E8143EA0C036365CAF81850FBF7A2F8C8
:104F60000BF1010B2046FBF771F809F1200940F223
:104F70000113BBF1090F29F8043C94D111B0BDE82D
:104F8000F08F013A012A7FF678AF4FF0000B38E737
:104F9000BCF1000F7FF471AFA86800223B4904E028
:104FA00001320C31102A00F088834B689842F7D107
:104FB00052B269795046FCF703FC354A4068002339
:104FC00051680133884208D0102B02F124023FF4CB
:104FD00054AF516801338842F6D1DBB22D4A013B10
:104FE00003EBC30302EB830393F9E030002B7FF460
:104FF00044AFC9EBC909204B03EB8903A36042E727
:10500000009B002B7FF41EAF09F101091C35B9F19B
:10501000080F7FF4DCAE36E7BBF1010F3FF4F1AED1
:1050200009F101091C35B9F1080F7FF4D0AE2AE768
:10503000042C00F049824FF48671124A01FB0522CC
:1050400011690491002900F00483906001304FF051
:1050500054019C46C4B20D4882F8101182F81141E7
:105060006A1C08494A60049A11689768029151794C
:10507000002216E00C00002048EB0A08E0720B0842
:10508000482E0024040000200000FEA70400002495
:10509000C40000240000002401320C30102A00F06B
:1050A0000C8343689F42F7D152B20298CDF814C0E6
:1050B000FCF786FB944B4FF48672DFF87C8202FB90
:1050C00005310022059B0132D0E90170C1E907706A
:1050D00041464868874208D0102A01F124013FF474
:1050E0004DAF486801328742F6D1D2B28749013AC2
:1050F00002EBC20201EB820292F9E01000297FF478
:105100003DAF4FF4867182F8E1400693542401FBD1
:1051100005F37F4882F8E0409A107E49059300FB32
:1051200002F201F560747848C2EBC20C02EBC202D5
:10513000184401EB4C1104EB4212C0F80CA0C0F86B
:10514000B410C0F8FC203322C0F8B8208C22C0F87C
:105150000021714A0298D418FFF7E2FD069B062B46
:1051600000F0B981072B6D496D4B6E4A18BF1A4686
:105170006D4B18BF0B464FF48671DDF808A0B0FBED
:10518000F3F3B0FBF2F2013B5F48013A01FB05018A
:105190009BB2A1F8BC20A1F874302366059B03F1F3
:1051A000580100F10803504619440023A4F8583070
:1051B0006366E36561F082FDDAF8003043F0800356
:1051C000CAF80030049B5B791A4606930C2A1CD857
:1051D000DFE812F003021B001B001B00DD011B00B7
:1051E0001B001B00BB011B001B001B009601C7F12D
:1051F0002F072D0402FA07F3324643EA0C036365D6
:10520000CAF81850FAF74EFFAAE63F4A4FF48673E1
:1052100002984FF0000A03FB05230222CDF828A0D4
:1052200059690368079123F00103CDF834A0CDF844
:105230003CA00360602308934FF480730E93012316
:1052400009930A23CDE90B3208AA61F0B9FB07994B
:10525000B1F5807F00F0288240F24081B1F5805F97
:1052600000F00E82B1F5803F00F00482B1F5806F4E
:1052700015BF4FF4006308234FF03C0A4FF0040AB7
:10528000029A183252F80A100B4342F80A30049B73
:105290001879002840F0CB81029A136843F001038B
:1052A00013600023D8F804200133974200F0BC813A
:1052B000102B08F12408F5D14FF0FF330027134AD3
:1052C00003EBC30302EB8303D3F8C400174B9842EC
:1052D00014BFA120A0205DF0F9FF069A0C2A00F26D
:1052E000A081134B03EB4203B3F8B0CE4FF48673A7
:1052F000054A104803FB0523DDF808E000F532619C
:10530000A3F818C0002320E00400002000000024BF
:105310006B4CA407E05301240C000020D0DD0600F4
:10532000449508001055220040771B000000024001
:1053300078DD0A08FC100020C4000024964500F027
:105340009D810133042B00F0BB8151F83320002AEA
:10535000F4D1D0F81C2B0132C0F81C2B00EBC30099
:10536000029ADB00C0F8202B1944384623469022CD
:105370008F884CEA070C0027A1F804C0C349FCF74A
:105380008FFA4FF48673C24A40214FF4403CC14823
:1053900003FB052A4FF48052DAF81C502B6843F0C7
:1053A00010032B602B6843F014032B60C4E91F77B4
:1053B000C4E92777C4E92977DAF82030A167E9B290
:1053C000C4F89430069310394FF48063C4F898C041
:1053D000A0FB01014FF4804CC4F88430DAF8B80027
:1053E0000909059BC4F8900025F0FF00DAF80C804D
:1053F000C4F8882008F118020491029008F11008FE
:10540000226703F17002A44B1A44DAF8B430C4F8EE
:105410008CC0636761F0CAFDD5F800C0059BC4F875
:1054200020C0D5F814C003F1B8029B4BC4F824C0C7
:10543000D5F804C01A44069BC4F828C0D5F808C0A3
:105440000499C4F82CC0D5F80CC0C4F8DC304FF473
:105450008063C4F8C870C4F8CC304FF40033C4F88B
:1054600030C0C4F8E0300298C4E93077C4E9397735
:10547000C4E93B774FF40067DAF80031C4F8B8802C
:10548000C4F8D0704FF48047C4F8D830DAF8FC3054
:10549000C4F8D470C4F8BC3061F088FD2B68D6F82D
:1054A00000A063636B69A3636B68E363AB68236409
:1054B000EB6863642B6843F010032B602B6843F0A8
:1054C00014032B60B5881AE50323744A82F80B3164
:1054D00011B0BDE8F08F724A724B4CE6102900F013
:1054E000E98000F2BD80012900F0E280042915BFA7
:1054F0004FF4006308234FF03C0A4FF0000ABFE668
:1055000002984FF4867262494FF0020A036802FB68
:1055100005124FF4805123F00103516108AA036082
:1055200000230A930D930F93602308934FF4807325
:105530000E93012309930A23CDE90B3A61F040FA57
:105540004FF0040A4FF400639AE602984FF4867213
:105550004F494FF0020C03684FF0040A02FB05129A
:105560004FF4807123F00103516160220360002336
:105570000E910A930D930F930123CDE908230A237B
:1055800008AACDE90B3C61F01BFA082378E60298E3
:105590004FF486723E494FF0000A03684FF0020E46
:1055A00002FB0512102123F00103CDF828A0516160
:1055B00008AA03606023CDF834A008934FF48073E9
:1055C000CDF83CA00E93012309930A23CDE90B3EAD
:1055D00061F0F6F94FF4006352E602984FF48672D8
:1055E0002B494FF0000A03684FF0020E02FB051230
:1055F000012123F00103CDF828A0516108AA03601E
:105600006023099108934FF48073CDF834A00E9372
:105610000A23CDF83CA0CDE90B3E61F0D1F9082377
:105620002EE64FF0000C61E6DFB27B1E47E6FDF789
:10563000CBFE824638B1049B0221DA79FCF7C6FC26
:105640005423AAF80630029A536C43F4004353647F
:1056500022E60223114A82F80B3111B0BDE8F08F27
:10566000402915BF4FF4006308234FF03C0A4FF068
:10567000000A05E608234FF03C0A01E6DB0073E66A
:105680004FF400634FF0040AFAE500BF0100000088
:1056900004000020ABAAAAAA0C000020482E002477
:1056A000882A1100A0BB0D0008234FF0040AE7E58B
:1056B0000823E5E54FF40063E2E500235B68FFDEC5
:1056C00000239B88FFDE00BF2DE9F04FB04D8FB067
:1056D00095F80C81B8F1000F03D100200FB0BDE8A0
:1056E000F08F00222F2140460EF048F90646002890
:1056F000F3D090F80590A74FD0F800A0A7F84C94ED
:10570000FCF786F80028E8D0D0E901430193002C8B
:10571000E3D0DFF8B8B20022594601E0102ADCD00D
:105720004B68013224319C42F8D1D2B29A4B013AF3
:1057300002EBC20203EB820292F9E030002BCCD1E3
:105740002F2150460293A2F8E010C7F800A4FFF7FB
:10575000E7FA924A029B904280F0FA801A460123AF
:10576000039350460292FFF7DBFA029A039BC7F8B5
:1057700004248B49B0FBF3F2120A8A48A1FB0221F0
:105780000022C7F81024C7F808240A090909A0FB59
:105790000202C7F80C145208A5F810215200A5F80F
:1057A0000E2197F83D2402F0FF01002A00F0DE8070
:1057B000022250467C4987F83D2456F087FE01229C
:1057C000404687F8482487F83E2487F83F2487F826
:1057D000402487F8412487F8422487F8432487F837
:1057E000442487F8452487F8462487F8472487F817
:1057F0003D24FDF7E9FDC5F8140128B12F21C18032
:105800004E21F279FCF7E2FB684A0021019B4FF43C
:10581000806CC5F82411B9F10C0FC5F83411C5F826
:105820003C11C5E94643C5E95111D2F8D80040F012
:105830000100C2F8D800D2F8D80000F001000490AE
:105840000498D2F8D80040F00200C2F8D800D2F88C
:10585000D82002F002020592059A4FF04002C5F8E6
:1058600020214FF48052C5E94AC24FF48042C5F866
:1058700030214FF40032C5F838214FF00302C5F84B
:10588000402176D84A4A02EB4902B2F8CC8EC24691
:10589000484A08F108084849C5F8502107EB880232
:1058A000C2F80014594600224B68013224319C4250
:1058B00062D0102AF8D14FF0FF32374B02EBC20210
:1058C00003EB8202D2F8C4003C4A904214BFA120EC
:1058D000A0205DF0FBFC0022DBF8043001320BF16C
:1058E000240B9C424BD0102AF6D1002007EB8807EE
:1058F000534660223249FBF7D3FFD7F8000452F039
:10590000E5FE00287FF4E9AEB479002760260C900C
:1059100063004A4606A9274803F002030893E30000
:10592000CDE9066703F00803002600270993CDE9B7
:105930000A675DF035F800287FF4CFAEA30749462B
:105940001C481ED556F0CAFEB0FA80F04009C5E6E4
:105950005046FFF7E5F91B4A1B490244A1FB02121E
:10596000920D531E9AB2531C0393FAE687F83C1427
:105970001EE78A4688468BE7D2B2013A9DE7D0B24D
:10598000B4E756F017FDB0FA80F04009A6E600BF74
:10599000482E0024501D002400000024006CDC026E
:1059A000598B4F01ABAAAAAA5421002400440258E3
:1059B00078DD0A0850210024602F002400000240F6
:1059C000D502000000366E01819F5E16C4000024DF
:1059D000830AA3F58013522B00D970472DE9F041BB
:1059E00015460F4AD65C0D2E17D80E4C4FF04C08BA
:1059F000013908FB064789B2C7F8741DFFF790F913
:105A000007F66C51B0FBF5F2013AD7F8680DC7F80C
:105A10006C2DBDE8F04156F059BDBDE8F08100BFE6
:105A200078DD0A08501D0024830AA3F58013522B49
:105A30006ED82DE9F0439046714A85B0D65C0D2EA4
:105A400063D84C256F4F044606FB05F507EB0509A7
:105A5000D9F8683D834258D00139C9F8680D083536
:105A600089B2C9F8741DFFF75BF907F66851002386
:105A7000B0FBF8F00D440138C9F8703DC9F86C0D61
:105A8000C5E9023399F8A53D03F0FF02002B40D091
:105A90004C25022305FB061105FB06750431D5F8DC
:105AA000688D85F8A53D404656F010FD012385F828
:105AB000B03D85F8A63D85F8A73D85F8A83D85F859
:105AC000A93D85F8AA3D85F8AB3D85F8AC3D85F844
:105AD000AD3D85F8AE3D85F8AF3D85F8A53D4A4B17
:105AE0009C4219D0B4F1804F16D0A3F57C439C4260
:105AF00012D003F580639C420ED003F580639C4274
:105B000060D003F578439C425CD005B0BDE8F083DB
:105B1000704789F8A42DBBE74C2303FB067393F869
:105B2000A42D012AF1D0022283F8A52D374AD8F8F6
:105B300008100A40C8F80820012283F8A52D002289
:105B400083F8A42D00224C232F4903FB06730392F4
:105B50008845CDE901224FF0020283F8A52DD8F83F
:105B60000420D8F8083028D001F58061884524D079
:105B700022F07002C8F80420254A90450DD0B8F1F3
:105B8000804F0AD0234902F50062904518BF88452E
:105B900003D002F54062904503D123F08003C8F89A
:105BA00008304C230121002203FB067383F8A51D56
:105BB00083F8A42D05B0BDE8F08317491140C8F85B
:105BC0000410EAE74C2303FB067393F8A42D012A83
:105BD0009BD0022283F8A52D0C4AD8F808100A4061
:105BE000C8F80820012283F8A52D002283F8A42DEF
:105BF0000A4B9C42A6D003F578439C42A2D084E78E
:105C000078DD0A08501D0024000001408800CEFF06
:105C100000040040000800408FFF0FFF000C004010
:105C20002DE9F0410468A30AA3F58013522B03D891
:105C30002C4DEE5C0D2E01D9BDE8F0812046FFF71A
:105C4000F3FE4C22284B02FB063393F8A52D012AC4
:105C500010D00023254951F8332094421CD0013341
:105C60000E2BF8D1012100205DF040FA204B0122DB
:105C70001A60E1E70221D3F8682D83F8A51D1D4BBA
:105C800091680B40062BE4D0B3F5803FE1D0136858
:105C900043F001031360DCE705EBC3050126144F55
:105CA00095F8664D314604F01F0520465DF01EFA5A
:105CB0001B2C4FEA541806FA05F547F8285009D06E
:105CC0002E2CB9D131462C205DF010FA4FF48053C0
:105CD0007B60B1E7314619205DF008FA4FF00073A0
:105CE0003B60A9E778DD0A08501D0024D8EA0A08BD
:105CF00000E100E007000100F8B5134C94F89E3471
:105D000003F0FF05002BF9D1104B012693F89031D9
:105D100084F89E6403B9F8BD0D4AB4F89C74138EE0
:105D200034320C483946FAF735FF034610B184F88F
:105D30009E54F8BDD4F85044324639460548636253
:105D4000BDE8F84064F0F0BB501D0024482E00244C
:105D5000A0060124A021002437B590F86738044636
:105D6000032B2FD10023204D8DF807309DF80730ED
:105D700094F868289A4201D803B030BD9DF80730E6
:105D800005EBC30393F898318BB181F0010383B124
:105D90009DF8073005EBC303D3F89401FCF70AF92B
:105DA0009DF807300133DBB28DF80730DEE70B4694
:105DB000EDE79DF8073005EBC303D3F89401FCF73A
:105DC000FFF8EDE7D0E910039B7903F00103994256
:105DD00004D003B0BDE83040FCF7ECB803B0BDE838
:105DE0003040FCF7EDB800BF482E002438B504461B
:105DF00000790D4650B1FDF7E7FA08B10323C380DF
:105E0000E2792946BDE83840FCF704B938BD10B541
:105E100004462221FFF7EAFF2046FEF7B3FD2046A5
:105E20000121BDE81040FEF785BD10B504460121F3
:105E3000FFF7DCFF00212046BDE81040FEF77ABDE9
:105E400038B510F8133CA0F66C041BBB94F8583816
:105E50008BBBD4E909239A421CD05A1CA169A262C7
:105E6000CB5C21695B008A4228BF002243F40073A7
:105E7000A262A4F85C380A2384F85A38012384F813
:105E8000583894F86738012B01D0042B02D1606C8C
:105E9000FFF7CBFF94F85438002B6DD194F85538A8
:105EA0000133DBB2092B84F8553825D12046BDE8F3
:105EB0003840FAF7CFB994F95A586DB1B4F85C1874
:105EC000013D20464B0801F00101A4F85C38FFF7C2
:105ED00043FF84F85A58DDE7D4E9092384F8585879
:105EE0009A42D7D194F86738012B01D0042BD1D135
:105EF000606CFFF78CFFCDE70A2B3DD194F8573843
:105F00002BB9B4F85E3843F00103A4F85E38237966
:105F1000D9070AD5B4F85E08820501D4C30718D49E
:105F2000B4F864380133A4F864380122002384F8FB
:105F3000542894F8572884F85538012A1CD16179DF
:105F4000606C84F8573801F00101BDE838405BF01F
:105F500069BEE36AC0F3470013B1216B9847E4E7D9
:105F6000E3696269D054E369E2680133B3FBF2F19B
:105F700002FB1133E361D8E738BD2DE9F84310F88F
:105F8000133CA0F66C047BB1B4F8603801339BB2CB
:105F9000082BA4F860381BD90021606C84F85918CC
:105FA000A4F860185BF03EFE374F97F8D481B8F143
:105FB000000F03D101212046FFF7CEFE94F8583898
:105FC0004BBBD4E909239A4204D1002387F8D4318A
:105FD000BDE8F883B8F1020F12D808F1010814BF28
:105FE000FF237F2387F8D481A4F85C380823606CF2
:105FF00084F85A38012384F85838BDE8F84314E788
:106000005A1CA169A262CB5C2169DBB28A42EBD344
:106010000022A262E8E794F95A685EB3B4F85C988B
:1060200097F8D55119F001010BD0012D01D80121AC
:1060300003E0AB1E012B09D800212046FFF78CFEA0
:1060400004E015F0FD03F2D0012BF6D00135EDB2DE
:10605000032D87F8D551BBD9013E4FEA59090023DA
:1060600076B2A4F85C9887F8D53184F85A68002E87
:10607000A7D0ADE7D4E909239A42A9D1606C84F88E
:106080005868BDE8F843C2E6482E00242DE9F043E5
:10609000BFB0BFF35F8FA24A0020516A0346044697
:1060A00021F4803151620146C2F89400C2F8983060
:1060B0000133C2F89C10112BC2F8A010F6D10523B1
:1060C000C2F89430536A43F480335362BFF34F8F66
:1060D000BFF36F8F9348944A9449121A67F076FA87
:1060E0009348944A9449121A67F070FA934BDA6D08
:1060F000042A00F0FB8005D8012A00F09383022ACD
:1061000000F0A683864A00238D4C0120D2F8881027
:106110008C4E41F470018C4DC2F8881020602361D0
:10612000216841F0800121602168014321602168DC
:1061300041F480312160216841F480512160A361E4
:10614000E3612362A362E36223636363A363E363A4
:1061500023646364216821F4802121607B492366E4
:10616000C1F808014FF000614FF6FF00784B9160D5
:10617000D16801400B43D36055F0B0FEA3690246DD
:106180000F20C3F30323A169334493F85C3203F077
:106190001F0322FA03F3C5F80C3351F015FF6D4AC3
:1061A000D36813F0040FD36840F0A2806A4B00213B
:1061B000684A0591D96A21F00101D962DB6A03F0CE
:1061C00001030593936943F440439361936903F496
:1061D00040430593059B93699B04FCD54C22002109
:1061E0000EA85E4C67F050FA5D4A42F20303126853
:1061F000B3EB124F4FF000030893A4F1140308BF50
:106200001C46E268002A4DD0534B5249D86A20F010
:106210000100D862DB6A03F0010308938B6923F461
:10622000404313438B618B6903F440430893089BFD
:10623000484A93699F04FCD5414B4FF44037494885
:106240000321D3F8E02042F08002C3F8E0200122CD
:10625000D3F8E03003F080030793079B87610D9B21
:1062600000910193002361F0DFFE022322690EA852
:10627000CDE91733A3781E9201221993A3881A93AC
:10628000A3791B93E3791C93237A1D9300231F9317
:106290004FF48033CDE90E2355F068FB03283BD043
:1062A00098B1FEE72B4A2C4B916941F44041916132
:1062B000926902F440420892DA6A42F00102DA621C
:1062C000DB6A03F001030893B1E7274B1A6812F069
:1062D0000E0F4DD11A6822F00F0242F002021A602E
:1062E0001B6803F00F03022B42D0FEE7DC6509E7D1
:1062F00023F007031D4C43F00203D360D4F850177A
:1063000006E0D4F850375B1AB3F57A7F3FF64EAF0C
:1063100053689804F5D549E772B6FEF7FDF900BF5A
:1063200000ED00E000000000B84B0000EC0E0C088F
:10633000000000200400002055840C080040005894
:106340000044025878DD0A08000000240080005153
:106350000003FA05004802580004005824030024F2
:106360000010005C001C025800200052501D002448
:106370006E4A936903F070033F2B05D8936923F0AD
:10638000700343F040039361684AD36903F07003DC
:106390003F2B05D8D36923F0700343F04003D3614A
:1063A000624AD36903F4E063B3F5806F05D2D36921
:1063B00023F4E06343F48063D3615C4A136A03F01F
:1063C00070033F2B05D8136A23F0700343F040039A
:1063D0001362564B9A69140705D49A6922F00F028A
:1063E00042F008029A61514A936923F47063936101
:1063F000136898017FF579AF136941F288304C4CEE
:1064000023F0070343F003031361D4F8501705E0AA
:10641000D4F850375B1A834200F2BC81136903F051
:106420003803182BF4D1936903F00F03082B05D917
:10643000936923F00F0343F0080393613D4A136807
:1064400003F00F03022B0BD9136823F00F0343F063
:1064500002031360136803F00F03022B7FF445AFB0
:10646000324A936903F07003402B05D9936923F0F6
:10647000700343F0400393612C4AD36903F0700327
:10648000402B05D9D36923F0700343F04003D36157
:10649000264AD36903F4E063B3F5806F05D9D36965
:1064A00023F4E06343F48063D361204A136A03F06A
:1064B0007003402B00F266811C4F55F00FFD034620
:1064C000D5F83803BA69B969C2F30322164496F8BD
:1064D0005C2202F01F02D340C5F80C3351F074FD6A
:1064E000002840F09E811023159017900EA80E935F
:1064F00055F03CFA002840F044813B680E4A43F0D6
:1065000080033B60D7F8F43043F00203C7F8F4305F
:10651000D7F8F43003F002030493049B136A43F0AA
:1065200001031362054BD4F850170CE000440258E5
:10653000501D0024002000520004005800E2040016
:10654000013B3FF4E9AED4F850279142F8D0D4F89B
:106550005027D4F850379B1A0A2BFAD9C04C4FF465
:1065600080224FF440130EA80E924FF000082F9394
:1065700060F010FFD4F8EC3041F20302B949032671
:1065800043F002030EA80227C4F8EC30D4F8EC3034
:1065900003F002030393039BD4F8943043F0020307
:1065A000C4F89430D4F8943023F00203C4F8943043
:1065B0000B68AD49B2EB134FAC4BAD4A28BF0A464E
:1065C0005A601A6822F47C5242F400521A601A6827
:1065D00042F060021A600E96CDE92B8860F0DAFE78
:1065E0004FF4E0430EA8CDF8E4800E93CDE9258862
:1065F00060F0D0FE18230EA8CDF8B8800E93CDF829
:10660000CC8060F0C7FED4F8D43005220EA843F445
:106610008033C4F8D430D4F8D430CDF8588003F4A3
:106620008033129611970293029B4FF480330E939E
:1066300021934FF4FA73CDE90F230423CDE9148895
:10664000139360F0A7FE4FF400230EA80E934FF4AF
:106650000033369360F09EFED4F8E0303A464FF4B3
:106660008071844843F00103C4F8E030D4F8E0308E
:1066700003F001030993099B4346CDE9006861F0EB
:10668000D3FC23693A467C4823F0FE7343F08873B9
:106690002361D4F8E03043F00403C4F8E030D4F8C8
:1066A000E03003F004030693434606994FF400716B
:1066B000CDE9006861F0B8FC236923F07E4343F024
:1066C000FC43236155F00AFC6C4B6D4A4146C5F80A
:1066D0000C031846D21A66F0D7FF6A486A4A6B491B
:1066E000121A66F073FFBFF35F8F694D4646694C1F
:1066F00001276B6A23F480336B62C5F8948023E032
:10670000002946D0D4F80090637A103414F8060CAF
:106710001B0643EA007343EA410314F8051C43EAED
:10672000814314F8041C43EA414314F8031CC5F8E0
:106730009860013643EA0143C5F89C90032E43F06C
:106740000103C5F8A03026D06368217A002BD7D08A
:10675000D4F800900029D7D129F01F01A3EB01083C
:10676000B8F1200F38BF4FF02008404666F06CFFAC
:10677000431E014607FA03F0804508BF1946C9B217
:10678000C2E7FEE7136A23F0700343F0400313628D
:1067900092E6FEE7A9E50523C5F894306B6A43F459
:1067A00080336B62BFF34F8FBFF36F8FBFF34F8F99
:1067B000BFF36F8F0022C5F85022BFF34F8FBFF396
:1067C0006F8F6B6943F400336B61BFF34F8FBFF37F
:1067D0006F8FC5F88420BFF34F8FD5F8805043F6F4
:1067E000E0762B49C5F34E34C5F3C905640104EACC
:1067F00006002B4640EA8372013BC1F86022F9D2C1
:10680000203C14F1200FF2D1BFF34F8F4B6943F4BA
:1068100080334B61BFF34F8FBFF36F8F3FB0BDE845
:10682000F08362E50E4A02201B49D865D2F8F430A5
:106830000343C2F8F430D2F8F43003400E930E9ABA
:10684000D1F8003883F30888D1F804389847FEE778
:1068500004210320FBF718FE72B6FDF75DFF00BFB1
:10686000004402580010005C7FBB220000840040FE
:106870007FBB2230000002580008025860F000245C
:10688000A0060124C0EE002460F0002459840C0806
:1068900000ED00E03C0300240090F01F10B4EFF383
:1068A0001182102383F312880B4B4FF0E020002459
:1068B000D2B2596E0131596681699966C3F8984719
:1068C000016982F31188D3F850275DF8044B013237
:1068D000C3F85027704700BF501D002410B4EFF3D9
:1068E0001181102383F312884FF0E0229469136919
:1068F00013F4803F0C4B03D00120C3F89807946930
:10690000586EC9B2D3F8982781F311880244D96E22
:106910004FF47A7000FB01F31B1B5DF8044BB3FBD3
:10692000F1F300FB02307047501D00242DE9F047C1
:10693000DFF89080FAF7E4FF4FF4867900210646ED
:10694000D8F804501D4F002D2DDD00231C4609FBF7
:106950000382013392F80521AB4244EA0204F6D1E6
:1069600021435FFA81FA7B68C3F30803C3B9EFF3ED
:106970001183ABB9F9F7C8FC801BB0F5FA6FCCBF37
:10698000002104F001010029DDD1BAF1000F04D08B
:106990000B4B93F89D27542A08D05046BDE8F0874A
:1069A000FFF79CFFE8E78A460024DCE7B3F8A4275A
:1069B00050460132A3F8A427BDE8F08700ED00E0BF
:1069C000501D002404000020454B5B68C3F30803FE
:1069D0002DE9F0430546002B5ED1EFF31183002B28
:1069E0005AD1404B4FF0E0245A6EA069596E8A424A
:1069F000FAD1996E8842F7D8DE6E4FF47A7101FBB6
:106A000006F4241AB4FBF6F401FB0244344E1027BA
:106A10004FF0E02C4FF47A7E4FF001087268C2F319
:106A20000802CAB9EFF31182B2B95A6EDCF8180045
:106A3000596E8A42F9D1996E8842F6D8D3F86C9093
:106A40000EFB09F1091AB1FBF9F10EFB0212121B40
:106A5000AA42E3D3BDE8F083EFF3118287F31288F3
:106A6000DCF81800DCF81010C90303D5C3F89887C8
:106A7000DCF81800D3F86490D2B2D3F8981782F3F8
:106A800011884944D3F86C900EFB09F2121AB2FB3C
:106A9000F9F20EFB0122DAE7EFF31181102383F301
:106AA00012884FF0E0229669136913F4803F0D4B72
:106AB00003D00120C3F898079669586EC9B2D3F87D
:106AC000982781F311884FF47A710244D86E01FB44
:106AD00000F4A41BB4FBF0F401FB024496E700BFF2
:106AE00000ED00E0501D00242DE9F0473A4B471E11
:106AF0003A4D10264FF0E0204FF47A7C4FF0010819
:106B00006A68C2F30802002A52D1EFF31182002A08
:106B10004ED15A6E8469596E8A42FAD1996E8C426E
:106B2000F7D8D96E0CFB01FEAEEB040EBEFBF1FEF6
:106B30000CFB02EE6A68C2F30802E2B9EFF31182BD
:106B4000CAB95A6E8469596E8A42FAD1996E8C42DA
:106B5000F7D8D3F86C900CFB09F1091BB1FBF9F1E4
:106B60000CFB0212A2EB0E02B2F57A7FE2D3013FD8
:106B7000C6D2BDE8F087EFF3118286F312888469EC
:106B80000169C90302D5C3F898878469D3F864A062
:106B9000D2B2D3F8981782F31188D3F86C9051448D
:106BA0000CFB09F2121BB2FBF9F20CFB0122D9E734
:106BB000EFF3118186F3128884690269D20302D54A
:106BC000C3F898878469D3F864E0C9B2D3F89827EA
:106BD00081F311887244A4E7501D002400ED00E009
:106BE0002DE9F04FA74C83B0814601F1FF3AA64D45
:106BF00010265AF03BFB4FF4FA7B4FF0E0214FF4A4
:106C00007A774FF0010C6B68C3F30803002B40F058
:106C10005D81EFF31183002B40F05881636E88692A
:106C2000626E9342FAD1A26E9042F7D8E26E07FBF1
:106C300002FEAEEB000EBEFBF2FE07FB03EE6B683E
:106C4000C3F30803002B40F02381EFF31183002BE3
:106C500040F01E81636E8869626E9342FAD1A26E23
:106C60009042F7D8D4F86C8007FB08F2121AB2FBF6
:106C7000F8F207FB0323A3EB0E03B3F57A7FDED311
:106C8000BBF1010BBFD1D4F8A81494F8B004D4F828
:106C9000A42441B180F002038F88C3F340031B0199
:106CA0009F400B689F6132B100F0010390881B0187
:106CB00098401368986101274FF0E023CC4641B11A
:106CC00008688988D0F814E011EA0E0F18BF09048B
:106CD000816132B1116892884869024218BF12047A
:106CE0008A616A49B1F8D621002A40F06A810A46D1
:106CF00091F8DC11D2F8D821002940F05C811AB15A
:106D00009188106809048161FA224FF47A7E019219
:106D10006A68C2F30802002A40F01581EFF311827D
:106D2000002A40F01081626E9969606E8242FAD149
:106D3000A06E8142F7D8E06E0EFB00FBABEB0108C2
:106D4000B8FBF0F80EFB02886A68C2F30802002A5A
:106D500040F0E480EFF31182002A40F0DF80616EA2
:106D60009869626E9142FAD1A26E9042F7D883463A
:106D7000E06E0EFB00F2A2EB0B02B2FBF0F20EFB98
:106D80000122A2EB0802B2F57A7FDDD3019A013A23
:106D90000192BDD1D4F8A82432B111689288486913
:106DA000024218BF12048A61D4F8A42432B11168D7
:106DB00092884869024218BF12048A613349B1F8C7
:106DC000D621002A40F01B810A4691F8DC11D2F846
:106DD000D821002940F00C8112B11068918881619E
:106DE000FA224FF47A7E01926A68C2F30802002AFE
:106DF00040F0C580EFF31182002A40F0C080626E3F
:106E00009969606E8242FAD1A06E8142F7D8E06E35
:106E10000EFB00FBABEB0108B8FBF0F80EFB0288A1
:106E20006A68C2F30802002A63D1EFF31182002AD4
:106E30005FD1616E9869626E9142FAD1A26E904202
:106E4000F7D88346E06E0EFB00F2A2EB0B02B2FB1A
:106E5000F0F20EFB0122A2EB0802B2F57A7FDFD33B
:106E6000019A013A0192BFD10CF1FF3C5FFA8CFC10
:106E7000BCF1FF0F00F0D580D4F8A814D4F8A424F6
:106E80001DE700BF501D002400ED00E0482E002447
:106E9000EFF3118386F31288D1F818800A69D003C2
:106EA00003D5C4F898C7D1F81880606EDBB2D4F867
:106EB000982783F311880244E06E07FB00F3A3EBED
:106EC0000803B3FBF0F307FB0233D4E6EFF31182C0
:106ED00086F3128888690B69DB0302D5C4F898C76A
:106EE0008869636ED2B2D4F898E782F3118873444C
:106EF0009CE6EFF3118286F31288D3F818B0196973
:106F0000C90303D5C4F89877D3F818B0606ED2B22D
:106F1000D4F8981782F31188014493E7EFF31182B4
:106F200086F31288D3F818B01969C90303D5C4F8D9
:106F30009877D3F818B0606ED2B2D4F8981782F36D
:106F40001188014414E7EFF3118086F312889969E0
:106F50001A69D20302D5C4F898779969626EC0B2F3
:106F6000D4F8988780F31188E06E42440EFB00F855
:106F7000A8EB0108B8FBF0F80EFB0288E4E6EFF39B
:106F8000118086F3128899691A69D20302D5C4F870
:106F900098779969626EC0B2D4F8988780F31188A7
:106FA000E06E42440EFB00F8A8EB0108B8FBF0F8D5
:106FB0000EFB028834E7002A3FF4A6AE10689188E1
:106FC000A1E65449D1F8F421002A3FF49DAEB1F86E
:106FD000F8010A4600283FF497AE4F49D2F8E02165
:106FE000B1FBF0F1491011604A4A82F8F1718BE669
:106FF000002A3FF4F5AE918810680904EFE6454891
:10700000D0F8F421002A3FF4EBAEB0F8F821002AC2
:107010003FF4E6AE0021D0F8E021116080F8F111D4
:10702000DEE64FF47A7B4FF0E0214FF0010C5F4633
:107030006B68C3F30803002B59D1EFF31183002BC6
:1070400055D1636E8869626E9342FAD1A26E904206
:10705000F7D8E26E07FB02FEAEEB000EBEFBF2FEBF
:1070600007FB03EE6B68C3F3080313BBEFF3118355
:10707000FBB9636E8869626E9342FAD1A26E904248
:10708000F7D8D4F86C8007FB08F2121AB2FBF8F2BA
:1070900007FB0323A3EB0E03B3F57A7FE2D3BBF127
:1070A000010BC5D1BAF1010ABFF4A3AD03B0BDE82D
:1070B000F08FEFF3118386F31288D1F818800A69F4
:1070C000D20303D5C4F898C7D1F81880606EDBB23C
:1070D000D4F8982783F311880244E06E07FB00F38D
:1070E000A3EB0803B3FBF0F307FB0233D2E7EFF3A4
:1070F000118286F3128888690B69DB0302D5C4F814
:1071000098C78869636ED2B2D4F898E782F3118881
:1071100073449EE7482E002440420F002DE9F043BF
:10712000144C83B0DFF85090DFF8508004F590667F
:1071300002E00834B44219D094F90650002DF8D179
:107140002768083407EB08039B0A09EB4303B3F8ED
:1071500048025CF0BBF834F8041C01232A46384688
:10716000CDE9005560F060FFB442E5D103B0BDE861
:10717000F08300BF4425002478DD0A080000FEA744
:10718000704700BF0223054A52085B0090429BB241
:1071900001D2FF2BF8D91846704700BF80F0FA02E1
:1071A000F0B503798BB02E4C002B14BF01220022C6
:1071B00084F85C2303D184F830330BB0F0BD04F5C0
:1071C0005977054690F9001038464FF0E9FFAE7840
:1071D000002E38D1234B2448C4F8F833C4F86C632C
:1071E000FFF7D0FFA4F868034FF47A70FFF77CFC38
:1071F000D4F86C3313B11A689B8893611B4DEC462D
:107200000FCDACE80F000FCDACE80F0095E8030000
:107210008CE80300694638464FF038FED4F86433F2
:107220001A6A002AFCD11EB10D213046FAF7CEFEB3
:10723000616E01220023C4F8201384F8302384F8FF
:1072400024330BB0F0BD3046FCF7BEF806460028EC
:10725000C0D01E2300222C21C380FAF7B7FEB9E765
:10726000501D00245C200024801A060060EC0A08EF
:107270002DE9F04F002385B0DFF800A34FF001099E
:107280000193B94B0AF1F00BB84FA3F104080BE0DE
:10729000019B09F101090AF1280A0BF1050B0133E1
:1072A000062B019300F0F1809AF80030022BEFD109
:1072B0009BF90320511C00F0EB80D2B2944602EB04
:1072C0004204A94B9DF8041003EB84040F2A5ED8F6
:1072D000A74802E00330B84259D00378002BF9D117
:1072E00045788D42F6D18578D8F8C8606068A56089
:1072F000B042257000F04481D8F8EC60B04200F054
:107300005E81D8F81061B04200F06281D8F8346133
:10731000B04200F06281D8F85861B04200F06C8150
:10732000D8F87C61B04200F08081D8F8A061B0420A
:1073300000F07681D8F8C461B04200F08081D8F8BE
:10734000E861B04200F07681D8F80C32984200F043
:107350008C81D8F83032984200F08181D8F85432CC
:10736000984200F0A581D8F87832984200F09A81CE
:10737000D8F89C32984200F0A781D8F8C0329842E1
:1073800000F0A881D8F8E432984200F097810132E9
:107390000C34D2B2624599D9002303939BF904209F
:1073A000531C79D0D2B2964602EB42046E4B9DF844
:1073B000041003EB84040F2A5DD86D4802E003300B
:1073C000B84258D00378012BF9D145788D42F6D1D7
:1073D0008578D8F8C8606068A560B04225705FD035
:1073E000D8F8EC60B04200F0EF80D8F81061B042FD
:1073F00000F0F880D8F83461B04200F0F880D8F896
:107400005861B04200F0FD80D8F87C61B04200F0D5
:107410000281D8F8A061B04200F0F880D8F8C461C9
:10742000B04200F01781D8F8E861B04200F00C815A
:10743000D8F80C62B04200F02481D8F8303298427B
:1074400000F01981D8F85432984200F02581D8F81C
:107450007832984200F01A81D8F89C32984200F0B5
:107460004B81D8F8C032984200F04081D8F8E4321D
:10747000984200F0358101320C34D2B296459AD24E
:1074800000220023CAE9042302E705B0BDE8F08F1B
:107490004FF00F0C002212E74FF00F0E002283E78F
:1074A00000231E46029306EBC600013608EB80005F
:1074B00090F9E0C0BCF1000FDDD1624680F8CC301D
:1074C000AC462C4B1546029AC0F8D0C0134480F845
:1074D000E190CAF81430132380F8E0303046FAF710
:1074E000BBF9039B002BCBD0DAF814402046F8F709
:1074F00087FDDAF81000F8F783FDDAF81830C16874
:10750000DAF80420596240215D60996002F120019F
:107510009D631960C3E90355C3E90555C3E90755E0
:10752000C3E90A55C3E90C55A4B1DAF81C3030326E
:10753000E1681D625962C3E900254FF48032C3E956
:107540000255C3E90455C3E90655C3E90B55C3E920
:107550000D559A620023304607491A46FAF7A0F9FA
:1075600001238AF80C3093E6040000246EDE0A083A
:10757000F0DD0A08C4000024390A00004830002465
:107580001846029300EBC00E013008EB8E0E9EF9F8
:10759000E060002E7FF4FBAE029A8EF8CC30594B9F
:1075A000CEF8D05013448EF8E190CAF8103014236E
:1075B0008EF8E030FAF750F901230393EEE6242029
:1075C000012302901846DDE724201E4602906AE758
:1075D0004820022302901846D4E76C20032302902F
:1075E0001846CFE7022348201E4602905BE703239C
:1075F0006C201E46029056E7902004230290184605
:10760000C0E7042390201E4602904CE70623D820B2
:107610001E46029047E70523B4201E46029042E72B
:10762000D820062302901846ACE7B4200523029028
:107630001846A7E74FF4907002900820A2E7FC20BC
:107640000723029018469DE74FF490730826029393
:10765000002328E70723FC201E46029023E74FF46F
:10766000B470022302900A208CE74FF4A273092021
:107670000293012386E74FF4B47002230A26029096
:1076800011E74FF4A270092602900CE74FF4D8736B
:107690000C260293042306E74FF4C6730B260293CD
:1076A000032300E74FF4D8730C200293042369E707
:1076B0004FF4C6730B200293032363E74FF4077361
:1076C0000F20029307235DE74FF4EA730D20029326
:1076D000052357E74FF4FC730E200293062351E76E
:1076E0004FF407730F2602930723DCE64FF4FC7375
:1076F0000E2602930623D6E64FF4EA730D26029374
:107700000523D0E6C40000242DE9F04F4C484FF08B
:10771000010A4C494FF002094B4B4FF0040808276F
:107720001026202540244FF0800EDFF820C130F8CD
:10773000022F12F0010F03D01960083323F804ACB4
:1077400012F0020F03D01960083323F8049C12F0E2
:10775000040F03D01960083323F8048C12F0080FCB
:1077600003D01960083323F8047C12F0100F03D003
:107770001960083323F8046C12F0200F03D019604D
:10778000083323F8045C12F0400F03D0196008336B
:1077900023F8044C12F0800F03D01960083323F84B
:1077A00004EC12F4807F05D04FF4807B196008331D
:1077B00023F804BC12F4007F05D04FF4007B19605D
:1077C000083323F804BC12F4806F05D04FF4806BAB
:1077D0001960083323F804BC12F4006F05D04FF48D
:1077E000006B1960083323F804BC12F4805F05D0E5
:1077F0004FF4805B1960083323F804BC12F4005F77
:1078000005D04FF4005B1960083323F804BC12F470
:10781000804F05D04FF4804B1960083323F804BC27
:10782000D20B05D04FF400421960083323F8042C22
:1078300001F5806161457FF47AAFBDE8F08F00BF4C
:10784000E2DF0A0800000258442500240024025800
:107850002DE9F0470546086888B00C464FEA902CA1
:10786000BDF84080ACF5801C9DF844A0BCF1520FDF
:1078700058D819462E4B13F80C600D2E52D806EB33
:10788000C6032C4F06EB430307EB8307FEF7CCF848
:1078900094F80590A379BAF1000F01D083F00103A9
:1078A0005A004FF48071DB00384602F00202CDF836
:1078B000088003F0080303924A460493602301936F
:1078C0004FF40073CDE90613002301A905935BF083
:1078D00067F8A379384649469F0726D454F06AFDD5
:1078E0004C22154B02FB063393F8A52D012A10D12B
:1078F0000221D3F8682D83F8A51D104B91680B4029
:10790000062B06D0B3F5803F03D0136843F0010384
:1079100013602168637901F1340269600021D01895
:107920002860D15008B0BDE8F08754F0D7FED7E703
:1079300078DD0A08B82A0024501D00240700010041
:1079400010B4284C94F8303763B3226D904234D091
:10795000012B27D0D4F82C21824236D0022B21D003
:10796000D4F80822904232D0032B1BD0D4F8E42262
:1079700090422ED0042B15D0D4F8C02390422AD0A8
:10798000052B0FD0D4F89C24904226D0062B09D08A
:10799000D4F87825904222D0072B03D0D4F854266F
:1079A000824210D0DC22591C02FB034284F83017BB
:1079B000106518465DF8044B70470023DBB25DF894
:1079C000044B184670470723F8E70123F6E7022324
:1079D000F4E70323F2E70423F0E70523EEE70623A9
:1079E000ECE700BFFC10002008B556F031F81B2072
:1079F000FBF7EAFC08B12923C3801C20FBF7E4FC59
:107A000008B12923C3805CF03BFE10485CF024FEE3
:107A10000F4B93F81523022A01D0012008BD0D4A0F
:107A200092F85C2D012A0ED0022AF6D10A4AD3F828
:107A3000F405C3F8F02560F051FA0023074A184610
:107A400082F8233008BD064AF1E700BFAC030024EA
:107A5000482E0024501D00246C03002400ED00E09B
:107A60008C0300240A4B93F8E4231AB9094A92F8CC
:107A7000F80570470849CA6D032AF7D10020054A66
:107A80004FF0010C83F8E40382F8F8C5C865EEE70F
:107A900000000024482E002400400058002103204C
:107AA00008B5FAF7F1FC72B6FCF736FE2A4C08B5B9
:107AB000D4F8FC3594F80206002B3DD114200025A3
:107AC000FFF712F8254900BFD4F8FC355BB1186800
:107AD00094F802269B880069034012B91BB1FFF796
:107AE000DDFF002BFBD04A6ED1F80833D31A322BBE
:107AF00012DCD4F80436D31A002BE4DDD1F8A43418
:107B000033B118689B884669334218BF1B048361F0
:107B10003232C4F80426D6E7D1F8A4244AB191F849
:107B2000B034908803F0010312681B0100FA03F3DC
:107B30009361C4F80456C6E719689A880B69134024
:107B400020B1002BBAD10B691340FAE7002BB5D056
:107B50000B691340FAE700BF482E0024501D002493
:107B6000024BD3F804331B6A184700BF501D002492
:107B70000A4AD2F8603373B11968988892F85D3375
:107B80000A6910401BB1B0FA80F040097047003814
:107B900018BF012070470120704700BF501D00240E
:107BA000034BD3F8040308B183691847704700BF3B
:107BB000501D0024154908B5D1F860336BB1186821
:107BC00091F85D239B880069034022B12BB100230B
:107BD00081F8303308BD002BF9D091F83033032BF6
:107BE0000ED891F824330133DBB2072B81F824330C
:107BF000EDD84A6E0123C1F8202381F8303308BD47
:107C00000348FFF7BFFAA1F86803EAE7501D002414
:107C1000801A060030B5002299B004469525134617
:107C20008DF80C108DF80D5044F0400504930120A0
:107C300065F307028DF81C300A938DF830308DF80B
:107C40004430159317931D4D069010908DF85800F1
:107C500002A8CDE90D33CDE913330B0E099005F5DC
:107C6000597063F30F220B0C090A63F317420DF1ED
:107C70000703059361F31F62114B029208930623D9
:107C8000104A0DEB03010B93082312920F9104A9E4
:107C900085F8FC334FF0FAF8D5F86423136A002B0B
:107CA000FCD19DF80730FF2B00D01CB99DF80600D1
:107CB00019B030BD4FF0FF30FAE700BF501D00246F
:107CC000F1090408290A040830B52B4C9DB0FD25A4
:107CD00000230122002000218DF8065004F559757B
:107CE000C4F82C338DF83C3010938DF85030159338
:107CF00018931A930E928DF86420CDE912320DF18B
:107D00000603CDE90C01CDE916010CA92846119313
:107D10004FF0BCF8D4F86423136A002BFCD10DF1AA
:107D20000701012228468DF8143009930B93049221
:107D30008DF8282084F8FC23CDE902310F49069103
:107D400002A9CDE907334FF0A1F8D4F86433186ADB
:107D50000028FCD19DF80730FF2B07D0626E092365
:107D6000C4F8202384F830331DB030BD0423022032
:107D700084F830331DB030BD501D0024290A04089A
:107D80002DE9F041A34C92B094F85C63002E00F012
:107D9000E58194F830335A1E082A00F26C81DFE83E
:107DA00012F032006D00BA006A013D0179011A003B
:107DB0006A01090058F0F6FE002840F0BE82D4F8AF
:107DC0002033626EFA33934280F05281FFF7F2FE65
:107DD00094F83033DFE758F0E5FE0028EFD0D4F810
:107DE0002C330022012B84F8242340F2B882D4F8EB
:107DF0002823013B08210132C4F82C3384F83013C6
:107E0000C4F8282301E100210846FFF703FFD4F856
:107E10006423C5B2136A002BFCD10A20FEF7D4FDFF
:107E2000D4F86C3313B11A689B889361012D40F02C
:107E30001F81002740F2AB11082084F82573FFF75B
:107E4000E9FEC0B2052800F0E081012800F0BD8104
:107E5000D4F86423136A002BFCD10A20FEF7B4FD8A
:107E6000D4F86C3313B11A689B88936194F8253366
:107E7000002B00F05F82022384F8303394F82553FE
:107E800000213720A5F10205FFF7C4FE2920B5FA2D
:107E900085F56D09AD072946FFF7BCFED4F86423CC
:107EA000C5B2136A002BFCD10A20FEF78DFDD4F871
:107EB0006C3313B11A689B889361002D40F0D88011
:107EC00094F82533022B00F0EA810021092084F880
:107ED0002653FFF79FFE002800F09C810025D4F870
:107EE0006423136A002BFCD10A20FEF76DFDD4F841
:107EF0006C3313B11A689B889361002D00F0B88031
:107F000000210A20FFF786FEC0B2002840F0B681AB
:107F1000032384F83033102103A8F9F77BF80028F5
:107F200040F0A680BDF80D309DF80C205BBA9DF89E
:107F3000111062F307009DF80F20A4F838339DF864
:107F4000193062F30F209DF810201B019DF814508A
:107F500062F317409DF81A20DBB261F31F60DDF871
:107F6000151043EA121302F00F0209BAC4F83A03DB
:107F700003F5FA6384F84823C4F840132909A4F8E8
:107F80004633BDF81230D4F86423A4F83E3305F02C
:107F90000F0384F8441384F84533136A002BFCD193
:107FA0000A20FEF711FDD4F86C3313B11A689B88D0
:107FB000936194F82633B3B94FF400711020FFF7A2
:107FC00029FED4F86423C5B2136A002BFCD10A2021
:107FD000FEF7FAFCD4F86C3313B11A689B889361EE
:107FE000002D7FF4F3AE0C480021FFF7CBF80422FC
:107FF000A4F868031346C4F82C1384F83023042B28
:1080000018BF082B0CBF01260026304612B0BDE871
:10801000F08100BF501D002440787D014FF40071B5
:10802000D4F80C03F8F7F6FF012800F09D80022831
:1080300000F0A180E0B9D4F86423136A002BFCD1CE
:108040000A20FEF7C1FCD4F86C3313B11A689B8880
:10805000936104230020D4F8185384F8303384F853
:108060002403002DD1D0D4F81C33D4E9C321A84770
:1080700094F830335A1ED2B2022AC0D8636ED4F8B4
:1080800020239B1AC82B00F295800026304612B0A0
:10809000BDE8F081D4F86423117B136A002946D02F
:1080A0005269002A43D094F8EC23002A3FD0B3FA57
:1080B00083F35B09002BDBD0002302A90122B24825
:1080C000ADF808308DF81830079308938DF82C30F0
:1080D00011938DF84020CDE90313022105910DF194
:1080E0000701CDE9091203A9CDE90C33CDE90E331F
:1080F0004EF0CCFED4F864331D6A002DFCD19DF8FF
:10810000073003F01F03052B00F0FF80FFF752FD3F
:10811000D4F81873002F3FF43CAED4F81C332A4631
:10812000D4F810130120B84794F8303333E6D4F86C
:108130000C334FF4807294F81413934803EB01212D
:1081400058F0EAFC94F814230132D2B2A2F10203EF
:1081500084F81423B3FA83F35B09ABE7304684F861
:10816000306312B0BDE8F081D4F82033626E64331E
:108170009342BFF47DAFD4F86423136A002BFCD183
:108180000A20FEF721FCD4F86C3313B11A689B88DF
:108190009361FFF70FFDD4F81853002D3FF4F9ADAC
:1081A0000022D4F81C33D4F810131046A84794F8D2
:1081B0003033F0E5FFF7FEFC94F83063082E18BF6B
:1081C000042E0CBF012600261FE702AB03A96E4850
:1081D0000493042303978DF81870079705930A9763
:1081E0008DF82C500C97CDE908774EF04FFED4F85F
:1081F0006423136A002BFCD19DF80B30AB2B7FF46A
:1082000029AE022384F8253324E6D4F8642384F8C5
:1082100025531FE610215D48F8F7FCFE00287FF487
:108220005DAE94F85B3313F001033FF457AE94F85E
:108230004C23921100F0AE80012A7FF44FAE94F8E7
:1082400053231621524F02259200D2B2C5F10803E2
:108250008B4228BF0B46C3F108059840C91A42FA61
:1082600005F24FF0000540EA020017F8012FEDD1AA
:10827000013083023546C4F8343330E6D4F8642341
:10828000136A002BFCD10A20FEF79EFBD4F86C3356
:10829000002B3FF49BAD1A689B88936196E52946B5
:1082A0003A20FFF7B7FC02ABC7B203A9049304233B
:1082B00035480593012303958DF82C308DF818501F
:1082C0000C95CDE90755CDE909554EF0DFFDD4F801
:1082D00064331A6A002AFCD187B91A6A002AFCD1D1
:1082E0000A20FEF771FBD4F86C3313B11A689B882F
:1082F0009361029D2DBAC5F38075E6E51A6A002ADE
:10830000C1D01A6A002AF9D1BDE70722636ED4F8FA
:10831000185384F83023C4F82033002D3FF4B5AE51
:10832000D4F81C330120D4E9C321A84794F8303392
:108330005A1EA0E684F83033A7E6D4F86423136A03
:10834000002BFCD10A20FEF73FFBD4F86C3313B1AD
:108350001A689B889361042384F8303355E661D012
:108360000423D4F8642384F83033136A002BFCD13F
:108370000A20FEF729FBD4F86C33002B3FF478AECB
:108380001A689B88936173E6B42000249C20002423
:10839000A320002494F851031146DFF8A0C0032560
:1083A00000F00F0294F85503062780019340C0B2F5
:1083B000C7F10802AA4228BF2A46C2F10807914025
:1083C000AD1A40FA07F04FF0000741EA00011CF82F
:1083D000010FEDD194F852030231DFF864E00C276D
:1083E00080014FF0060CC0B2CCF108024FF0000C37
:1083F000BA4228BF3A46C2F108089540BF1A40FA6F
:1084000008F045EA00051EF8010FEDD10135D81737
:1084100005FA01F2A2FB033102FB00125B0A43EAF8
:10842000C25327E7FFF750FC02287FF421AED4F8AF
:1084300064331A6A002AFCD19AE700BFA520002401
:10844000A2200024034B93F82400032894BF0020AB
:10845000012070475C2000240048704784200024DD
:10846000034B93F82400003818BF0120704700BF69
:108470005C200024034B93F82400032894BF0020C1
:10848000012070475C2000240048704784200024AD
:1084900070B4154D00202B4693F82A4014B1DE69C4
:1084A0008E4205D0013010330B28F5D170BC7047D7
:1084B000AAB1AB6903EB40239A4201D1022C07D049
:1084C00095F8E83113B9012385F8E83101236B7081
:1084D00005EB0015012385F82A3070BC704705EBC9
:1084E000001585F82A20E1E75035002430B4002338
:1084F000184C204684F8D43003E0013310300B2BA5
:1085000017D0C5698D42F8D190F82AC0BCF1030F8D
:10851000F3D182B1A16901EB43218A4204D094F8DE
:10852000E8219AB10122627004EB0314012384F85C
:108530002A3030BC7047D4F8D02004EB0313042158
:10854000013283F82A10C4F8D020F2E7012284F81F
:10855000E821E7E750350024A0B183681BB10C4B3C
:1085600007229A7070470A4A04211078137503286D
:108570009170C2E9033314BF4FF480738023C2E9C2
:1085800001337047024B012283F8E8215A7070478B
:108590005035002410B58C18A14215D001F1FF3ED2
:1085A000013C41F2210C1EF8012F082380EA022031
:1085B00002B24000002A8CEA420180B2B8BF88B201
:1085C000013BF5D17445EED110BD00BF704700BF2F
:1085D0002DE9F047002BDDF820A0884607460CBFA8
:1085E0004FF020094FF030095646002A144616F87D
:1085F000011B23DD11B3334601E0002C05DD13F828
:10860000012B2546013C002AF7D1023D3CB14946E9
:108610003846C047013DFAD29AF8001059B13846A1
:10862000C047334616F8011B0029F8D1A4EB0A0411
:108630001819BDE8F0872046BDE8F087002C04F14A
:10864000FF35E4DC00240029E9D1F4E703685A1C73
:1086500002601970704700BF10B56FF00044024609
:10866000044404E0B3EB0E0015D1A24214D012F87A
:10867000013BA3F14100192811F8010BA0F1410CB5
:1086800098BF203300F1200EBCF1190FEAD91B1A54
:1086900004D10028E9D110BD002010BD184610BD3E
:1086A000884230B54FF001043AD301FB04F4B0FB2B
:1086B000F4FC8C45F9D2BCB102BB06E0A14203F840
:1086C000015B11D81446B0FBF2FCBCF1090F0CF1B0
:1086D00057050CF1300E04FB1C00B4FBF1F2EDDC8D
:1086E000A14203F801EBEDD900221A7030BDA1427E
:1086F00003F8015BF8D81446B0FBF2FCBCF1090F9B
:108700000CF137050CF1300E04FB1C00B4FBF1F248
:10871000EDDCA14203F801EBEDD900221A7030BD67
:108720008446002AEAD1D0E7002870B503DA2D2369
:10873000404201F8013B092886464FF0010307DD5E
:1087400003EB83035B00B0FBF3F2092AF8D89BB17B
:108750000F4CA4FB030CBEFBF3F2092A4FEADC0C1E
:1087600002F1570602F1300503FB12EE07DD092B7B
:1087700001F8016B6346ECD800230B7070BD092B28
:1087800001F8015B6346E4D800230B7070BD00BFA5
:10879000CDCCCCCC0378202B03D110F8013F202B7B
:1087A000FBD0092BF9D02D2B00F0A9802B2B75D0F5
:1087B000B7EE000AA3F13002D1B2092977D8F2EE60
:1087C000046ADFED5F7A07EE102A10F8013FB8EE79
:1087D000C77AA3F13002D1B2A7EEA67A0929F0EE4A
:1087E000477AF0D92E2B66D003F0DF03452B40F0FB
:1087F000838010B442782D2A00F096802B2A00F056
:108800008380A2F130030130092B00F28480002420
:10881000002303EB830302EB430310F8012FA2F1C3
:108820003001303B0929F4D9B3F59A7F1A46B7EEE7
:10883000007A28BF4FF49A72072B09D91346DFED4F
:10884000416A083B27EE267A072BFAD802F0070286
:10885000DAB1F2EE046A012A27EE267A15D0022A4E
:1088600027EE267A11D0032A27EE267A0DD0042A85
:1088700027EE267A09D0052A27EE267A05D027EE9C
:10888000267A062A18BF27EE267A002C45D0C7EE96
:10889000877A5DF8044B20EE270A70474378B7EEDD
:1088A000000A0130A3F13002D1B2092987D92E2B59
:1088B000DFED237A98D143780130A3F13002D1B2B1
:1088C000092991D8B2EE047AF0EE475A06EE902AC2
:1088D00010F8013FB8EEE66AA3F13002D1B2C6EE5D
:1088E000076A092927EE257A77EEA67AEED903F0F2
:1088F000DF03452B3FF47DAF20EE270A7047437816
:10890000BFEE000A013055E782780230A2F1300351
:10891000092B7FF67CAFB7EE007A67EE877A5DF8B9
:10892000044B20EE270A704782780230A2F1300310
:10893000092B01D801246BE7B7EE007AA7E700BF47
:108940000000000020BCBE4CF8B5164D6B78BE2B65
:1089500026D1AC1C144F022229464FF6FF70FFF7B8
:1089600019FE22884AB1A618BE4219D2052A17D983
:1089700021463446FFF70EFEF3E721460222FFF7B9
:1089800009FE0222A1180634FFF704FE074B641B00
:10899000A3F8584241F60F53C31A58425841F8BD44
:1089A0000020FCE700000208000004085035002405
:1089B000032870B51CD80F4BC943C60003EBC00099
:1089C00001F0010190F8605290F8612281EA0504FB
:1089D000A2420DD0D0F85C223AB14D1B10689288AB
:1089E0006942694109018A408261334483F86142E6
:1089F00070BD00BF503500242DE9F8430546884678
:108A000017461E462D4C94F8240004280AD0082846
:108A100006D1E369AB423FD0FFF756F90228F2D006
:108A2000012035E0A37E002B34D169021820FFF726
:108A3000F1F8C0B290BB94F82430082B2CD0FE2162
:108A40001F4BA26D83F87C121E4B117BC3F828804C
:108A500051B1526942B194F8E020002A14BF4FF49A
:108A600000724FF4807201E04FF48072DFF858908A
:108A7000144948461A634EF009FA012206230020E1
:108A800049F8588C6560E7602661227284F82430CA
:108A9000BDE8F8832946C9E7FC21D1E7A26D136A36
:108AA000002BFCD10A20FDF78FFF236E13B11A684B
:108AB0009B889361FFF77EF80320E9E75C200024A0
:108AC000503500244C040024B420002470B5204EFE
:108AD00005460C4696F82430042B08D0082B1ED1EE
:108AE000F369834219D0FFF7EFF8022817D100216C
:108AF0003720FFF78FF821461720FFF78BF8C0B219
:108B0000A8B9B37E6BB969021920FFF783F870B971
:108B10000823C6E9075486F82430022070BD0120DE
:108B200070BD29461920FFF775F80028F0D0B26D06
:108B3000136A002BFCD10A20FDF746FF336E13B1F8
:108B40001A689B889361FFF735F8032070BD00BF5A
:108B50005C2000242DE9F0411F4C0746884616464C
:108B600094F824C01D46BCF1040F09D0BCF1080FD5
:108B700002D00020BDE8F081FFF7A6F80228F8D166
:108B8000A37E9BB139461120FFF744F8C0B2A0B9CB
:108B9000124B05220120C4F800801B6884F82420B1
:108BA0006760E660C4E90453BDE8F08179021120F2
:108BB000FFF730F8C0B20028EAD0A26D136A002B8C
:108BC000FCD10A20FDF700FF236E002BD1D01A68DC
:108BD00000209B889361CDE75C200024B41D002415
:108BE00008B5FAF779FD48B10F4A137E0133DBB2BD
:108BF000072B137603D9002382F8243008BD536D68
:108C000043B1186892F851109B880069034041B144
:108C1000002BF0D1054B01211B6882F82410536111
:108C200008BD002BE7D0F5E75C200024B41D00242C
:108C300010B50379184C002B14BF0122002284F8D0
:108C4000502025D0154B626D5B78003B18BF012387
:108C500084F8F23082B111689388096994F8512040
:108C60000B403AB143B1237E0022013384F8242023
:108C7000237610BD002BF6D0FAF72EFD0028F2D196
:108C8000074B012220761B6884F82420636110BD05
:108C900084F8243010BD00BF5C200024C4290024C7
:108CA000B41D002470B5134C05460E4694F82430CC
:108CB000042B0FD0082B1AD1E36983420FD0002375
:108CC00094F8F220236212B10B4AC2F88032F9F70D
:108CD0004FFF30B10823C4E9075684F8243002203E
:108CE00070BD064B09221B6884F8242063610120B3
:108CF00070BD00BF5C20002450350024B41D00244A
:108D0000F8B5864C94F85060002E00F0BD8094F8C1
:108D100024506B1E082B1DD8DFE803F09A8E4E1CE2
:108D200035059E1C27007E4B5B6A002B40F08D8032
:108D30007C4B0722E5681B6884F824206361002DC2
:108D400000F0838023690120D4E90021A84794F82A
:108D500024506B1EDBB2022B71D9042D18BF082DD5
:108D60000CBF012600263046F8BDF9F701FF0028A8
:108D700040F0BD806B4A63691268FA339342ECD2CB
:108D8000FFF72EFFC3E7664B1F6A002F40F0A78056
:108D9000F9F7EEFE0028BAD00423E568277684F8B8
:108DA0002430002DDFD02369384622686168A84747
:108DB00094F824506B1ECDE7F9F724FF00283ED12C
:108DC000594B206293F82C10DA8D84F82E10A2856E
:108DD000196B1A6B090E120C84F82F1084F83020CE
:108DE0001A6B196B120A84F8321093F8341084F855
:108DF000312084F8331093F8351093F835200909A1
:108E000002F00F0284F8381084F839209A6BD88F5A
:108E10006263DA8FD98FC2F30B1301F00F020421C2
:108E200043EA102384F83C2003F00F0384F8241055
:108E300003F5FA6363876AE7F9F79AFE40BB394B9B
:108E400062691B689B1AC82B3ED800263046F8BDC5
:108E5000022384F824305AE7F9F78AFE002889D0E3
:108E6000226A0023012A237645D9E169013A0131BA
:108E7000C4E9071294F8F22012B12C4AC2F88032E9
:108E8000082384F824306EE7304684F82460F8BD67
:108E9000F9F7B8FE0028D2D1254B1B78002BA3F19F
:108EA0000203B3FA83F308BF01255B096576A37655
:108EB000F9F7A8FE00287FF463AF1B4B03229B6CDD
:108EC00084F82420A36222E7FFF78AFE94F8246046
:108ED000042E18BF082E0CBF0126002643E7114AB6
:108EE0006369126864339342FFF411AF35E70423DA
:108EF00084F8243037E7FAD194F8F220236212B1D3
:108F00000A4AC2F88032F9F733FE0028EFD1054B48
:108F100009221B6884F82420636196E75C20002402
:108F200004220024B41D0024E82900245035002424
:108F3000402A00242DE9F84F3A4C1F4605460E46BC
:108F400094F824309046042B12D0082B40D1E369CA
:108F500083420DD0002394F8F220236212B1324AEA
:108F6000C2F88032F9F704FE60B3042384F8243099
:108F7000DFF8B4B0DBF88092C9F34F230F2BC4E9BC
:108F8000006528D8D4F820A0BAF1000F23D094F8B7
:108F9000F23003B325484FF400723146484464F080
:108FA00015FB09F50073C3F34F22CBF880325B0A3F
:108FB000102A02D0BAF1010F28D19BB21B4E5A1EC3
:108FC000AD1A09E01A4B09221B6884F8242063615A
:108FD0000120BDE8F88F01230621284601253246ED
:108FE00084F824100021C4F80C802761257259F000
:108FF000B1FB0028EDD0FFF7F3FDE66826B1236949
:10900000002261682846B0470320E2E7E2690AF1DE
:10901000FF33042102200132236284F82410E2612C
:10902000D7E700BF5C20002450350024CC59002431
:10903000B41D00242DE9F843284C80468946174684
:1090400094F824C01E46BCF1040F13D0BCF1080FE5
:1090500002D00020BDE8F883002394F8F2202362B8
:1090600012B11F4AC2F88032F9F782FD20B30423FF
:1090700084F8243019F01F0F25D10125194A1A4B05
:10908000414615624FF400724846C3F800905A609A
:109090002A469D6059F0E2FAA8B9144B05222846E9
:1090A000C4F800901B68C4F8048084F8242063612D
:1090B000C4E90376BDE8F8830C4B09221B6884F8E9
:1090C00024206361C5E7FFF78BFDE568002DC0D064
:1090D0000022236961681046A847BAE75C20002493
:1090E000503500240422002434220024B41D00241E
:1090F000092917D0B1FA81F35B0999B101390360ED
:109100004A0001F0030102F00802C1EB01119300D3
:10911000C1EB0111A3EB92038900C3EB0313818020
:109120009B004380704700BFB5EEC00ADFED357A83
:109130000023F1EE10FA30B5C8BF30EE270A87B031
:10914000D8BF30EE670ADFED307A054603A90293F7
:1091500020EE270ACDE90033FDEEC07A17EE904AE3
:1091600084EAE470A0EBE47055F062FD002C03A8E3
:10917000B4BF2D2320238DF8003061F093FA01282D
:109180002AD0022834D003281ED003A9684664F0F0
:1091900083FA684661F086FA044669462846033C2D
:1091A000E4B2224664F012FA002328462B5561F0FF
:1091B00079FA2E22431C0DEB04012A54E81864F0BE
:1091C00098FA284607B030BD302303A968468DF8C9
:1091D000013064F061FADCE743F23002302303A986
:1091E0006846ADF801208DF8033064F055FAD0E7F9
:1091F00043F2300303A96846ADF8013064F04CFA3D
:10920000C7E700BF6F12033A00007A4409F0AABB17
:1092100038B5054658B14C1E14F8011F284619B937
:10922000BDE8384009F0B2BB09F09CFBF4E738BD5B
:1092300008B5202164F03FFA034618461BB10278B6
:109240000133202AF9D008BD08B5CB0701D4FBF7BC
:10925000B7FA08BD2DE9F3410023134D044600EB96
:10926000810685F8843205F52175104FB44203D18B
:109270000F4802B0BDE8F081394628464FF000089B
:1092800064F00AFA2146684664F033FA2021684601
:1092900064F011FA28B969462846043464F0FCF9F0
:1092A000E4E780F80080F1E7503500247FEE0B08FA
:1092B000D43700240378022B12D00E494368026988
:1092C000D1F84C02023A184010B4400AD1F8444296
:1092D000D1F8401204FB02005DF8044B08447047CB
:1092E000044B4268D3E98D0100EB410000EB5220B2
:1092F000704700BF503500242DE9F04F83B002F0D5
:1093000002077F4E019308B9002F4DD1D6F83C4299
:10931000C4BB4FF0FF3E7A4C4FF0000CF146F246D2
:10932000F046E36994F82A50984247D015B3012DCE
:1093300006EB0C1B0ED19BF82B50EB070AD415F053
:109340007E0F07D1ED0940F09780656AA84584BF7C
:10935000A846E1460CF1010C1034BCF10B0FE0D132
:10936000BEF1000F80F2AC80BAF1000FC0F2918024
:10937000D44626E0E6460CF1010C1034BCF10B0F8C
:10938000CFD1EDE7D6E9903505FB0434A042C0D338
:1093900096F8E83113B9012386F8E8310123737098
:1093A000002003B0BDE8F08F96F8E831002B6CD0B8
:1093B00001230220737003B0BDE8F08F002D40F050
:1093C0008180D6F8CC5006EB0C1E0CF1020401355E
:1093D000CEE9070506EB041EC6F8CC50CEF80450C3
:1093E0000025CEF8085006EB0415AD7A042DDBD825
:1093F0000FF2040E5EF825F00D9404084194040861
:10940000A1930408419404084394040812F0010550
:10941000D6F818E064D106EB0410019B4FEAE20E87
:1094200090F80B80032B6EF3C71880F80B8055D98A
:109430004FF6FF70834228BF034606EB04100381FA
:1094400067BB500705D506EB0410C37A43F0010350
:10945000C372D30608D506EB0414E37AC3F34502BE
:10946000013262F34603E372B369012003EB4C233C
:109470000B6003B0BDE8F08FE2460CF1010C103434
:10948000BCF10B0F7FF44DAF6AE7012386F8E8319A
:109490008EE7B9F1000F83DBCC4692E7D6F8D00017
:1094A000D6F8CC3001300133C6F8D00006EB0C10F2
:1094B000C6F8CC30036206EB041304209872C0E7B0
:1094C000F4467EE7D6F8CC500CF10204013506EBE9
:1094D000041EC6F8CC50CEF8045084E72B46ACE707
:1094E000084B0EEB4C21084A1B689D680023A847D7
:1094F00000283FF455AF06EB04140223A3724FE794
:1095000050350024542000249184040870B5104D77
:1095100082B00E462B78022B15D1020AC4B2D5F8C0
:109520003402002301A910440322FFF7E5FE0128BD
:1095300007D12B78019A022B0CBF22F8146042F855
:10954000246002B070BDC0F3D41200F07F04E6E7DF
:10955000503500242DE9F04F434E0D4683B0174699
:1095600031782B6803293DD002295FD14FEA1329B6
:109570004FF4807A5FFA83F8421E012A23D84FF015
:10958000010B9F421AD901288CBF00240124D6F870
:10959000AC211AB1D6F8C81199424AD0D6F8340293
:1095A0000023092201A94844FFF7A6FE012822D082
:1095B000022813D020B12B689F42E8D803202F60E7
:1095C00003B0BDE8F08FB8F1000F12D096F8E83183
:1095D00013B9012386F8E83101237370022003B028
:1095E000BDE8F08F4FF0800AC3F3D41903F07F0871
:1095F000C2E7D346C5E73178022913D00329EDD15C
:10960000019B53F8282022F07042B2FA82F22B68B4
:109610005209A2421FD0D8445B44D0452B601DD2D2
:109620000229EDD1019B33F81820EEE74FF4807A40
:10963000DAE7D6F84412013A02EB41224902B2FBC2
:10964000F1F21344B3FBFBF20BFB12320AB15B44A1
:109650009B1A2B60B0E79F42B2D8AFE709F101092E
:109660004FF00008A8E700BF503500242DE9F04F67
:10967000DFF884918B4685B0174699F800C00968D9
:10968000BCF1020FD9F8345240F08280CEB24FF4D0
:10969000807305EB1125A6EB010890449844B9426C
:1096A00008F1FF38B8FBF3F84AD200F00103A844F0
:1096B0006FF0404A0193BCF1030F07EB0604A8EBDF
:1096C0000503284614BF4FF480728022641A03A950
:1096D000944228BF1446944228BF002E14BF012292
:1096E00000220A32FFF708FE01282AD199F800C0AB
:1096F000DBF800E0BCF1020F0EF1010324D0B4420C
:1097000055D9039806EB0A02011F00EB820201EB18
:10971000840142F8043F8A4203F10103F9D1DBF8E6
:109720000030A11B19448F42CBF8001002D1019BDD
:10973000002B48D18F4205F101054FF00006BAD841
:10974000012005B0BDE8F08FB44246D903986FF010
:109750000042811E324401EB440100EB420222F838
:10976000023F914203F10103F9D1A11B71448F42E1
:10977000CBF80010DED1019B002BDBD086466FF0CA
:1097800000434FF6FF72012023442EF81320D8E740
:1097900001F07F06C1F3D413BCF1030FA6EB01085F
:1097A0001D4414BF4FF480738023904476E7AEEBE2
:1097B000060E0EEB04018F42CBF80010BAD1019BCC
:1097C000002BB7D003986FF040434FF0FF32234493
:1097D00040F82320DBF80010ACE7AEEB060E0EEBF2
:1097E00004018F42CBF80010A4D1019B002BA1D023
:1097F000DDF80CE0C3E700BF5035002430B5044667
:10980000C06983B010B9012003B030BD0D460023FC
:10981000032201A9FFF770FD0128F5D1B4F920203A
:10982000002A19DB019B012D4FEA421103EB421282
:1098300003D0022D1AD1E5205854A368D3612378B0
:10984000032B04D10023137753779377D377636A7D
:10985000190C53839182D6E7054A92F8E81109B9A9
:1098600082F8E801012302205370CDE7E368E5E7C1
:10987000503500242DE9F041022382B004460E4603
:1098800094F83C20042A7BD8DFE802F02D036F4EC9
:109890003E00404D4FF6F777DFF8FC8018E0BC45FE
:1098A00061D857F00DF901284FF00001034637D178
:1098B000206BFFF72BFE0128034631D10199D5F823
:1098C00048024A1E2163824228BF0246C5F8482248
:1098D000287801A9226B03281FFA82FC1046DED1EA
:1098E0004245DED93FE07100204601F0FE01FFF75E
:1098F00085FF0128034643D1626B002A14BF022270
:10990000012284F83C20BBE794F82830042B02D1D4
:10991000002384F82830A36B0BB12046984701231D
:10992000184602B0BDE8F0811A4D0021E26AD5F870
:10993000C83105F5D270C5F8C8219B1AD5F8442264
:1099400002FB03F3D5F8AC2102EB4322C5F8AC21AE
:10995000D5F8B02102EB4322C5F8B021FFF74EFF46
:10996000012803460CD10422CBE7626B04F13001DD
:109970000020FFF77BFE0128034601D10322C0E748
:10998000022BCDD194F82820042AC9D1002284F8D2
:109990002820C5E750350024F7FFFF0F38B50446EF
:1099A00094F83430052B60D8DFE803F031251D131F
:1099B0000D0394F82830082B3FD02D4B01220220B4
:1099C00083F8E92138BD94F82830082B30D00120E5
:1099D00038BD00212046FFF711FF012845D10420A2
:1099E00084F83400DCE7D4E90B01FFF78FFD012890
:1099F0003BD10320F4E74FF0FF31206BFFF786FDEA
:109A0000012832D1E36A002BF3D00220E8E7184D99
:109A100004F130010120D5F83C220232FFF79AFD13
:109A2000012813D00238C0B201281ED80520D7E77C
:109A30000023012084F82830CAE7002301220220F5
:109A400084F828300A4B83F8E921BBE7E368D5F8AE
:109A50004412226B03EB4123C5F84822C4E90332C8
:109A6000E36A002BBCD16262BAE7002038BD00BFB8
:109A700050350024F8B50446022094F83830032B02
:109A800007D8DFE803F021180B0200212046FFF77A
:109A9000B5FE431EDBB2012B3FD9F8BD0120626B3E
:109AA00004F13001FFF7E2FD01284FF00303F0D18C
:109AB00084F83830E1E700211D48FFF79FFE0128B8
:109AC0004FF00203F4D0E4E71A4BE6681A78D3F8B3
:109AD0004412032AD3F8C85114BF4FF48072802275
:109AE000256102FB01F1AF1A2A4406EB4126E6602C
:109AF000D3F8AC61C3F8C821A6EB4126C3F8AC612A
:109B0000D3F8B061A6EB4121C3F8B011E36A256335
:109B1000626353B965620123CAE794F82830062BC3
:109B2000BBD1002384F82830F8BD2763F3E700BFDA
:109B3000F4360024503500244368C3F308020A4475
:109B4000B2F5007F2DE9F041054682B00C4605D202
:109B500023446B60012002B0BDE8F08190F91A2027
:109B6000501C09D04049023201EB0212D17A21F097
:109B70000101D172FF22AA7695F91B20511C0ED04B
:109B800002323948FF2600EB0210C27AC2F34501C7
:109B9000013921EAE17161F34602C272EE762A7858
:109BA000022AD5D0304FD7F84422B4EB422F4FEAE7
:109BB00042282BDCD7F84C621E407242A24225DCC0
:109BC000A2192869424513D32A7E120729D5D7F84E
:109BD000C821411C8A421BD300D100214344A4EB7D
:109BE0000808686108469B1B08EB060429616B6046
:109BF0000028AFD03A78032A31D080B24FF6F772FE
:109C00009042A7D81A4614446C60A3E70020A2E74C
:109C100097F8E82102BB012387F8E8317B706B6875
:109C2000DCE701A956F04CFF0128EFD16B68A4EBEB
:109C3000080428699844297868613444A8EB06032D
:109C4000019802291A466B602861D1D1D7F85412C5
:109C5000B3EB412FD7D37DE701227A70BEE7034AE9
:109C600090423FF677AFCDE750350024F7FFFF0F66
:109C70002DE9F0474FF0010882B0044694F83830DF
:109C8000032B00F2A380DFE803F055170C0200203D
:109C9000236C84F8280003B19847022002B0BDE885
:109CA000F0870022236C84F828200BB120469847C7
:109CB000012002B0BDE8F08723786768022B03D04B
:109CC000434BD3F84C321F40C7F34F272046FFF7D2
:109CD000F1FA3F4E3F1A0546BFB207EB050C0222D0
:109CE00001A9002328461FFA8CF9FFF705FB01287C
:109CF0004FF400724FF00001D0D1019863F0C4FC22
:109D0000E3694FF4007120460BB16368EBB1D6F8FC
:109D10004432013B994547D20135FFF70DFF00283A
:109D2000DBD196F8E83113B9012386F8E83186F8DB
:109D30000180D2E72046FFF731FE012802D0022839
:109D400044D1032084F8380098E7019B4FF020327B
:109D50004FF0100E4FF02E0C42F62E6AC3F8012081
:109D6000C3F80520A3F8092083F800C0D4F824C064
:109D7000A3F820A083F80BE0C3F82220C3F8262024
:109D800083F82A20E26BA3F81AC02CFA0EFC5A873B
:109D900022FA0EF2A3F814C083F82BE09A86D6F8C4
:109DA0004432013B9945B7D3C3EBC3532046590214
:109DB000FFF7C2FE20B996F8E8311BB1012373709A
:109DC0000220BFE7012386F8E831F7E7002065E7C6
:109DD00050350024B1F904300F2B2DE9F0410D4628
:109DE00082B00446164631D02046FFF763FA94F954
:109DF0001B80B8F1FF3F3AD0584F07EB0813DB69DF
:109E0000984211D097F8E831002B6BD001237B707A
:109E10002378022B5CD02269002A71D10023012013
:109E2000336002B0BDE8F081B96901EB4821002937
:109E300064D0AB88204601331BB201EB4311AB80E9
:109E40003160FFF737FA28600120EAE74FF400712C
:109E5000FFF772FE002841D04FF6FF732046AB801B
:109E6000FFF728FA94F91B80B8F1FF3FC4D123789B
:109E7000022B3BD02269002AD0D0384F3B78032BED
:109E800062D093B24FF6F7718B4294BF0023012347
:109E9000002BC1D128B997F8E831002B47D0012316
:109EA0007B700023112201A9FFF726FA012825D192
:109EB0000199BB69CB1A48BF03F2FF13B3F5B05F3A
:109EC0004FEA63222AD24FFA82F884F81B80AEE769
:109ED000D7F854226368B3EB422F9FD2002002B020
:109EE000BDE8F081012387F8E8318FE71B4F6368F5
:109EF000D7F85422B3EB422FCCD38FE7237888E7EF
:109F00003B78032B17D093B24FF6F772934294BF6E
:109F100000230123002B81D10020E0E797F8E831EE
:109F200013B9012387F8E83101237B70CDE70123C2
:109F300087F8E831B3E70A4B9A4294BF0023012324
:109F4000002B7FF46BAFE7E7054B9A4294BF0023E9
:109F50000123002B7FF460AF9CE700BF5035002445
:109F6000F7FFFF0F70B50378044690F818C0023B66
:109F7000012B02D91CF0060F59D11CF0200F39D14A
:109F800094F91A30591C09D02F4A0233FF2102EBF1
:109F90000313DA7A22F00102DA72A17694F91B3007
:109FA0005A1C0ED00233284901EB0311CB7AC3F3BC
:109FB0004502013A22EAE27262F34603FF22CB72C3
:109FC000E2761CF0080F0CD01F4D95F8CC31072B12
:109FD00004D095F8E83193B301236B70002385F822
:109FE000CC310023E26A237084F82830F2B1BDE856
:109FF00070401047144D0023E0692A46D1691032A1
:10A00000884206D001330B2BBAD0D1691032884276
:10A01000F8D1023305EB0315EB7AC3F34502013A9D
:10A0200022EAE27262F34603EB72A9E770BD0121F6
:10A03000FFF7E4FB0128F9D194F818C09DE701234C
:10A0400085F8E831C8E700BF5035002438B5194C11
:10A0500094F814322BB970B190F828201AB1184630
:10A0600038BD002038BD0146442204F5F67063F087
:10A07000ADFA012038BD04F5F675014644222846A4
:10A0800063F002FB237803224FF6FF71022B284670
:10A09000A4F8061218BF1346D4F8501284F804220C
:10A0A000102284F8EC31C4F8101284F805225AF01A
:10A0B000C9FDDEE7503500242DE9F0414FF0FF30B7
:10A0C0002C4C00232246054603E0013310320B2BB3
:10A0D00014D092F82A100429F7D104EB031191F857
:10A0E0002B10CF07F1D46E1C116A01D08842ECD935
:10A0F0001D460133084610320B2BEAD1002D02DA3F
:10A100000120BDE8F081AF1C2E01DFF8708004EB68
:10A1100007131989C1B9A319D8F80020A169D86912
:10A120000023166901EB4521134AB047A0B102286C
:10A1300008D1D4F8D03004EB07170122013BBA72E2
:10A14000C4F8D0300020DCE704EB0513D869D8F858
:10A150000030DB689847DEE7D4F8D03004EB07170F
:10A1600003210122013BB97284F8D420C4F8D03015
:10A17000E8E700BF50350024ED8404085420002493
:10A180000823484041B240000029C0B2B8BF504047
:10A19000013BF7D1704700BF30B5056804468D42DA
:10A1A00018D901F1FF3E681E00231EF801CF0821D7
:10A1B00083EA0C034FFA83FC5B00BCF1000FDBB2B7
:10A1C000B8BF53400139F5D17045EED16A1C226009
:10A1D0002B7030BD00236A1C22602B7030BD00BF85
:10A1E0009FED067AF7EE007A60EE870A60EE800A4D
:10A1F00030EEA70A80EE800A704700BFDB0FC9402F
:10A2000010B52DED028B08EE101ADFED807ADFED30
:10A21000800A0446B8EE488A28EE008A28EE278A8B
:10A22000B0EE480A62F028F99FED7A7AF0EE407AB3
:10A23000B4EEC70AF1EE10FA40F3BD809FED746AE8
:10A24000DFED756AB0EE677A77EEC67AB4EEE67A3D
:10A25000F1EE10FAF6DC9FED717AF4EEC77AF1EECA
:10A2600010FA40F3C5809FED6B7A77EE677A27EEA0
:10A27000A76ADFED6B5ADFED6B6A9FED6B7AE6EE56
:10A28000256A9FED660A67EE865ADFED610A38EEB1
:10A29000000AA6EE267AE5EE877AB0EE678A62F0CB
:10A2A000EBF8DFED5C7AB4EEE70AF1EE10FA5BDD75
:10A2B000DFED576A9FED587AF0EE407A30EE660A8D
:10A2C000F4EEC77AF1EE10FAF6DCDFED547AB4EE74
:10A2D000E70AF1EE10FA62DDDFED4E7A37EEC00AE2
:10A2E000F7EE007A9FED517A20EE004ADFED4C6ADE
:10A2F000DFED4C4A0023B0EE673A9FED4B5AE4EE97
:10A30000264AC4ED097A60EE043AA361A8EE073A42
:10A310006361F0EE675A2362F8EE006AE361A4EE2F
:10A32000245AE8EE475A87EE836AA3EE850AB6EE12
:10A33000007ABDEC028B77EEC07A26EE077A66EEE5
:10A34000266A27EE865A67EE277A25EE866A26EE7B
:10A35000807A84ED015AC4ED007A84ED046AC4ED7C
:10A36000027A84ED037A10BDDFED317AB4EEE70AAC
:10A37000F1EE10FAA9D5DFED266A9FED2E7AF0EE08
:10A38000407A30EE260AF4EEC77AF1EE10FAF6D4EF
:10A39000DFED227AB4EEE70AF1EE10FA9CDCDFED95
:10A3A000267AB4EEE70AF1EE10FA99D5DFED207ABD
:10A3B00037EEC00A94E79FED1E7AB4EEC70AF1EEBD
:10A3C00010FA7FF548AF9FED126ADFED1A6AB0EE22
:10A3D000677A77EE867AB4EEE67AF1EE10FAF6D482
:10A3E0009FED0E7AF4EEC77AF1EE10FA3FF73BAF2D
:10A3F0009FED117AF4EEC77AF1EE10FA7FF537AFE0
:10A400009FED0B7A77EE677A31E700BF27D4D2361B
:10A41000DB0FC940DB0F4940E4CB1641DB0FC93FDE
:10A4200092E741B99730083C15A82ABEF304353F9E
:10A43000DB0F49C0E4CB16C1DB0FC9BFDFED2D0A2E
:10A4400008B562F019F8DFED2C7AB4EEE70AF1EE08
:10A4500010FA28DDDFED276A9FED287AF0EE407ACA
:10A4600030EE660AF4EEC77AF1EE10FAF6DCDFEDB4
:10A47000247AB4EEE70AF1EE10FA2FDDDFED1E7A52
:10A4800037EEC00A20EE007A9FED1E6ADFED1E6AED
:10A49000DFED1E7AE7EE066A20EE076AE6EE877ABF
:10A4A000A6EE270A08BDDFED1A7AB4EEE70AF1EE50
:10A4B00010FADCD5DFED0F6A9FED167AF0EE407AE8
:10A4C00030EE260AF4EEC77AF1EE10FAF6D4DFED9C
:10A4D0000C7AB4EEE70AF1EE10FACFDCDFED0E7A7B
:10A4E000B4EEE70AF1EE10FACCD5DFED097A37EEDB
:10A4F000C00AC7E7DB0FC940DB0F4940E4CB164178
:10A50000DB0FC93F92E741B99730083C15A82ABE36
:10A51000DB0F49C0E4CB16C1DB0FC9BFDFED2F7ADB
:10A52000DFED2F0A30EE270A08B561F0A5FFDFED59
:10A530002D7AB4EEE70AF1EE10FA28DDDFED286A95
:10A540009FED297AF0EE407A30EE660AF4EEC77A93
:10A55000F1EE10FAF6DCDFED217AB4EEE70AF1EE67
:10A5600010FA2FDDDFED1F7A37EEC00A60EE006AC9
:10A570009FED1E6A9FED1E7ADFED1E7AA6EE867AAB
:10A5800020EE266AE6EE877AA6EE270A08BDDFED02
:10A590001A7AB4EEE70AF1EE10FADCD5DFED106AB4
:10A5A0009FED167AF0EE407A30EE260AF4EEC77A86
:10A5B000F1EE10FAF6D4DFED097AB4EEE70AF1EE27
:10A5C00010FACFDCDFED0E7AB4EEE70AF1EE10FA06
:10A5D000CCD5DFED097A37EEC00AC7E7DB0FC93FFC
:10A5E000DB0FC940DB0F4940E4CB164192E741B98C
:10A5F0009730083C15A82ABEDB0F49C0E4CB16C132
:10A60000DB0FC9BFB0EEC07AF0EEE06AF0EE407A40
:10A61000C6FE875AF5EE405AF1EE10FA3BD086FEA0
:10A62000C75A85EE256A9FED1D2A9FED1D3A9FEDC5
:10A630001D4ADFED1D4ADFED1D2AF7EE005ADFED62
:10A640001C3A9FED1C5AA6EE423AE6EE223AA6EEDE
:10A65000034AE6EE235AE6EE044AA6EE245A85EEB5
:10A66000250AF4EEC76AF1EE10FA03D59FED127ACF
:10A6700037EE400AF5EEC00AF1EE10FA03D59FED71
:10A680000F7A37EE400AF5EEC07AF1EE10FA48BFC5
:10A69000B1EE400A70479FED070AE2E739094E3DE7
:10A6A000E3B59E3E88FA163E45FE7F3F99FB243F68
:10A6B00069A2163EA7DFA834DB0FC93FDB0F494074
:10A6C0002DE9F04F884689B01E461178531C03933C
:10A6D000002900F01681002514460746A94609E026
:10A6E00038460135C047039C621C2178039200293B
:10A6F00000F08F802529F3D16078A31C3028CDE9A4
:10A70000033923D0A0F130034FF0000ADBB2092B4C
:10A7100026D96C282AD078287FD8572878D9A0F154
:10A720005803202B79D8DFE803F0BD787878787863
:10A73000787878787882AF78787878787878787858
:10A74000AA787878789E788A7878BD00E31CA0781B
:10A750004FF0010A0393A0F13003DBB2092BD8D8E4
:10A7600004AA03A954F080FB6C28D4D1039B1A7867
:10A770005C1C782A0394B7D8572A40F28E80A2F145
:10A780005803202BB0D801A151F823F0C3A8040826
:10A79000E9A60408E9A60408E9A60408E9A604084D
:10A7A000E9A60408E9A60408E9A60408E9A604083D
:10A7B000E9A60408E9A6040831A80408DFA80408EB
:10A7C000E9A60408E9A60408E9A60408E9A604081D
:10A7D000E9A60408E9A60408E9A60408E9A604080D
:10A7E000E9A6040881A80408E9A60408E9A6040863
:10A7F000E9A60408E9A6040869A80408E9A604086B
:10A80000EFA80408E9A60408E9A60408C3A80408F8
:10A8100028B9284609B0BDE8F08F039C64E72528D5
:10A82000FBD1039C252138460135C0475CE7039CDA
:10A8300056F8041B38460135C9B2C04754E70DF13C
:10A84000140B00220A2156F8040B5B46039CFDF70B
:10A8500027FF5346049A41463846CDF800B0FDF72D
:10A86000B7FE054440E7039C56F8040B0023049A06
:10A87000414600903846FDF7ABFE054434E7039CA3
:10A8800056F8043B1D602FE70DF1140B56F8040B2E
:10A89000039C5946FDF748FFDBE7002AB9D0252A7B
:10A8A000C0D021E7A0F158020DF1140B102156F889
:10A8B000040BB2FA82F25B465209FDF7F1FE039CEB
:10A8C000C7E7A2F158020DF1140B102156F8040B42
:10A8D000B2FA82F25B465209FDF7E2FEB9E70DF1EA
:10A8E000140B56F8040B5946FDF71EFFB1E70DF1A6
:10A8F000140B00220A2156F8040B5B46FDF7D0FE2C
:10A90000A7E70D4685E7F8B5134C07460D461646F2
:10A91000D4F8A802C0B11149FEF77AFC3946D4F840
:10A92000A802FEF775FC0E49D4F8A802FEF770FCE9
:10A930000C4933462A46D4F8A802FFF7C1FE0A495B
:10A94000D4F8A802FEF764FC94F8AC3213B10123EA
:10A9500084F8AD32F8BD00BF503500248AE70B08FB
:10A9600004FE0B080D92040897E70B080EB400B51F
:10A9700084B0084905AB019001A853F8042B039358
:10A98000FFF79EFE0022019B1A7004B05DF804EBF5
:10A9900003B070474D860408F7B50023114E0C46EE
:10A9A000154686F8AE32104904EB45050F4B104FA3
:10A9B000002818BF194606F2AE2006F2AE2662F055
:10A9C0006BFEAC4202D10B4803B0F0BD394634F8FF
:10A9D000022B6846FFF7CAFF6946304662F05CFE0C
:10A9E000EFE700BF50350024A4E70B089BE70B08F6
:10A9F000ADE70B08FE370024F7B50D4D00220446E5
:10AA000000EB410685F8DF2205F2DF25094FB4424D
:10AA100002D1094803B0F0BD394634F8022B68462C
:10AA2000FFF7A4FF6946284662F036FEEFE700BF55
:10AA30005035002485090C082F380024F8B54E1E27
:10AA4000054601F11F04054F16F8012F2846394627
:10AA50000235FFF78BFFA642F6D1F8BDB2E70B082F
:10AA600003685A1C02601970090A03685A1C0260C4
:10AA70001970704702681346511C016013F802CB2D
:10AA80000360D31C5178036093781B0443EA0123CD
:10AA9000111D43EA0C030160D07843EA006070475F
:10AAA000A0F13003092B07D920F0200041381928E4
:10AAB0008CBF0020012070470120704730380928E2
:10AAC0008CBF002001207047413819288CBF00201E
:10AAD00001207047613819288CBF00200120704781
:10AAE00020280BD0092809D00A2807D00D2805D026
:10AAF0000B3801288CBF00200120704701207047CF
:10AB0000A0F14103192B98BF20307047A0F16103D9
:10AB1000192B98BF2038704702B3844610B58418AB
:10AB200003E0981A15D1A44514D01CF8013BA3F1F9
:10AB30004100192811F8010BA0F1410E98BF2033F4
:10AB400000F12002BEF1190FEBD91B1A04D1002825
:10AB5000E9D110BD002010BD184610BD1046704749
:10AB600070B5044608460D465FF09CFD064602E0BF
:10AB700014F8013F43B1324629462046FFF7CCFF87
:10AB80000028F5D1204670BD1C46204670BD00BF90
:10AB90002DE9F043064686469EF800C074460EF145
:10ABA000010EBCF1200FF7D0BCF1090FF4D0BCF1BD
:10ABB0000A0FACF10B00EFD0ACF10D05B5FA85F53D
:10ABC0006D09002DE8D10128E6D9BCF12B0F3DD04D
:10ABD000BCF12D0F39D0102A3ED04FF0FF3E9046E9
:10ABE000BEFBF2FE02FB0EF7FF43FFB2002014F89B
:10ABF00001CBBCF1390F4CF02009ACF1300C0DD871
:10AC00005FFA8CFC944510DA7045264602D819D1BB
:10AC1000674517D21D404FF0FF30E8E7A9F1570C08
:10AC2000B9F1600F5FFA8CFCECD801B10E6003F053
:10AC30000103D5B9002803DA002B18BF6FF00040DC
:10AC4000BDE8F08300FB08C0D1E70125102A94F885
:10AC500001C004F10104C0D1BCF1300F10D06FF07D
:10AC6000704E0F274FF01008C0E7B0F1004F04D925
:10AC70001BB14FF00040BDE8F0834042BDE8F083D7
:10AC800060786FF0704E0F274FF01008A0F141066A
:10AC9000192E04F1010698BF203078280CBF023429
:10ACA0003446A3E701230A22002171E770B50D465F
:10ACB0001446FEF7BDFA0646A0B1FFF7F3FF40F6D3
:10ACC000340319229842A8BF1846B0F5617FB8BF77
:10ACD0004FF46170A0F56173B3FBF2F32B7023782E
:10ACE000013323703046FEF7A3FA0646A0B1FFF702
:10ACF000D9FF40F6340319229842A8BF1846B0F590
:10AD0000617FB8BF4FF46170A0F56173B3FBF2F3DC
:10AD10006B70237801332370304670BD03880021A7
:10AD2000184AA3F5FA6C70B503F0030490F802E03A
:10AD3000154E40F2B5550EF1FF3E04EB44044FEAC8
:10AD40009C0C0EEB8403C47836F81330013C05FBF1
:10AD50000C3390F804C02344847903EB430322446A
:10AD60004FF47A740CEBC30C43790089CCEB0C1CC8
:10AD700003EB8C03C3EB031302EB8302C2FB04015E
:10AD800070BD00BF80436D38A4EC0A082DE9F04186
:10AD900016461F46404D0446394630464FF47A72F7
:10ADA000002360F0DDF83D4B05443D4F3D4E83FBF5
:10ADB0000510E9172844C1EB601183FB0103C81794
:10ADC0000B44C0EB631087FB003CC317C3EBAC0321
:10ADD00086FB03764FEAE37ECEEBE61EC1EB01165F
:10ADE000A5EB860CC0EB00154FEA8E0684F806C072
:10ADF000A1EB8501617103EB4301A0EBC10040F2BF
:10AE0000B55101FB1E332071B3F5896F33DA40F27F
:10AE1000DA218B4237DCB3F5B77F234FB4BF4FF055
:10AE2000000E4FF0010E0EEB4E0175464FEA4E0834
:10AE300007EBC101C88A08EB0E0C0B2107EBCC0C09
:10AE40000CF1160C01E03CF8020D984210DD0139BE
:10AE5000F9D1F044012137F8380006F5FA6E0133D4
:10AE6000A17075441B1A22812580E370BDE8F08132
:10AE70000131C9B2F1E7032540F296500A4F4FF075
:10AE80000608AE46D7E7022540F22940064F4FF0AC
:10AE90000408AE46CFE700BF80BC92C78988888887
:10AEA000ABAAAA2A73B06D16A4EC0A080D4B10B514
:10AEB000D3E9C24354EA03020AD10146002340F217
:10AEC000011218460B80C1F802208B710B8110BD56
:10AED000054A1268121943F10003FFF757FF0120DA
:10AEE00010BD00BF50350024B41D00242DE9F047EB
:10AEF000044688B094F83030042B11D8DFE803F012
:10AF0000481359035200237E9A0640F1DD80002346
:10AF1000112205A9E069FEF7EFF9012800F0D480BD
:10AF200008B0BDE8F087C24D01AE04F11C0705F57D
:10AF3000F679324639464846FEF74CFF012800F0C4
:10AF4000DC800228ECD195F906325F1C09D002336F
:10AF5000FF2205EB031385F80622DA7A22F00102BC
:10AF6000DA7295F907325E1C0ED0023305EB03133B
:10AF7000DA7AC2F34501013921EAE17161F346024F
:10AF8000FF21DA7285F80712042384F83030B1E724
:10AF9000A84859F057FE4FF6FF720123228484F827
:10AFA0003030A7E70020E36A207008B0BDE8F04722
:10AFB00018479F4D95F81432002BB1D104F11C07AE
:10AFC00001AE05F5F678324639464046FEF702FFF7
:10AFD000012840F0E380DDF80490B9F1000F00F0A3
:10AFE000BC8099F800300BB1E52BECD1AB69B9EB23
:10AFF000030348BF03F2FF13B3F5B05F4FEA6322C8
:10B0000080F00B8112018C4B13449A7B042A0CD0E4
:10B01000D5F8CC200132C5F8CC205A6004229A73AE
:10B02000D5F8D0300133C5F8D03095F90632581C28
:10B0300009D0023305EB0313DA7A22F00102DA7247
:10B04000FF2385F8063295F90732591C0ED00233DA
:10B05000FF2105EB0313DA7A85F80712C2F34501E5
:10B06000013921EAE17161F34602DA7220220021FE
:10B07000484662F009FBD4F83120D4F8353005A8F1
:10B08000C9F80020C9F8043094F83B30B4F83920EE
:10B0900089F80A30A9F80820637E89F80B30FFF799
:10B0A00005FFBDF81430002B40F0F78044F28172A8
:10B0B0000321A9F81020A9F80E30A9F81820A9F842
:10B0C000163084F8301015E7204659F0BBFD23698F
:10B0D000002B6AD0237E03F0F70213F004032276DC
:10B0E00070D1122A00F085800022E36A204684F89D
:10B0F000282008B0BDE8F0471847DDF80480B8F113
:10B10000000F00F09B8098F80030002B00F0968034
:10B1100098F80BA01AF0080F7FF40BAF0B2204F184
:10B120003101404662F0A0FB00287FF402AF637E4D
:10B130008AEA0303DF0640F1E68095F906325E1CD9
:10B140003FF40FAF0233FF2105EB031385F806121E
:10B15000DA7A60F30002DA7203E795F8EC3109223B
:10B16000022B3FF411AF95F81432002B7FF40CAF93
:10B1700085F8243285F820322E4885F81422C5E956
:10B180008A33D5F80032C5F81832D5F84832C5F8F8
:10B190001C32FEF76DFD01283FF415AF02287FF445
:10B1A000BFAE042384F83030A4E6237E1B079BD572
:10B1B0001F4B93F8CC21002A7FF4B2AE072283F80C
:10B1C000CC2191E70023A5682046E66A294684F849
:10B1D0002830FEF7B1FC002840F08F8094F828302A
:10B1E000002B7FF49DAE0223C4E90B6584F8283060
:10B1F00096E6E06A0421626AA063204684F83C3047
:10B2000084F8281063636362C4E90B22C4E9023343
:10B2100008B0BDE8F04759F015BD95F8E83113B90D
:10B22000012385F8E83101236FF00F026B70EAE625
:10B23000503500243C3700246C35002495F9063243
:10B24000591C09D00233FF2205EB031385F80622AF
:10B25000DA7A22F00102DA7295F907325A1C0ED01E
:10B26000023305EB0313DA7AC2F34501013921EA0F
:10B27000E17161F34602FF21DA7285F80712237E3D
:10B28000DB067FF581AE3E4859F0DCFC4FF6FF72DD
:10B290000223228484F830302CE605A8B5F9105337
:10B2A000FFF73CFD4FF47A7200235FF059FE3C2318
:10B2B00092B205FB03014FF47A700023C1FB002317
:10B2C00002A8FFF763FD9DF80A309DF80B209DF85A
:10B2D0000E1042EA4312BDF80830A3F2BC7342EAF2
:10B2E00043229DF80D305B0192B243EA51039DF871
:10B2F0000C1043EAC1239BB2DAE6002E3FF410AEF5
:10B300002046334651E6B8F81420B8F81A3043EA1C
:10B310000243D5F8442263625202D8F81C30B3FBD2
:10B32000F2F102FB1131A36009B113445B1AE3602F
:10B3300084F819A095F90632591C09D00233FF226E
:10B3400005EB031385F80622DA7A22F00102DA729D
:10B3500095F907325A1C0ED0023305EB0313DA7A43
:10B36000C2F34501013921EAE17161F34602FF218F
:10B37000DA7285F80712032384F83030BAE500BF8B
:10B380003C3700242DE9F04190F8283082B0044683
:10B39000013B082B0BD8DFE803F0393D1F24052AB9
:10B3A0000A2F34000121FEF765FA012802D002B00D
:10B3B000BDE8F08100222378216C84F82820002B3E
:10B3C000F5D00322E162D4E9010384F82820834206
:10B3D00038BF03462046A36002B0BDE8F041FEF747
:10B3E000C1BD002102B0BDE8F041FEF743BA02B092
:10B3F000BDE8F041FEF73EBB02B0BDE8F041FEF70C
:10B40000CDBA02B0BDE8F041FEF732BC02B0BDE8F3
:10B41000F0416BE5DFF84C814268D8F84C52036B81
:10B420001540D8F8441290F800E0E8184E02B0EB4E
:10B43000412F41D34FF6F777BEF1020F14D02169A7
:10B440000846002963D16068A3680021E26A83424C
:10B4500084F8281038BF0346A360002AA7D02046EE
:10B4600002B0BDE8F0411047D8F854126068B0EB64
:10B47000412F34D22069217E09073AD5D8F8C81166
:10B4800000F1010C614530D298F8E81100294FD144
:10B49000012388F8E83188F80130626894F800E008
:10B4A000236B9B1B32442B44521B00259E4262603F
:10B4B0002363C4E904C0BFD9BEF1020F0ED02169D5
:10B4C0000029C0D098F80000032843D089B24FF675
:10B4D000F7708142B7D898186060B5E76068D8F80F
:10B4E0005412B0EB412FF6D3AEE7DAD14FF0000C97
:10B4F000D7E701A955F0E4FA01287FF458AF206995
:10B50000DDF804C094F800E06268236BC9E798F89E
:10B5100000C0BCF1030F11D01FFA81FCBC4594BFE1
:10B520004FF0000C4FF0010CBCF1000FC8D1A2E7A6
:10B53000012188F8011094F800E0B2E7DFF820C09C
:10B54000614594BF4FF0000C4FF0010CBCF1000FAF
:10B55000B6D190E7024881423FF675AFBBE700BF26
:10B56000F7FFFF0F503500242DE9F0410446154642
:10B5700008469442B4FBF2F607D205FB1644134B7F
:10B580001B5D00F8013BBDE8F0819642B6FBF2F787
:10B590000CD20E4B05FB176705FB1644DA5D1B5DED
:10B5A00000F8012B00F8013BBDE8F081BA42B7FB7F
:10B5B000F2F807D905FB1878044B13F8082000F8B7
:10B5C000012BE7E74046FFF7CFFFF3E7FC720B08DC
:10B5D00030B56F4C83B0B4F84037B3F57A7F03D9F8
:10B5E0004FF47A73A4F84037B4F84237B3F57A7F52
:10B5F00003D94FF47A73A4F84237B4F84417B1F57D
:10B600007A7F04D94FF47A731946A4F84437B4F812
:10B610004607B0F57A7F03D900231846A4F84637C9
:10B62000B4F84837B3F57A7F4CD94FF47A73B4F84D
:10B630004A279A42A4F8483749D900238842A4F8F7
:10B640004A3780F08F80B4F85627B4F858379A42BA
:10B6500002D90023A4F856374E4B1B88EBB14E4D50
:10B66000AA78062A52D9297900297ED19FED4B7AF2
:10B6700094F8602707EE903AAB7906EE902AF8EE40
:10B68000E77AB8EEE66AC6EE276A0BB137EE077ABC
:10B69000B4EEE67AF1EE10FA46DC94F86927032A54
:10B6A00025D83F4B03EB421394F86827C4F878374A
:10B6B000032A14D8EA213B4B02FB0133C4F87C3740
:10B6C00003B030BDB4F84A27B2F57A7F18D8884263
:10B6D00012D29A42B7D30023A4F84837B3E7002226
:10B6E000304B84F86827C4F87C3703B030BD0022A3
:10B6F0002B4B84F86927D7E70021A4F84417E8E723
:10B7000000228842A4F84A27E3D3F5E7264901EB53
:10B71000820191ED187A29790029A9D0531F032BB2
:10B72000BBD9002AB9D025E067EE877ABCEEE77A6C
:10B730008DED017A9DF8043007EE103AB8EEC77A25
:10B74000F4EEC77AF1EE10FA01DD0133DBB2EBB1B2
:10B75000102BA8BF1023DBB2934238BF134684F8E6
:10B7600060379AE7A4F844376DE7053A032A94D97D
:10B770009FED0A7AB7EE000A80EE070A60F0EEFE4F
:10B780002B88834228BF03462B8086E70123E2E70C
:10B7900050350024481C00202C2F00246F12033841
:10B7A00064380024E4380024A4EC0A082DE9F04FA2
:10B7B0009D4E83B096F8803700AFA3F11702022A9E
:10B7C00000F29B82994B7B6096F898370024DFF853
:10B7D00078A23B60964B03F1780998461FE098F9F0
:10B7E0000410142900F08482584662F0FDF81BF41E
:10B7F000003F21D0012800F07B82082800F37882E6
:10B8000015B11BEA0A0F06D1396858465CF0C4FE30
:10B81000002800F06D8208F10C08C14512D0D8F85C
:10B8200000B01BF00105DAD05846013462F0DCF8B4
:10B830001BF4003FE4B2DDD10128DEDC08F10C0886
:10B84000C145ECD1013C022C00F2528200230220BF
:10B8500086F840380EF026FE96F84838D6F8445858
:10B86000022B00F0ED82002800F04383714B4FF46F
:10B870007A7E96F8A5A84FF0000C03F56A794FF090
:10B88000640B33F8082CB2F57A7FB3F8462088BFF2
:10B8900023F808ECB2F57A7F33F8062C88BFA3F8BA
:10B8A00046E0B2F57A7F33F8042C88BF23F806EC23
:10B8B000B2F57A7F02D9002223F804CC33F8061CB3
:10B8C0009142B3F85A10B3F85C2098BF23F806CC25
:10B8D000914293F86B2003F1650102F1FF3288BFBA
:10B8E000A3F85AC0632A93F86C2002F1010288BFC2
:10B8F00083F86BB0D2B2092A4FF0000288BF83F8F8
:10B900006CC013F83200013211F8014F844238BF85
:10B9100081F800C0032AF4D1BAF1010F03F1EA0360
:10B9200018BF03F864CC9945ABD1DFF8209199F8A2
:10B930000230042B00F0B1822BB9B9F80030B3F516
:10B94000F07F00F2F881FFF743FE3B4896F8B81805
:10B95000FDF7CEFB103096F8D718FDF7C9FB103075
:10B9600096F8E718FDF7C4FBB6F8F628B6F8F438F1
:10B970001343B6F8F82813431BB213B10123A6F8FA
:10B98000FA382E4B2B40002B00F0C082E80700F164
:10B990007182690400F1D4812A0740F13E82284A6D
:10B9A000D6F8983815401340C6F84458C6F8983869
:10B9B0002C0440F11782002386F89F3786F8AF37B2
:10B9C000E80440F1198296F80739022B02D10123CD
:10B9D00086F80739DFF86CA053460AF1780402E0D4
:10B9E00006339C420CD01A780A2AF9D19978DA7871
:10B9F000914202D35A79002AF2D00A2021F0E4F8C9
:10BA000000234FF4806086F840380EF04BFD00288C
:10BA100000F05C820B4DAB469BF8051019B39BF808
:10BA20000000F0B1534616E050350024A4EC0A089B
:10BA3000143D0024EE380024183E00240960000262
:10BA4000FE9FFFFD5C3E0024BC0202002C2F002460
:10BA500006339C4207D01A788A42F9D15A79002AD3
:10BA6000F6D021F0B1F80BF1060B5C45D4D199F872
:10BA700002A0BAF1080F00F0D58196F8A53896F823
:10BA80003D27A3F10103032AB3FA83F34FEA5313CB
:10BA900086F8843996F8A638A3F10103B3FA83F344
:10BAA0004FEA531386F88A39D6F89838C3F3C03171
:10BAB00086F8871902D9002286F83D27BA49D6F8B8
:10BAC00044280B400A4096F87617C6F89838C6F80E
:10BAD0004428002900F0D081B6F8A039002B40F0AE
:10BAE000BF81D6F8A439B3F5000F02D30023C6F8FE
:10BAF000A439D6F8AC39AD4A1A401AB140F2022343
:10BB0000C6F8AC3996F8A839013B042B02D90123B9
:10BB100086F8A839AAF1050AA54BBAF1030F93F8E4
:10BB2000908540F23681B8F1000F1CD000233B60B5
:10BB3000DFF8A8A206E0ABF1060BABEB090BD8458A
:10BB400040F20081D3461AF8010F0028F3D007F025
:10BB500001FE0028EFD081798B07ECD53B680122EC
:10BB6000002B40F0F48099F8063013B1002389F8D7
:10BB70000630B6F8B63903F00F02042A03D8C3F32F
:10BB80000313022B03D94FF42063A6F8B639B6F895
:10BB9000B83903F00F02042A03D8C3F30313022BAE
:10BBA00003D940F60123A6F8B83996F8291A96F871
:10BBB000352A96F8283A914205D9002286F8292A92
:10BBC00053B1A6F82C2A96F8342A9A4204D20023BC
:10BBD00086F8283AA6F82C3A96F82A2A96F81E3BB8
:10BBE0009A4202D9002386F82A3ADFF8F4C10CF110
:10BBF000800B6346796813F8032D02EB42020A4476
:10BC000092F834A292F8359292F836E213F8010FC6
:10BC100099795045DA78A8BF50464945A8BF4946AA
:10BC200072451870A8BF724663459971DA70EDD1FC
:10BC300003F1200CDC45DCD1D6F8BC27002A00F04B
:10BC400023810020012102E00635AC420ED02B7882
:10BC50002B2BF9D16B78043301FA03F31342F3D0A1
:10BC6000063522EA03020120AC42F0D108B1C6F841
:10BC7000BC27504C6D4604F10808234601E0984566
:10BC800073D013F8012F072AF9D9002304F8013FD4
:10BC90000133082BFAD1B6F89E28AD46B6F89C3889
:10BCA0009A4202D3444BC6F89C38444BFF22444C82
:10BCB00003F1780086F8502B13F9082C142A05D0CC
:10BCC00053F80C1C34EA010100F0E4800C33984274
:10BCD000F2D13C4A5379012B04D0022B04D13A4BC8
:10BCE0001B790BB9002353710C37BD46BDE8F08FAB
:10BCF000364937484CF0D2F8A8E5364A11467A6002
:10BD0000DA0001EBC30393F87C1021B1D3F8803043
:10BD1000002B00F0D7807B68134493F87D20002A25
:10BD20003FF452AD93F85C31002B7FF44DAD1823F6
:10BD300086F8803748E54FF4F073A9F8003002E642
:10BD4000254A2DE63B680022002B3FF40CAF99F802
:10BD50001130002B7FF40DAF99F80530012B3FF423
:10BD600002AF002A7FF4FFAE03E788B02022FF2154
:10BD7000E946484661F088FC0E4A03E0424549F82E
:10BD8000233088D012F8013F59F823100131F5D043
:10BD90007BE7002389F80430B8F1000F00F0B4808D
:10BDA00001233B60C4E600BFBDD77718FDFDFFFF50
:10BDB000481C00203E2F0024AE014A01203D0024F3
:10BDC0000100020058310024A82A0024143D002458
:10BDD000A85B0C08A4EC0A08F6DFFFFD332F002453
:10BDE0006938002496F89F37002B7CD00023E804A4
:10BDF00086F8AF373FF5E7AD29067FF5E4AD96F855
:10BE00008027182A04D8464BD340DA073FF5DBAD2C
:10BE1000DFF81CA10AF17804F2E5AB047FF5C8ADA8
:10BE2000404ABDE599F80630002B3FF426AE99F85C
:10BE30001130012B7FF421AE022389F811301CE66A
:10BE400000283FF413AD90F904404FF0FF0901E0E2
:10BE500080F8089020460EF015FB0028F8D105E583
:10BE600096F89C0907F076FC00287FF43AAEA6F815
:10BE7000A00936E62C4A93E52C490A430B43C6F841
:10BE80004428C6F8983827E62B2020F09DFED6F8E7
:10BE9000BC27D6E686F8502B1BE7D6F8983825F451
:10BEA000805523F48053C6F84458C6F89838B9F83A
:10BEB0002030B3F57A7FBFF446AD4FF47A73A9F81A
:10BEC000203040E5172386F8803724E7D6F8443839
:10BED00023F00063C6F84438D6F8983823F000639E
:10BEE000C6F8983896E542F201031D427FF47EAF12
:10BEF00066E5D6F8983825F0800523F08003C6F86B
:10BF00004458C6F89838B1E4424620E7D6F8983845
:10BF100045F0080543F00803C6F898383FE500BF30
:10BF200000410001F6BFFFFDF79FFFFD0004050083
:10BF30005C3E00242DE9F04F844E83B096F8543BCC
:10BF4000013B012B40F2EC80D6F8842B804BDFF8CC
:10BF5000208202F2DC524345C6F8842B80F0F28046
:10BF6000DFF8109201229B467A4D09F102070192F7
:10BF7000B9F80210002900F0BD80052907EB010285
:10BF800040F2B880AA4280F0B580BBF800003C4681
:10BF9000C0F30B000BE0118814460A44002900F09E
:10BFA000A980AA4280F0A680052940F2A38061887A
:10BFB0008142F0D161798B07EDD123885846DBF8B7
:10BFC000081094F804A000934BF068FFBBF8001031
:10BFD000BAEB113F00F0948000230193BBF80410EA
:10BFE0000BF11C0B5BF8140CC1F30B015BF8044C58
:10BFF00054F010F8C3452060BAD3D6F84438564CF4
:10C00000C6F89838FFF7D2FB96F86837EA22534D06
:10C0100003FB0242A4F18003C6F87C2796F8692747
:10C0200003EB4213C6F878371FF0CCFF4FF0FF3315
:10C03000D6F87C072B6528F0BBFA20F00BFE04F540
:10C04000AF6304F5BE6102E00633994262D01A780C
:10C05000002AF9D19C78D878844202D358790028F4
:10C06000F2D096F80439B6F8081985F8542003EB95
:10C070008303642203EB830302FB01F100229B0094
:10C080006429C6F8842BC6F8882BB8BF6421642BBA
:10C09000C6F88C2BB8BF6423C6F8801BC6F8981B63
:10C0A000C6F87C3B2E492F4BC6F8902BC1F83C3785
:10C0B000C6F8942BA6F89C2B86F89E2B2FF0B6FB87
:10C0C00096F8A21BB6F8A00B22F0E8FB3EF0CAFDE2
:10C0D00018F06EFF96F8543B013B012B2AD9224BF6
:10C0E000012201981B6886F89D2BC6F8843B03B09B
:10C0F000BDE8F08FDBF8081058464BF0CFFE6BE739
:10C10000009BA11D58469A1F4BF0FEFE00287FF4AD
:10C1100065AF61E796F87727003A18BF0122A0E7DC
:10C12000F5F7EEFB114B0222034486F8742BC6F898
:10C13000703B09E7F5F7E4FB0223C6F8700B86F8BD
:10C14000743BCCE70123019357E700BF503500242F
:10C15000AC5A0C0800000408E43800244C04002405
:10C16000481C0020443E0024B41D002460E3160057
:10C17000BC640C0800000208114B0122032810B512
:10C18000044683F8442705D9601CBDE81040C0B2BE
:10C190000EF0F8BA0B4BEA2203F5657083F8684796
:10C1A00004FB0200C3F87C0728F002FA25F096FB96
:10C1B00025F078FC601CBDE81040C0B20EF0E2BA79
:10C1C000481C002050350024054B0121D3F8A82B32
:10C1D00083F8A41B42F40012C3F8A82B704700BFD9
:10C1E0005035002470B5046886B005460E46C4F389
:10C1F00010033BBB01220393CDE901332023CDE99A
:10C20000042304F17843B3F5801F19D3A4F101632B
:10C21000B3F5801F10D2A4F58013022203F17843F6
:10C22000694601A802925B0C03934DF051F848B1A6
:10C230004FF0FF3006B070BD55F0EAF955F0EAFF57
:10C240002346EBE73146204654F0B2FF18B92B687D
:10C2500020332B60EEE76FF00200EBE72DE9F041B1
:10C260006A4E90B03378B12B7ED1FCF76DFB80F035
:10C270000104E4B2664B04F00104664DB3F84332A6
:10C28000654FADF80030BD4270D3002C00F0BC808B
:10C290002822002106A861F0F7F9604B04969B1B49
:10C2A00005935F4BDA68D40770D45D4BD3F80C214B
:10C2B000D00774D44FF480730222694604A8ADF805
:10C2C0003C305DF0FFF8022269464FF6FF70514D99
:10C2D000FCF760F94FF000080446BD4269D3002521
:10C2E000022201A904A8ADF804505DF0EBF8022287
:10C2F00001A92046FCF74EF940BA022202A9C04328
:10C30000ADF8080004A85DF0DDF80E9888B106AB22
:10C31000C0F120022946184461F0B6F99DF93C00AD
:10C3200018B906A904A8FFF75DFF00238DF83C00AB
:10C330000E939DF83D307BB1394BDA6842F0010233
:10C34000DA60DA68D20707D5D3F80C2142F001028F
:10C35000C3F80C21D3F80C319DF93C00B0FA80F001
:10C36000400910B0BDE8F081012483E7AB691C35BA
:10C3700035F8181CD3F8008055F8140CC1F30B01E4
:10C3800053F048FE804518BF01247CE7254A5A60D7
:10C3900002F188325A60DB68D90786D58AE7214ADC
:10C3A000C3F8042102F18832C3F80421D3F80C3118
:10C3B00080E7AE8802A904A88DF80D80C6F30B06AD
:10C3C0001C35B31DADF8083035F81C3CC3F30B0227
:10C3D0001B0BADF80A2006228DF80C305DF072F8C8
:10C3E000062202A92046FCF7D5F8044655F8141C8D
:10C3F000324604A85DF066F8204655F8141C324613
:10C40000FCF7C8F8044668E70120AAE70000020824
:10C41000A4EC0A08AC5A0C08BC640C080000040820
:10C42000002000522301674570B5274CFFF7BEF985
:10C4300094F8543B013B012B34D9D4F8843B0122BE
:10C440000325224E03F2DC5384F8AC2BC4F8843B62
:10C45000FFF704FF58B13378B12B08D1FCF774FA19
:10C46000013D0AD058B9FFF7F9FE0028F3D1013D8C
:10C47000EED155F0CDF855F0CDFE0028F9D094F866
:10C48000543B0022013B84F8AC2B012B14D9104BF8
:10C49000012100221B6884F89D1B84F8AD2BC4F891
:10C4A000843B70BDF5F72CFA0A4B0222034484F852
:10C4B000742BC4F8703BC0E7F5F722FA0223C4F8E6
:10C4C000700B84F8743BE2E750350024000002084A
:10C4D000B41D002460E3160010B5084A0124084B7F
:10C4E00082F8444783F87647FFF79EFFFFF722FD67
:10C4F0002046BDE810400EF045B900BF481C0020A2
:10C500005035002490F89230B7EE007ADFED6A6A79
:10C51000014607EE903A90F89630684AB0EE476AC6
:10C5200005EE103A90F89430F8EEE77A04EE903A7F
:10C5300090F89530B8EEC55A05EE903A90F89830DC
:10C5400067EEA67A04EE103A25EE265AF8EEE44A93
:10C55000F8EEE55AB8EEC44A25EE275A64EEA64A2C
:10C5600065EEA65A24EE264A64EE854A65EEA75A81
:10C5700024EE274AB0EE473AF0B590F8917000F1FA
:10C580006F0602F118050024137807EE903AF8EED2
:10C59000E77A67EE857A67EE867AFDEEE77A17EE40
:10C5A000903AFA2BA8BFFA2323EAE3730B7253786D
:10C5B00007EE903AF8EEE77A67EEA47A67EE867AAD
:10C5C000FDEEE77A17EE903AFA2BA8BFFA2323EA9A
:10C5D000E3734B72937803EE903AF8EEE33A63EE2E
:10C5E000A57A67EE877AFDEEE77A17EE903AFA2B96
:10C5F000A8BFFA2323EAE3738B72938807EE903A7D
:10C60000F8EEE77A67EE847A67EE867AFDEEE77AEF
:10C6100017EE903AD5ED007AB3F57A7FF8EEE77A27
:10C62000A8BF4FF47A7323EAE3738B812B68002B46
:10C630003FDD90F89730B0EE436A02EE903AF8EEA4
:10C64000E22AA2EEE66A63EE863A83EEA76AA2EEDB
:10C65000A66A65EEA77A013467EE877A67EE867A76
:10C66000FDEEE77A17EE903AFA2BA8BFFA23BC4208
:10C6700023EAE37306F8013F00DDF0BD012C13D17E
:10C6800090F8933007EE103A90F89B3006EE103A8F
:10C69000B8EEC77AB8EEC66A27EE267A26EE266A84
:10C6A0000435083208316FE7B7EE007AB0EE476A1A
:10C6B000F6E7B7EE006ACCE70AD7233CB4F30A08E2
:10C6C00090F899306BB3B0F864308BB190F89A2041
:10C6D000642102EB8203C3EB0313B3FBF1F3A0F875
:10C6E0006430962312FB03F3B3FBF1F3A0F866303A
:10C6F00043884BB190F89A30642203EB8303C3EB79
:10C700000313B3FBF2F34380B0F850304BB19622E1
:10C7100090F89A3013FB02F36422B3FBF2F3A0F813
:10C720005030704790F821304BB3438B83B190F871
:10C730002230FA22642113FB02F203EB8303B2FBE3
:10C74000F1F2B3F57A7F4283A8BF4FF47A73838303
:10C75000838843B1FA2290F8223013FB02F364225B
:10C76000B3FBF2F38380C3884BB190F8223003EB24
:10C770008303B3F57A7FA8BF4FF47A73C380704701
:10C7800010B5064C4FF48072002104F5C87060F0BB
:10C790007BFF0023C4F8903210BD00BF4846002440
:10C7A000034BD3F8940208B106F0F0B8704700BF0D
:10C7B0004846002408B50B4605490246D1F89402C4
:10C7C00028B10449FDF77CFFBDE80840E8E708BD53
:10C7D000484600240D920408024B0146D3F8940207
:10C7E000FCF716BD484600240048F5E756EC0B0858
:10C7F0000CB4C30607B500D561B905A90498019129
:10C80000FFF7D8FFFFF7F0FF012003B05DF804EB5E
:10C8100002B070470020F8E708B5FFF7DDFFBDE87C
:10C820000840E1E710B504460348FFF7D5FF20466E
:10C83000BDE81040F0E700BFB7E70B08034B014627
:10C84000D3F8940208B106F08DB87047484600242A
:10C850000CB407B510F020000BD079B92320FFF7F6
:10C86000EDFF05A904980191FFF7A4FFFFF7BCFFB6
:10C87000012003B05DF804EB02B070470020F8E738
:10C880000FB407B504A951F8040B0191FFF792FF0B
:10C8900003B05DF804EB04B0704730B52A4885B0AA
:10C8A000FFF79AFF294B1B7923B9294805B0BDE84A
:10C8B0003040B1E7FBF75CF908B92648F6E7FBF72B
:10C8C0006FF908B92448F1E7244B1B68DB699847E6
:10C8D0000028F7D0FBF744F902680446037D81790C
:10C8E0005208407CE51D0C34029020790190E088CC
:10C8F00000901B48FFF7C4FF15F8010BFFF79EFFE0
:10C90000AC42F9D1174C1848FFF766FF6378022B49
:10C9100006D007D9032B0ED11448FFF75DFF0AE0BC
:10C920001348FAE71348FFF757FF94F8E831022B52
:10C9300005D0032B05D005B0BDE8304054E70E48C4
:10C94000EBE70E48E9E700BFBCE70B08A82A002484
:10C95000C6E70B08D5E70B08E3E70B0854200024D3
:10C96000F2E70B085035002420E80B0826E80B08F6
:10C970002CE80B0839E80B083FE80B0858E80B08CF
:10C980000FB407B504A951F8040B0191FFF712FF8A
:10C99000FFF72AFF03B05DF804EB04B070470349CA
:10C9A000034801F500610EC9EAE700BF00E0F11F8E
:10C9B0006AE80B080EB403B503AA52F8041B0192EF
:10C9C000FDF7A1FF074BD3F894322BB9064B07496B
:10C9D000D3F8A802FCF71CFC02B05DF804EB03B02E
:10C9E000704700BF484600245035002456EC0B0821
:10C9F0000EB403B503AA52F8041B0192FDF783FF9E
:10CA0000054B0649D3F8A802FCF702FC02B05DF81A
:10CA100004EB03B0704700BF5035002456EC0B0800
:10CA2000154BD3F8A83D2DE9F041044688B0F3B189
:10CA30001A6804A91846D56A6A46A847064688B106
:10CA400004AC6D460027DFF83C80013735F8022B37
:10CA500034F8021B4046FFF793FFBE42F5DC08B0F6
:10CA6000BDE8F08105492046FFF7C2FFF7E704491A
:10CA700008B0BDE8F041BBE75035002498E80B084A
:10CA8000B0E80B087EE80B0870B5054608460C4672
:10CA90005DF008FE024668B1062804D12146084828
:10CAA00060F0E2FE30B12846054B064A0649BDE873
:10CAB00070409DE702490548BDE8704060E700BF4F
:10CAC000B7E80B08BEE80B08C9E80B08F3E80B0849
:10CAD00070B5054608460C465DF0E4FD024668B1B7
:10CAE000032804D12146084860F0BEFE30B1284634
:10CAF000054B064A0649BDE8704079E702490548FA
:10CB0000BDE870403CE700BF01E90B0805E90B08F0
:10CB1000C9E80B0815E90B082DE9F04307469BB05F
:10CB200008460C465DF0BEFD06462022002101A805
:10CB300060F0AAFD2EB3402E07D0402332463A497A
:10CB400038461BB0BDE8F04352E701AD04F14008A0
:10CB50004FF0000902222146684660F097FE00234C
:10CB6000102209A968468DF80290FEF711F8099B7A
:10CB70000DF10202934223D1023405F8010BA045C6
:10CB8000E8D109AC41220021284D204660F07CFD0F
:10CB9000002E3CD095F89862D6B1202205F299215A
:10CBA00001A860F0C5FE98B105F299212046FDF775
:10CBB00045FF23461E4A38461E49FFF719FF04E089
:10CBC0001A7838461C49FFF713FF1BB0BDE8F08305
:10CBD00095F8B932DBB9D6B901AB184E1A4608360A
:10CBE00003CAA24246F8080C46F8041C1346F5D1C5
:10CBF00001232046114985F8BA32FDF71FFF10487E
:10CC0000FFF710FE21460F48FFF7BAFEDDE795F863
:10CC1000BA321BB995F89832002BF3D00749204659
:10CC2000FDF70CFFEEE700BF28E90B08484600249B
:10CC300066E90B08C9E80B084AE90B08E14800243B
:10CC400070E90B087FE90B082DE9F74FDFF81C812D
:10CC5000834608460C465DF025FDD8F84478064624
:10CC600028B1024632492046FDF756FF80B93946C1
:10CC7000304851F04DFF3049304821EA070151F06A
:10CC800047FF2F492F4803B0BDE8F04F51F040BF98
:10CC900023782D2B23D10134013E4FF0010A2A4B7A
:10CCA0004FF000094FF0FF3553F8041B51B13246E5
:10CCB00020460193FDF730FF0028019B0ABF4D4637
:10CCC0000021012109F10109A1B9B9F11D0FEBD131
:10CCD00022461E49584603B0BDE8F04F88E64FF0A3
:10CCE000000ADCE73B431A49C8F84438194B12E004
:10CCF000194913E00123104AAB401A40002AF7D02B
:10CD000007EA0302BAF1000FECD027EA0303134944
:10CD1000C8F84438124B002A18BF1946114B124864
:10CD200003EB8503D3F8342703B0BDE8F04F27E6C3
:10CD300029F80B08B7E90B08BDD77718C1E90B082C
:10CD4000422888E7CDE90B08D8F30A08DBE90B088D
:10CD5000AFE90B08A8E90B088CE90B0898E90B0868
:10CD60009FE90B08A4EC0A08AAED0B085035002433
:10CD70002DE9F74F019008460E46174698465DF09C
:10CD800091FC0446E0B93E4D3E48FFF779FD204650
:10CD90000DF008F93B68184206D020460DF014F952
:10CDA00001462846FFF76CFD0134172CEFD13B6894
:10CDB00013B93548FFF710FD03B0BDE8F04F13E598
:10CDC000024632493046FDF7A7FE0546A8B92C4673
:10CDD0002F4D3048FFF700FD20460DF0E3F810EA34
:10CDE000080F06D020460DF0EFF801462846FFF761
:10CDF00047FD0134182CEFD1DEE733782D2B28D1F5
:10CE00000136013C01254FF0000948F4000B48466B
:10CE10000DF0DAF82246824601463046FDF77CFEE8
:10CE200010BB48460DF0BEF81BEA000F1CD095B1B0
:10CE3000B9F1170F02D03B6840EA03081648C7F85B
:10CE40000080FFF7C9FC5146114803B0BDE8F04F20
:10CE500096E50025D7E7B9F1170F02D03D6825EA1E
:10CE600000050E483D60ECE709F10109B9F1180F22
:10CE7000CDD132460A49019803B0BDE8F04FB7E57D
:10CE8000F4F60B08ECE90B08F6E90B0829F80B0897
:10CE9000F5F60B08FDE90B089FE90B08AFE90B0855
:10CEA000DBE90B0840F20223004A61E7FC3E002464
:10CEB000014B024A5CE700BFFFFF7F00F43E002405
:10CEC00008B50C4B93F8542B032A05D193F8553B26
:10CED000092B05D00D2B09D00749BDE8084087E58F
:10CEE0002DF092FC0548BDE8084049E52DF06EFDA7
:10CEF000F8E700BF5035002408EA0B0817EA0B08D2
:10CF00002DE9F04798460B7981460F4603F0E0057E
:10CF10001646402D32D10024614DDFF8A081DFF8A4
:10CF2000A89116E03B7903F00703013B042B04D8DA
:10CF3000DFE803F014171A1D2100315D5848FFF790
:10CF40009FFC7B79013BA34202DD4846FFF744FC8E
:10CF500001347B79A342E5DCBDE8F08731572846F0
:10CF6000EDE736F81410FAE736F91410F7E756F83B
:10CF700024104046E3E756F82410F0E703F00703D7
:10CF8000052B56D8DFE803F0031E26282B3D347806
:10CF9000602D54D02BD8002D72D1B7F80550B7F8BA
:10CFA000076021463E48FFF76BFCAC4238DBB442D9
:10CFB00036DCB8F1000FCFD0324629463948BDE8FB
:10CFC000F0475DE496F90040602D38D00FD8002D71
:10CFD00056D14FE03488DBE7B6F90040F4E7D6F8E5
:10CFE00000A0202D54464BD033D9602D27D0802D62
:10CFF000B2D132782C4B2D48002A14BF3146194645
:10D0000034E0202D34683BD0EFD821462448FFF788
:10D0100037FCD7F80510A14202DB4B42A34220DDCA
:10D02000FFF7E2FB23463A6848462149BDE8F0474E
:10D03000C0E4202D23D01CD9602DD8D100247B79C9
:10D0400044FA03F3DB07BDE8F0474CBF19481A4820
:10D0500016E451461948FFF713FCD7F805108A4526
:10D06000DED8B8F1000F3FF477AF1548BDE8F047C0
:10D0700006E40024B7F90550B7F9076091E70024EA
:10D080007A79104B03EBC20393F8AC27A242C7DDB9
:10D09000D3F8A83753F82400BDE8F047FFF79CBB4E
:10D0A00086090C0867EE0B0863030C086CF30B0889
:10D0B0002AEA0B08CAEA0B08960A0C0862EA0B086F
:10D0C00024EA0B08A4EC0A0822EA0B08F0B506795A
:10D0D00006F0E003402B03D145794FF0FF3406E022
:10D0E000602B4FF00105F8D1447905FA04F40023D0
:10D0F000012006F00706AB4200D1F0BD052E0FD887
:10D10000DFE806F00308101D242448B1C85CD75C92
:10D1100078400FE020B1C856D756C71B78427841F7
:10D120000133E8E70028FBD031F8130032F8137020
:10D13000784080B220420CBF01200020F0E7002898
:10D14000EED031F9130032F91370E6E70028E7D08A
:10D1500051F8230052F82370DAE708B50346104669
:10D160000AB9002008BDDB0601D50029FAD0FFF777
:10D1700059FBF6E7F8B50D4E054696F8B93293B966
:10D18000F8BD25B12388C3F30B039D4204D0A288C8
:10D19000D4E9020160F01AFA1C34BC42F1D3002336
:10D1A00086F8B932ECE7024C024FF6E74846002415
:10D1B000AC5A0C08BC640C08037903F01803102B5C
:10D1C0001ED003D833B9B0F80B007047182BFAD033
:10D1D00000207047124BB0F80B0093F91831591C1E
:10D1E0000CD1104B93F8683703EB430203EB820337
:10D1F00003EBC30300EB430080B27047DBB2F3E7FD
:10D20000074BB0F80B0093F919315A1C05D1054BA7
:10D2100093F8693700EB4310EEE7DBB2FAE700BFA3
:10D220004C0400245035002470B50546B0F80900C0
:10D230004AF01EFE064B0446284693F8B962FFF7F3
:10D24000BBFF16B1E368184470BDA368FBE700BFDD
:10D25000484600242DE9F04F164685B0334C1A4657
:10D260004FF00009A246CDE9010100213046FFF749
:10D2700074FF06F0100300900393FFF791FA2379EF
:10D28000029A03F01803934203D0002A44D1182BCA
:10D2900042D14FF00D0B0BFB09A3B3F809004AF084
:10D2A000E7FD80462046FFF787FF0746D8E90221C1
:10D2B000024401442046FFF709FF80F001010546C2
:10D2C000009AC9B23046FFF748FF039B009003B1B4
:10D2D00015BB0BFB09FBB3065AF80BB00ED56DB9A5
:10D2E00059461348FFF7CCFAD8F808202B462146B8
:10D2F0003A440198FFF704FEFFF776FA59460D48C5
:10D30000FFF7BEFAD8F80C20002321463A440198D2
:10D31000FFF7F6FDFFF768FA09F1010940F29323E0
:10D320000D349945A9D105B0BDE8F08F74040B0800
:10D3300044EA0B0845EA0B0870B5164605460C464C
:10D340000846FFF771FF3346024621462846BDE8EE
:10D350007040D5E52DE9F041037903F0E002402A61
:10D360004DD009D83ABB03F00703052B1ED8DFE8E0
:10D3700003F0181D181D0910602A47D0802A41D0DB
:10D38000BDE8F081D0F805102348BDE8F041FFF773
:10D39000F7BAD0F8052051422048BDE8F041FFF728
:10D3A000EFBAB0F80720B0F80510F5E7B0F907209C
:10D3B000B0F90510F0E746790024194D194805EB3E
:10D3C000C605FFF709FA012395F8AC77A74203D801
:10D3D000BDE8F041FFF708BAD5F8A8674FEA84081E
:10D3E00056F824204AB113B90F48FFF7F5F956F85B
:10D3F00008100E48FFF744FA00230134E6E74179AC
:10D400000B48C2E7827941790A48C6E70A48BDE875
:10D41000F041FFF7B5BA00BF4FEA0B0865EA0B0809
:10D42000A4EC0A087CEA0B08D6F60B086CF30B0890
:10D430008DEA0B089EEA0B08B5EA0B0838B50546DD
:10D440000C46FFF7F1FE2A7902F0070302F0E00232
:10D45000602A29D1052B0CD8DFE803F0030B0F0B52
:10D460001B1B6A79012393400278DBB214B113438A
:10D47000037038BD22EA0303FAE76A790123934077
:10D4800002889BB214B113430380F2E722EA03033C
:10D49000FAE76B7901229A40036814B113430360E1
:10D4A000E7E723EA0203FAE7052BE2D8DFE803F017
:10D4B0000303050507070470DBE70480D9E7046070
:10D4C000D7E70149FFF794BACDEA0B080149FFF706
:10D4D0008FBA00BFDCEA0B0807B5009313460A4673
:10D4E0000249FFF785FA03B05DF804FBF3EA0B0885
:10D4F00020B10078B0FA80F04009704701207047F1
:10D500002DE9F74F81460846FFF7F2FF0E46054624
:10D5100070B1002401A92046013451F089FB014675
:10D520004846FFF7EDFF122CF4D103B0BDE8F08FB1
:10D530000846FDF7B7FBC4B2112C70D83C4D701CE7
:10D54000FBF776FE3B4E05EB44088346670098F8F0
:10D55000BCA2B8B9AAF102014B424B413D4495F837
:10D56000BC22B25C002B53D095F8BD32192040F29A
:10D57000EE2100FB031321462F4803B0BDE8F04F16
:10D58000FFF7FEB90178304660F095F880B1032CC2
:10D590002A49A0EB060394BF0022012202EB4202BB
:10D5A0000A4452FA83F393F878A9BAF1030F04D12D
:10D5B000484603B0BDE8F04F83E75846FBF738FE16
:10D5C000F0B1BAF1020FF3D1FDF76CFB40F6CA03DC
:10D5D00080B29842A8BF184640F2EE239842B8BFE6
:10D5E00018461923A0F2EE20B0FBF3F088F8BD0234
:10D5F000AAF1020253425341EA1982F8BCA2ADE7F4
:10D60000BAF1020FF4D1484603B0BDE8F04F5DE730
:10D6100021460B4803B0BDE8F04FFFF7B1B9112325
:10D620002A460849484603B0BDE8F04F54E700BF1A
:10D630004846002450810B080CEB0B08A4EC0A08A8
:10D640001CEB0B0829EB0B082DE9F04F0346A1B0AA
:10D650000846FFF74DFF054620B1184621B0BDE84A
:10D66000F04F33E7FF23DFF8C09207464FF0FF3853
:10D670008DF82830D9F8E0320B9093F83820ADF8C7
:10D6800030000D908DF838200F90ADF840001193C8
:10D690000991CDE90500934909A85FF0A5FF04466B
:10D6A00018BB01460AAC904F0B0190481A57002353
:10D6B00010F9016BB24240F0D2804E1C104651F07E
:10D6C000A1FA024631463846FFF75AF9022E4FF0CA
:10D6D0000101E9D19DF938A09DF92830534540F06A
:10D6E000C5808348FFF74CF94DE02378002BD2D05A
:10D6F000032FD4BF00260126062F00F2A980DFE801
:10D7000007F00447509104475000042F10D0794986
:10D710002046FDF725FA58B14FF480600CF0E0FE8A
:10D72000002800F0B48190F90400012306930AE078
:10D7300071492046FAF790FF70B9D9F8E03293F9B1
:10D740003800042F22D0119B119320AB03EB061657
:10D7500006F8580C01379EE7204651F049F9002899
:10D76000EFDA01230A2212A92046FDF711FA40B28E
:10D77000002803DB129B1B78002BE2D02246711C91
:10D780005E48FFF7FDF821B0BDE8F08F0023DBE72E
:10D790002046FDF787FA20AB03EB061646F8540C3B
:10D7A000D8E757492046FDF7DBF9B0F1000A5549A3
:10D7B000204618BF4FF0010AFDF7D2F908B14AF030
:10D7C000020A3301DFF864C1079320AB03EB0616AE
:10D7D000BCE80F0006F850AC12AE0DF1480A0FC6B7
:10D7E000BCE80F000FC6BCE80F000FC69CE80300A2
:10D7F00086E803000026B346DAF80010204660F001
:10D8000081F810B19AF804301E430BF1010B0AF1B4
:10D81000080ABBF1070FEFD1079B80336B4403F875
:10D820004F6C97E738492046FAF716FFA0B1374901
:10D830002046FAF711FF00288CD02046FDF732FA77
:10D840000328804686D901463148FFF799F89AE7C0
:10D85000224608212F4894E7012305937AE70133F4
:10D860000A2B7FF425AF01312B488AE70B9B1BB9AC
:10D87000AAF114025542554100235F1CE368002BB6
:10D8800061D194F900B058460CF0FCFDD4F8049036
:10D8900018B10668002E40F08A80B9F1000F237A93
:10D8A00014BF4E464FF46146666023B91B48FFF72C
:10D8B00067F803232372627A2AB13946184807921F
:10D8C000FFF75EF8079A02925846237ACDE9006383
:10D8D00000231A4619460CF01DFEE06040BB394695
:10D8E0001048B2E77FEE0B08B3EB0B088BF10A0888
:10D8F000D0EB0B084CEB0B0857EB0B085BEB0B0862
:10D9000076EB0B0858FD0B0879EB0B08F8E90B08D0
:10D910007FEB0B0897EB0B08BEEB0B08E9EB0B0852
:10D9200004EC0B081FEC0B084846002424F60A08F8
:10D9300058493346584A5948B9F1000F18BF0A46AA
:10D940003946FEF79DFF022F04F110044FF001034A
:10D9500093D1119E0D9F4DB15148FEF75DFF336885
:10D960001B6A1BB13A464F4930469847059B002B2E
:10D9700050D04D49474BBAF1140F18BF19464B48C8
:10D98000FEF7FEFFBAF1140F09D1059B002B43D01F
:10D990003368DB691BB10022454930469847069B36
:10D9A000002B43D100223146384651F039F8E66069
:10D9B000B9F1000F2CD04946304602F063F93D4AD8
:10D9C000B36839463C48FEF7DBFF94F80890B9F19C
:10D9D000000F0CD03279914509D04B463946374873
:10D9E000FEF7CEFF3368494630469B699847637A15
:10D9F00023B1727939463248FEF7C2FFF36A002B31
:10DA0000A1D039462F48FEF7BBFF0023F3629AE707
:10DA1000204AD5E71F49B2E7B8F1000FBFDB3368F2
:10DA2000DB69002BBBD042462749B6E7DFF89C9064
:10DA30000025DFF89CA04FF0030B05F0FBFA052052
:10DA4000F9F752F89AF89035AB42ABD919F8014F73
:10DA5000C4B1204605F07EFE804698B12046F5F719
:10DA6000B3FC0446EBB210B180F806B0C371204697
:10DA70000121F4F773FC98F806302046DB0703D544
:10DA8000F4F79EFA0135DDE7F4F794FAFAE74FF080
:10DA9000FF304AE658EC0B0831EB0B083BEC0B0867
:10DAA000F1EC0B0885FC04083FEB0B081AED0B08A2
:10DAB000499204083AEB0B0859EC0B087EEC0B0872
:10DAC000A1EC0B08D8EC0B08B1890408332F002413
:10DAD000481C00202DE9F04F914687B00C461A46AD
:10DAE000002180464D46FFF738FB00270646B9F176
:10DAF000000F63D02946062220465FF019FF002858
:10DB00003246404613BF012100214FF0010A4FF079
:10DB1000000AFFF722FB0646287817F0D5F983465E
:10DB2000F8B1687917F0D0F94FF461714FF0190C22
:10DB3000AB78EA789BF805E01CFB03131CFB021290
:10DB400095F801B0297900B14079CDE90410CDE90B
:10DB5000023251463B461A4A4046CDE900EBFEF7F9
:10DB600077FE207817F0B0F98346F8B1607917F0A6
:10DB7000ABF94FF461714FF0190CA378E2789BF880
:10DB800005E01CFB03131CFB021294F801B0217981
:10DB900000B14079CDE90410CDE9023251463B464F
:10DBA000074A4046CDE900EBFEF722FE0137063476
:10DBB0000635142F9BD107B0BDE8F08FCA46D0E7D9
:10DBC0003DED0B082DE9F041054686B008460F46AD
:10DBD000FFF78EFC064638B100235B4901201A4648
:10DBE00006B0BDE8F04175E70846FDF75BF813287D
:10DBF000044600F3A08006258DF81760534E454378
:10DC0000781CFBF715FB074660B1FDF74BF8C0B277
:10DC100017F074F930B17319027983F80C290123D4
:10DC20008DF817303846FBF703FB074668B1FDF760
:10DC300039F80D2809D8062303FB046383F80D097E
:10DC40009DF8173001338DF81730DFF8FC80A91CE0
:10DC50000DF1170238464144FDF728F8FBF7E8FAC2
:10DC6000074668B1FDF71EF8012809D89DF817305E
:10DC70000622013302FB04628DF8173082F8100986
:10DC80003846FBF7D5FA80B1FDF70CF8C0B217F0B3
:10DC900035F950B19DF817300622017902FB046274
:10DCA000013382F811198DF817309DF817200623DB
:10DCB000042A2FD103FB04630022A3F810290625B0
:10DCC0001EF0C8FF05FB046595F80C0917F0FCF879
:10DCD00095F80F1995F80E7919234FF46172804663
:10DCE00095F8110913FB012613FB072717F0ECF831
:10DCF0004379214698F80520039395F81039144884
:10DD00000097CDE9016395F80D39FEF739FE06B0AD
:10DD1000BDE8F081052A05D103FB0463002283F8E6
:10DD20001129CCE7062ACAD0002308EB050248F8DF
:10DD300005309380C3E7132332460649284606B0D0
:10DD4000BDE8F041FFF7C8BB5C3E0024503500241D
:10DD50003DED0B0856ED0B082DE9F04F904689B0CC
:10DD60001A460C46002181464546FFF7F6F93A4E21
:10DD700008F178030746DFF8E4B0079394F904004C
:10DD80000CF080FB00285CD0B8F1000F61D0294670
:10DD90000C2220465FF0CCFD00283A46484613BFCF
:10DDA000012100214FF0010A4FF0000AFFF7D5F9D9
:10DDB000074695F9040050F025FFEA7903465146DD
:10DDC00006EB82024846D2F8B82904922A7A06EB7A
:10DDD0008202D2F8B8290392AA7906EB8202D2F81D
:10DDE000B82902926A7906EB8202D2F8B829019228
:10DDF0002A6800925A46FEF72BFD94F9040050F071
:10DE000001FFE2790346514606EB82024846D2F80A
:10DE1000B8290492227A06EB8202D2F8B82903923A
:10DE2000A27906EB8202D2F8B8290292627906EB57
:10DE30008202D2F8B8290192226800925A46FEF76F
:10DE4000D7FC0C35079B0C34AB4297D109B0BDE829
:10DE5000F08FC246D1E700BFA4EC0A085CED0B08C6
:10DE60002DE9F04780468CB00846FFF741FB054698
:10DE700038B10023594901201A460CB0BDE8F047DB
:10DE80006AE7CDE909000B9007A8079154495FF0B4
:10DE9000ABFB064650F0ACFD431C04460CD12B46B0
:10DEA0000A2208A93046FCF773FE089B1B781BB9B1
:10DEB000C4B2132C0BD944B220460CF097FA054695
:10DEC00040B94046FFF7FDFA0CB0BDE8F0873334A7
:10DED00064B2F1E7424907A88DF828405FF084FB5F
:10DEE000B0B3002302260A221946FCF751FE09901E
:10DEF0000027DFF8EC90DFF8F0A0494607A85FF0B4
:10DF000073FBF8B1FCF7CEFE364A002352F8041B2F
:10DF100088421FD1DBB20AEB8302D2F8B8299042C3
:10DF200010D1022F20D0032F23D05A1E012FD2B29E
:10DF300015D00B2A03D88DF829300136F6B20137F7
:10DF4000042FDAD1052E1AD84046FFF7BFFABBE7F7
:10DF50000126CDE70133102BD8D10023DBE7052ABA
:10DF6000EDD88DF82A30E8E7092BE8D88DF82C3069
:10DF7000E3E79A1E0D2AE2D88DF82B30DDE709ABD6
:10DF800003CB286018686960A860204650F03AFE0C
:10DF9000154A9DF82B10034602EB8101D1F8B81900
:10DFA00004919DF82C1002EB8101D1F8B81903916E
:10DFB0009DF82A1002EB8101D1F8B81902919DF861
:10DFC000291002EB81020021D2F8B82908460192FB
:10DFD000099A0092054AFEF70BFC75E7143D0024F0
:10DFE0007FEE0B085CF60A08A4EC0A085CED0B084F
:10DFF0002DE9F04F90468BB000264FF0190A4546A8
:10E000004FF461790C461A4600210746FFF7A5F840
:10E010000990B8F1000F49D029460A2220465FF046
:10E0200087FC0028099A384613BF012100214FF0D0
:10E03000010B4FF0000BFFF790F82A890990334647
:10E0400006925946EA88384605922A790492EA7877
:10E050000392AA781AFB029202926A781AFB029241
:10E0600001922A780092124AFEF7F2FB2289334687
:10E070000136594606923846E2880A3505922279D9
:10E080000492E2780392A2781AFB029202926278DA
:10E090001AFB0292019214F80A2B0092044AFEF72E
:10E0A000A7FB1E2EB5D10BB0BDE8F08FC346DDE750
:10E0B00079ED0B082DE9F04380468BB008460F46FA
:10E0C000FFF716FA044638B100235E4901201A46CC
:10E0D0000BB0BDE8F0438BE70846FCF7E3FD1D28D5
:10E0E000054600F3A5800A268DF827404643781C94
:10E0F000FBF79EF810B101238DF82730FBF798F855
:10E10000514C074668B1FCF7CDFD0D2809D80A230C
:10E1100003FB054383F8E4029DF8273001338DF8B3
:10E120002730DFF82091711C0DF127023846494451
:10E13000FCF7BCFDFBF77CF8074668B1FCF7B2FDC5
:10E14000232809D89DF827300A22013302FB054213
:10E150008DF8273082F8E7023846FBF769F8074662
:10E1600068B1FCF79FFD0D2809D89DF827300A22D9
:10E17000013302FB05428DF8273082F8E8029DF852
:10E180002730062B0CD0002309EB0602404649F845
:10E190000630536013810BB0BDE8F043FFF796B92A
:10E1A0000A260023384606FB0546A6F8EA32A6F8FA
:10E1B000EC32FBF73DF8074618B1FCF773FDA6F803
:10E1C000EA023846FBF734F830B1FCF76BFD0A235E
:10E1D00003FB0543A3F8EC021C4B4FF0FF324FF456
:10E1E00061701A650A2303FB0542B2F8EC3206930C
:10E1F000B2F8EA32059392F8E832049392F8E732E3
:10E200000393192392F8E61213FB0101029192F88D
:10E21000E51213FB010300210193084692F8E43252
:10E220000B4A00932B46FEF7E3FA0BB0BDE8F083F0
:10E230001D232246074940460BB0BDE8F043FFF7D7
:10E240004BB900BF2C490024484600244C0400244C
:10E2500079ED0B0856ED0B082DE9F04F80469146FD
:10E260001E460C4615460027DFF81CA12DED088B35
:10E2700095B094ED008AB5EE408AF1EE10FA7BD0AD
:10E28000D4ED019A94ED029AD4ED038AB9F1000F0E
:10E2900049D0D5ED00BA95ED01BAB4EE6B8AD5ED53
:10E2A00002AA95ED03AAF1EE10FA6AD1F4EE4B9AA8
:10E2B000F1EE10FA65D1B4EE6A9AF1EE10FA60D17F
:10E2C000F4EE4A8AF1EE10FA0CBF01210021324629
:10E2D0008B46404681F00101FEF73FFFB0EE6B0A2E
:10E2E000064611A8FAF720FFB0EE4B0A07900EA8D9
:10E2F000FAF71AFFB0EE6A0A06900BA8FAF714FFB5
:10E30000B0EE4A0A059008A8FAF70EFF0599069A9A
:10E31000079B039040460291594601925246009352
:10E320003B46FEF795FAB0EE480A11A8FAF7FCFE54
:10E33000B0EE690A83460EA8FAF7F6FEB0EE490A77
:10E3400006900BA8FAF7F0FEB0EE680A059008A850
:10E35000FAF7EAFE069B059A0021039040460292D6
:10E36000524610341035CDE900B33B460137FEF775
:10E370003FFA082F7FF47DAF15B0BDEC088BBDE8E8
:10E38000F08F0021A3E700BF9CED0B082DE9F14FB2
:10E3900006460C46DFF894B12046FFF7A9F8074679
:10E3A00038B100235A4901201A4601B0BDE8F04FA8
:10E3B00052E7052257492046FCF7AEFB60B9544BA3
:10E3C00000221A601A611A621A631A641A651A66C0
:10E3D0001A6701B0BDE8F08F042259462046FCF7C9
:10E3E0009BFB05462046002D45D1FAF721FF074645
:10E3F0000028EED05CF056F9DFF834A15FFA80F81F
:10E400005AF8049BB9F1000F07D122464249304621
:10E4100001B0BDE8F04FFEF7EBBA42464946384638
:10E420000135FCF779FB84460028E9D1384A0346D8
:10E4300000211746013342F8101B082BFAD1374B45
:10E4400003EBC505D5F880E0BEF1000F05D14946C4
:10E450003348344CFEF794FA9EE795F87C50AC456F
:10E46000F5DA0EEB0C1307EB0C140CF1010C0FCBCF
:10E4700084E80F00F3E7FCF715FC072805463DD8B4
:10E480002046FAF7D5FE074658B3FAF783F9204B32
:10E49000012403EB051383ED000A3846FAF7C8FEA2
:10E4A000074638B1FAF776F9194B013403EB051337
:10E4B00083ED010A3846FAF7BBFE074638B1FAF792
:10E4C00069F9134B013403EB051383ED020A384657
:10E4D000FAF7AEFE38B9304601B0BDE8F04FFEF7AE
:10E4E000F5BF0446D9E7FAF755F9094B032C03EBBE
:10E4F000051383ED030A3FF454AFECE707233A46D4
:10E500000949304601B0BDE8F04FFEF7E5BF00BF56
:10E510008441002479EB0B08DBE90B08A4EC0A0822
:10E52000B5ED0B0858EC0B0856ED0B08B0ED0B08D9
:10E530009CF60A082DE9F74F92460C461A46002130
:10E5400081465646FEF709FE00258046DFF864B096
:10E55000BAF1000F2CD03146042220465FF0E8F9D2
:10E5600000284246484613BF012100210127002709
:10E57000FEF7F3FD738880465A46019339463AF810
:10E580002530484600932B46FEF762F963885A46C9
:10E59000394648460193043634F8043B00932B4631
:10E5A0000135FEF725F9042DD2D103B0BDE8F08F77
:10E5B0005746EBE7BFED0B082DE9F341054608464A
:10E5C000FEF796FF0C46074638B100233349012079
:10E5D0001A4602B0BDE8F041ACE731492046FAF7EF
:10E5E0003BF870B904222D4B4FF47A704FF4FA6166
:10E5F000013A1880598003F10403F9D102B0BDE853
:10E60000F0812046FCF74EFB0328064641D8204601
:10E61000FAF70EFE074698B1FCF744FB4FF00108ED
:10E6200004463846FAF704FE20B1FCF73BFBB8F18C
:10E63000000F09D1284602B0BDE8F041FEF746BF01
:10E6400040F2EE248046ECE7A4F2EE2240F2DC53E6
:10E650009A4203D8A0F2EE229A420AD940F6CA039F
:10E6600040F2EE220F49284602B0BDE8F041FEF725
:10E6700033BF0D4B00210D4A03EB8603A3F8104472
:10E68000A3F812043346CDE900400846FEF7B0F87F
:10E69000B4E703233A460649E5E700BF584A002499
:10E6A00079EB0B08D0ED0B0848460024BFED0B08B2
:10E6B00029EB0B082DE9F04F8FB089461746002152
:10E6C0001A4606460024FEF748FD0DF1240B0546C8
:10E6D000DFF86CA059F82480594602A8CDF80880CC
:10E6E00050F040FA4FB357F824302A463046984548
:10E6F000039313BF012100214FF001084FF00008E0
:10E70000FEF72BFD04A9054603A850F02BFA04A937
:10E7100023465246009130464146FEF799F823467B
:10E720000134524641463046CDF800B0FEF760F85D
:10E73000202CCFD10FB0BDE8F08FB846EFE700BF77
:10E74000DEED0B08F0B5074689B008460E46FEF729
:10E75000CFFE054638B10023194901201A4609B0F9
:10E76000BDE8F040A6E70846FCF79CFA1F280446DF
:10E770001DD83046FAF75CFD014620463CF0C4FB4C
:10E7800078B103AE0E48314600EB840050F0EAF950
:10E7900023460C4A294628460096FEF729F809B078
:10E7A000F0BD384609B0BDE8F040FEF78ABE1F2331
:10E7B0002A460549384609B0BDE8F040FEF78CBE50
:10E7C000684A0024DEED0B0856ED0B082DE9F04FEA
:10E7D000924685B00C461A46002181465546FEF702
:10E7E000BCFC00268046DFF86CB0BAF1000F2FD0D9
:10E7F0002946042220465FF09BF8002842464846FE
:10E8000013BF0121002101270027FEF7A6FCEB78AA
:10E8100080465A4602933946AB78484601932B8886
:10E8200000933346FEF714F8E3785A4639464846D3
:10E8300002930435A378019334F8043B00933346E4
:10E840000136FDF7D5FF102ECFD105B0BDE8F08F12
:10E850005746E9E7E8ED0B08F0B5074685B00846EE
:10E860000E46FEF745FE054638B100231C4901203F
:10E870001A4605B0BDE8F040A8E70846FCF712FAD2
:10E880000F28044623DC3046FAF7D2FC0146204626
:10E890003CF014FCA8B104F12002124B2946284692
:10E8A00003EB820393F82324029293F8222401922B
:10E8B000B3F820340C4A00932346FDF799FF05B0C6
:10E8C000F0BD384605B0BDE8F040FEF7FABD0F23B5
:10E8D0002A460649384605B0BDE8F040FEF7FCBDC3
:10E8E000E84A002448460024E8ED0B0856ED0B08E2
:10E8F0002DE9F04F85B014461A46054602910021D5
:10E90000FEF72BFC4FF00008064606234FF00009E7
:10E9100003FB08F7C037029B13F807B0002C7AD02E
:10E92000E35D324628469B45039313BF0121002136
:10E930004FF0010A4FF0000AFEF70FFC039B06465A
:10E94000374A51462846CDE900934346FDF780FFFC
:10E950004346334A514628460137CDE9009B09F129
:10E960000109FDF745FFB9F1060FD4D108F10108FF
:10E97000B8F1060FC9D1E427029BA7F1E40913F807
:10E9800007A0002C49D014F807B032462846DA45D3
:10E990000DBF4FF001084FF0000801210021FEF7E4
:10E9A000DCFB062306461E4A41462846CDE9009B6D
:10E9B000FDF74EFF01370623194A41462846CDE9A7
:10E9C000009AFDF715FFEF2FD6D1029B93F8EF7059
:10E9D000ACB194F8EF8032462846474513BF012179
:10E9E000002101240024FEF7B8FB00230C4A214635
:10E9F000009328460723CDF80480FDF729FF002364
:10EA0000074A21462846009307230197FDF7F0FEA9
:10EA100005B0BDE8F08FA2469AE7A046CAE700BF5E
:10EA2000FAED0B08F0B5054685B008460B46FEF733
:10EA30005FFD044638B100231B4901201A4605B08A
:10EA4000BDE8F04054E701AE184F6A461749184632
:10EA50005EF0F7FD88B1032C04D12846FEF736FDA1
:10EA600005B0F0BDFCF71EF96A4646F8040B3946BE
:10EA7000002001345EF0E5FDECE7032CEDD1039FAF
:10EA8000DDE901463A463146E0B23CF051FB18B9A7
:10EA90002846FEF716FDE3E73B463246214604488A
:10EAA000FDF76EFFDCE700BF684A00247FEE0B082D
:10EAB000FAED0B082DE9F04F0E46154689B01A46BF
:10EAC00000210446B046FEF748FB2F4681464FF032
:10EAD000000B002D7AD039460C2240465EF028FF0C
:10EAE00000284A46204613BF012100214FF0010AA9
:10EAF0004FF0000AFEF731FB97F90B2081465B4689
:10EB00000492514697F90A2020460392B7F908204B
:10EB10000292B7F906200192B7F904200092364A12
:10EB2000FDF796FE98F90B205B460BF1010B514661
:10EB30000492204698F90A200C3708F10C08039239
:10EB400038F9042C029238F9062C019238F9082C75
:10EB50000092294AFDF74CFEBBF1080FB9D14FF0E6
:10EB6000000BDFF898800C2303FB0BF985B300271B
:10EB700055F80900012356F8092003FA07FA424024
:10EB80003AEA020214BF1946002110EA0A0F07D020
:10EB90005B464246204600970791FDF759FE0799CC
:10EBA00056F809201AEA020F05D05B464246204675
:10EBB0000097FDF71DFE01370E2FD9D10BF1010B88
:10EBC000BBF1080FCFD109B0BDE8F08FAA46A9E785
:10EBD0002F46012356F8091003FA07F20A4206D01D
:10EBE0005B464246012120460097FDF701FE0137B2
:10EBF0000E2FEED1E2E700BF0EEE0B0826EE0B085B
:10EC0000F0B506468BB008460D46FEF771FC04468B
:10EC100020B300233D4901201A460BB0BDE8F04067
:10EC200048E72D2903D0A1F13003092B49D8052C41
:10EC300005DD30460BB0BDE8F040FEF747BC284686
:10EC4000FCF730F80AAB621C03EB440424F80C0C0C
:10EC500015F8013F303B092BFAD9144629780029D1
:10EC6000DFD1062CE5D1BDF81C20BDF91C30072AE8
:10EC7000DFD8BDF91E50A5F5FA7292B2B2F5FA6F5F
:10EC800018D8BDF92070A7F5FA7292B2B2F5FA6FF2
:10EC900010D8BDF922C065450CDC67450ADBBDF91B
:10ECA00024E00EF1640292B2C82A03D8BDF92640CE
:10ECB000112C11DD164930460BB0BDE8F040FDF7D0
:10ECC00097BE202902D101352246C6E730460BB057
:10ECD000BDE8F040FEF7F5BB0C200E4A64B200FB25
:10ECE00003220846A2F81455A2F81675A2F818C512
:10ECF00082F81AE582F81B45074A0095CDE903E43E
:10ED0000CDE9017CFDF774FD0BB0F0BD584B00243C
:10ED10003BEE0B08484600240EEE0B082DE9F04FA1
:10ED200089468DB0164600211A4607460024FEF794
:10ED300014FADFF8DCA00546C4EBC40309EB0302B8
:10ED400059F80300918840F3074892790890ADF88C
:10ED500024108DF82620B8F1000F53D0002E54D087
:10ED6000F218F0589188937907220A9008A8ADF814
:10ED70002C100AA98DF82E305EF0DAFD00282A4604
:10ED8000384613BF012100214FF0010B4FF0000B5B
:10ED9000FEF7E3F99DF82E30054652460693594694
:10EDA0009DF92D30384605939DF92C3004939DF83C
:10EDB0002B3003939DF92A3002939DF8293001935B
:10EDC0009DF8283000932346FDF742FD9DF826303C
:10EDD00052465946384606939DF9253005939DF9CC
:10EDE000243004939DF82330CDE902839DF821302F
:10EDF00001939DF82030009323460134FDF7F8FC81
:10EE0000102C99D10DB0BDE8F08FB346DEE700BFFE
:10EE100051EE0B082DE9F04F06468BB00D46DFF89A
:10EE2000A08228465BF03EFC034630B90246964974
:10EE300001200BB0BDE8F04F70E70522934928464A
:10EE4000FBF76AFE0446C8B9914D0146702205F5EC
:10EE5000AE605EF019FCC5F81045C5F81C45C5F854
:10EE60002845C5F83445C5F84045C5F84C45C5F8B2
:10EE70005845C5F864450BB0BDE8F08F0422414603
:10EE80002846FBF749FE044630BB2846FAF7D0F97E
:10EE900081460028EFD05BF005FCDFF828B28246FF
:10EEA0005BF8047B3FB92A467A4930460BB0BDE88F
:10EEB000F04FFDF79DBD524639464846FBF72CFE04
:10EEC00040B92046744D25F013FF39467348FDF7CD
:10EED00057FDA6E70134E3E7072271492846FBF70F
:10EEE0001BFE074600287AD1202128465EF0E3FB6E
:10EEF000044670BB6B4D6C48FDF7C2FC21460134E3
:10EF00002846FDF7BDFC0E2CF8D10025DFF8B8919E
:10EF1000664FFDF769FCDFF8B4810C260024DFF8AA
:10EF2000B0A129466E434846FDF7AAFC0123F259D9
:10EF30005F48A340013413420CBF41465146FDF7E0
:10EF40009FFC0E2CF2D10135FDF74EFC082DE4D1CB
:10EF500091E702AC574D01AA56495EF072FB0028BA
:10EF600048D0022F11D1029A072A07D8039C0D2CF2
:10EF700004D80378722B13D06E2B25D008230022DF
:10EF80004D493046FEF7A8FA75E7FBF78BFE01AA5C
:10EF900044F8040B2946002001375EF052FBDEE7FF
:10EFA0000C233B4903FB02110123D1F81015A340A8
:10EFB0000B4337490C2000FB02123949C2F81035C7
:10EFC0003046FFF727FF56E7314B0C20012100FBAD
:10EFD0000233A140D3F8103523EA0103E9E72846BC
:10EFE000002402AD334F01AA32495EF02AFB80B102
:10EFF000082C03D13046FEF769FA3CE7FBF752FED6
:10F0000001AA45F8040B3946002001345EF019FBD3
:10F01000EDE7082CEED1029B0F2B30D8DDF80CE089
:10F02000BEF1070F2BD8DDF810C0BCF10D0F26D8AC
:10F03000059F07F16402C82A21D8069DFF2D1ED81E
:10F04000079864281BD80899642918D8884216DACA
:10F05000099C032C13D8C3EBC3020D4B134483F854
:10F06000751583F870E50C4983F871C583F87275DE
:10F0700083F8735583F8740583F87645A0E70F4944
:10F080003046FDF7B5FCF6E6B84B002479EB0B08EB
:10F0900048460024DBE90B0858EC0B08B5ED0B08DB
:10F0A0006EEE0B0876EE0B086DF30B08584B002440
:10F0B0007BEE0B087FEE0B0881EE0B083BEE0B0896
:10F0C000B0ED0B089CF60A0886090C081CF10B0829
:10F0D00039EE0B082DE9F04F9246002689B04FF02B
:10F0E00019095546B3464FF461780C461A4600217B
:10F0F0000746FEF732F80790BAF1000F27D02946ED
:10F10000062220465EF014FC0028079A384613BFFA
:10F11000012100214FF0010B4FF0000BFEF71DF80D
:10F120006A790790334619FB0282594638460592A0
:10F130002A7919FB02820492EA780392AA78029251
:10F140006A7801922A780092104AFDF781FB627971
:10F1500033460136594619FB028238460635059278
:10F16000227919FB02820492E2780392A278029239
:10F170006278019214F8062B0092044AFDF738FBDE
:10F180000A2EB9D109B0BDE8F08F00BF87EE0B0899
:10F190002DE9F04F80468BB008460F46FEF7A8F9E0
:10F1A00038B10023534901201A460BB0BDE8F04F97
:10F1B00090E707900846504CFBF774FD0928054678
:10F1C00094F834BA94F835AA94F81E9B079A00F381
:10F1D000898006268DF827204643781CFAF728F800
:10F1E000074648B1FBF75EFD0D2805D8A31983F843
:10F1F000C00D01238DF827303846FAF719F8074675
:10F2000068B1FBF74FFD584509D8062303FB0543BA
:10F2100083F8C10D9DF8273001338DF8273038462B
:10F22000FAF706F8074668B1FBF73CFD504509D8E8
:10F23000062303FB054383F8C20D9DF827300133F5
:10F240008DF827303846F9F7F3FF074668B1FBF72A
:10F2500029FD814509D3062303FB054383F8C30D2C
:10F260009DF8273001338DF82730DFF88890311D65
:10F270000DF1270238464944FBF718FD9DF8273069
:10F28000062B0BD0002309EB0602404649F8063056
:10F2900093800BB0BDE8F04FFEF718B903FB0544AF
:10F2A0004FF46171192394F8C52D13FB02120592D6
:10F2B00094F8C42D13FB02130021104A049308464E
:10F2C00094F8C33D039394F8C23D029394F8C13D72
:10F2D000019394F8C03D00932B46FDF789FA0BB0DB
:10F2E000BDE8F08F0923064940460BB0BDE8F04F5A
:10F2F000FEF7F2B8104300245035002487EE0B08C7
:10F3000056ED0B082DE9F04F14468BB00F461A4608
:10F3100000210646FDF721FF0546002C00F0D780AE
:10F3200022783B789A42024630460DBF4FF00108E2
:10F330004FF0000801210021FDF70FFF237805465B
:10F340009B4A41463046FDF783FA3B784146984A4E
:10F350003046FDF74DFA002C00F0BB806278304655
:10F360007B789A422A460DBF4FF001084FF0000803
:10F3700001210021FDF7F1FE637805468D4A4146E3
:10F380003046FDF765FA7B7841468A4A3046FDF7FC
:10F390002FFA07F1C90307F1020A04F1CA0B05931A
:10F3A000A31C4FF000090693822307933B784B453B
:10F3B00000F39180002C00F0F58097F8EA30304699
:10F3C00094F8EA209A422A460DBF4FF001084FF008
:10F3D000000801210021FDF7C0FE94F8EA3005463F
:10F3E000754A41463046FDF733FA97F8EA30414610
:10F3F000714A3046FDF7FCF9002C00F0D58004F18D
:10F40000EA0307F1EA0204F1FA014FF0010833F8C8
:10F4100002CF32F8020F844518BF4FF0000899421E
:10F42000F5D188F001012A463046C9B2FDF795FEB4
:10F430000821054604F1EC00FBF7DEFA5F4A0346BB
:10F4400041463046FDF704FA97F8EA1007F1EC0060
:10F45000FBF7D2FA594A034641463046FDF7C8F950
:10F46000002C00F0A3804FF0FC094FF0010807EBDF
:10F47000090104EB0900F9F7EFF809F10409002884
:10F4800018BF4FF00008B9F58E7FF0D188F0010168
:10F490002A463046C9B2FDF760FE082104F1FC009F
:10F4A000F9F7D8FE464A034641463046FDF7D0F903
:10F4B00097F8EA1007F1FC00F9F7CCFE404A034642
:10F4C000414630460BB0BDE8F04FFDF791B9A0467C
:10F4D0003BE7A04657E7079BFB180993002C5FD03A
:10F4E000079B0998E31819460893F9F7B5F8059BA7
:10F4F0005A789BF800309A424FD1B0FA80F84FEA20
:10F500005818069AAAF102030AF10E01023A33F8DA
:10F5100002CF32F8020F844518BF4FF000088B422B
:10F52000F5D188F001012A463046C9B2FDF715FE33
:10F530006278069905469BF81800FBF72DFA0290B1
:10F540009BF8003041461F4A30460193089B0093C8
:10F5500009F10103FDF77CF9059B51467A7809F121
:10F560000109587E0AF1100AFBF716FA059A029073
:10F57000414612F8013F30460BF1010B0193099B04
:10F58000059200934B460F4AFDF732F9069B103364
:10F590000693079B0933079308E74FF00008B0E78D
:10F5A000A046D9E7A04620E7A0464DE7A0467FE762
:10F5B000A0EE0B08B2EE0B08E0EE0B08F8EE0B081D
:10F5C0000FEF0B08C7EE0B082DE9F04F8FB0044684
:10F5D0000846B24902AA5EF034F8054640B903462F
:10F5E0000246AF494120FFF78DFE0FB0BDE8F08F16
:10F5F000AC49F9F731F8064628BB02AAA7495EF0E4
:10F6000020F8FBF74FFB0828054606D908233246A9
:10F61000A5492046FDF760FFE7E7A44C94F8343A8B
:10F6200083420CDC84F8345ADFE731460136384631
:10F6300034F092FE94F8343AB342F6DCF2E7064630
:10F6400004F63427F6E79A492846F9F705F80646FE
:10F65000E0B902AA91495DF0F4FFFBF723FB08280B
:10F66000054603D9082332469249D2E78F4C94F8D5
:10F67000353A834202DC84F8355AB6E73046013623
:10F6800029464FF08DF9082EF8D1F4E78A4928462B
:10F69000F8F7E2FF064600BB02AA80495DF0D1FF01
:10F6A0000028A2D0FBF7FEFA0828054603D9082354
:10F6B00032468249ADE77D4C94F81E3B834209DD1A
:10F6C000014604F6342034F08DFE294604F6342039
:10F6D00034F096FE84F81E5B87E779492846F8F7F0
:10F6E000BBFF064618BB06AD704BDFF8B091014674
:10F6F000A8461022284693F81E7B5DF0C5FFBE4247
:10F7000002AA80F20A81494600205DF09AFF10B9F2
:10F710003A466C490AE1FBF7C5FA013628F8020BB4
:10F72000EDE7694C95E80F0084E80F005DE7674955
:10F730002846F8F791FF0646C0BB5C4B06ADDFF8E4
:10F740005C9193F81E7BBE4202AA80F2F380494688
:10F7500000205DF076FF014610B93A465C49E5E0CD
:10F76000AA464FF00008032228465EF08FF828468C
:10F770005AF098FF404502D801360435E3E79AF87D
:10F78000000008F10108FBF7C1F90AF8010BEEE7E8
:10F79000B60004464F4DB4423FF427AF06AB2819DC
:10F7A00003221919043434F0C1FDF4E74A4928460C
:10F7B000F8F752FF0746002840F0AC80DFF8EC80F5
:10F7C00002AA364998F8346A5DF03BFF00283FF4FE
:10F7D0000CAFFBF767FA451E01D4AE4203DC33469B
:10F7E00001223E4915E72D4902AA00205DF029FFBC
:10F7F000014600283FF4F9AE00260DF10C0908225D
:10F8000003A88DF814605EF041F803A85AF04AFF8F
:10F81000B0421BD802AA214900205DF012FF002847
:10F820003FF4E3AE0026037898F835AAB146019379
:10F83000564502AA19494FF0000080F285805DF01C
:10F8400000FF834650B9524625496FE099F8000001
:10F850000136FBF75BF909F8010BD6E7A6B99BF86F
:10F860000030303B092B0FD91E49F8F7F5FE38B1AF
:10F870001D495846F8F7F0FE70B15A461B4955E04D
:10F880004FF001094FF0FF365846FBF70BFA0028FE
:10F8900030DA5A46164949E0B146F3E77FEE0B08E5
:10F8A000843F002426EF0B082CEF0B085035002472
:10F8B00037EF0B0840EF0B084EEF0B085AEF0B0821
:10F8C0006CEF0B085BF00B087040002496EF0B0800
:10F8D0007BF00B0880400024C0EF0B08C5EF0B083D
:10F8E0009BF00B089CE70B08D1EF0B08D8EF0B0837
:10F8F0000DF00B080EAB03EB4603013623F8200C8A
:10F9000096E752461F4911E033F8022B013724F8DD
:10F91000022F30E02A461C4908E01C4900205DF017
:10F9200090FE00283FF4FDAE3A4619492046FDF707
:10F930005FF85AE6154900205DF083FE00283FF489
:10F9400027AF3A461349F1E75DF07BFE0028D8D196
:10F9500005EBC500104C082203A98230204404EBBB
:10F96000051434F0E3FC0198FBF7D0F808EB05032D
:10F9700083F8FE0A06ABBE42C6DC454485F8169BFA
:10F9800033E600BF22F00B0845F00B087FEE0B08B2
:10F9900078EF0B08A2EF0B08843F002470B50B4CE6
:10F9A000002504F56A7694F8913013B12046FCF7EF
:10F9B000A9FD20460135FCF783FE3046FCF7B2FE78
:10F9C000042D04F1EA04EED170BD00BFE438002438
:10F9D00038B50C46054615492046F8F73DFE30B9C6
:10F9E000FFF7DCFF1248BDE83840FCF715BF1149AE
:10F9F0002046F8F731FEA0B90F4B83F8250483F8B1
:10FA00002D0483F80F0583F8170583F8F90583F8AB
:10FA1000010683F8E30683F8EB0683F85D070748E1
:10FA2000E1E72846BDE83840FDF74BBDC0F00B08C4
:10FA3000C6F00B08E1F00B0850350024E9F00B0884
:10FA40002DE9F04F0F46904689B0002187EA08085B
:10FA50000646139A00250393FDF77FFBDFF8849099
:10FA60006FEA08030446069328460AF09BFA129BA5
:10FA7000184230D0069BDFF870B0034014BF4FF03F
:10FA8000010A4FF0000A049310EA070328460CBF4E
:10FA90004A465A46059307920AF096FA039B804617
:10FAA000079A514600903046FCF7D2FE049B22464E
:10FAB0003046B3FA83F14909FDF74FFB059A044636
:10FAC000039B002A0CBF5A464A4651463046CDF8A1
:10FAD0000080FCF78DFE0135172DC5D109B0BDE8BA
:10FAE000F08F00BF05F10B08AAED0B080379062B78
:10FAF0000ED1C9B2C2680D2996BF064B00215956D6
:10FB000001238B40134214BF08464FF0FF3070476B
:10FB1000481C7047E0720B0838B5074C074DAC42E3
:10FB200003D3074B01221A7038BDA288D4E9021012
:10FB30005DF04CFD1C34F2E7AC5A0C08BC640C08B8
:10FB400001490024204BB0F5FA6F1A680346A8BF9C
:10FB50004FF4FA63B3F57A7FB8BF4FF47A73D204E7
:10FB60001DD540F2DC5290421CD040F2DB5207EE31
:10FB7000903A9042F8EE677A96BFDFED146ADFEDB7
:10FB8000146A9FED147A77EEE67A92BF9FED120A1F
:10FB90009FED127A9FED120AA7EE870A7047B0F523
:10FBA0007A7F02D89FED0F0A704707EE903ADFED9B
:10FBB0000E6A9FED0E7AF8EE677A9FED0D0A77EEEA
:10FBC000E67AA7EE870A7047E83D002400007A44F1
:10FBD00000A0BB44D62000C000E08244D6200040F4
:10FBE000000083440000000000407A44661000409A
:10FBF00000004042704700BF704700BF00207047C0
:10FC000001207047704700BF704700BF704700BFBA
:10FC1000704700BF9FED010A704700BF0000000061
:10FC200000207047064B1B78834281BF00EB4000E9
:10FC3000044B03EBC003586998BF0020704700BF16
:10FC4000000600203C05002000EB4000024B03EBC7
:10FC5000C003587C704700BF3C050020024B187859
:10FC6000003818BF0120704700060020C3B25E2B89
:10FC70009ABF024B53F8200001487047EC250B084F
:10FC80008CB40B0803681B6903B11847704700BFA9
:10FC90000023084901E0152B09D003EB430201338F
:10FCA00011F802C00A448445F5D11046704700207F
:10FCB000704700BFA8240024F0B1B1FA81F35B09BA
:10FCC000D1B110B50D4C4FF0010E224602E00133C8
:10FCD0005B2B0FD092F804C01C328445F7D10EF193
:10FCE000010C71455FFA8CFEF1D1C3EBC30304EB49
:10FCF000830010BD002010BD00207047E4E00A081A
:10FD00002DE9F043070987B091461E46DDF838809B
:10FD1000403700F00F0439B3FFF7CEFFC379054633
:10FD2000164A49463046CDE900433B46C047C0B17C
:10FD30002868F2F76FF8AA796B7912F0020F104970
:10FD40004FEA93030F4A18BF0A46E979013300943A
:10FD5000CDE90321CDE901030B4A3B4600213046A2
:10FD6000C04707B0BDE8F0833B46084A49463046E5
:10FD7000C4460E9407B0BDE8F04360473AF10B0863
:10FD8000CBEA0B0858EC0B084CF10B086EF10B0892
:10FD90002DE9F04FDFF878B00F4601F10908012492
:10FDA000BBF8003004339DB217F8011BAC464FF08E
:10FDB000000E04FA0EF2ACF104030A409BB21BD110
:10FDC00003F1010A00EB83091FFA8AF3C9F8142032
:10FDD0009C45F5D10EF1010E0CF1040CBEF1080F9B
:10FDE0001FFA8CFCE5D120354745ADB2DCD10023AC
:10FDF000ABF80030BDE8F08F868903F1010900EB14
:10FE000083021FFA89F356616345F6D1E2E700BF2A
:10FE1000CC7900242DE9F047DFF87CA0884601F179
:10FE200006090024BAF8023001260B331FFA83FEBC
:10FE300018F801CB71460025A1F10B039BB23DB12F
:10FE4000092D20D06A1E06FA02F212EA0C0F1AD00F
:10FE5000878900EB830201339BB257619942F8D145
:10FE60000B1D01350C3100EB83030A2D89B25C6058
:10FE7000E2D10EF1780EC8451FFA8EFED8D1AAF84D
:10FE80000240BDE8F0871A1D01339BB200EB8202ED
:10FE90008B425460F7D1E3E7CC7900242DE9F84395
:10FEA0000E780446057B00F11003F64300F138029A
:10FEB000F6B243F8045F9342FBD12822002104F1FB
:10FEC0003C0005275DF0E0FB4FF000084FF0140EFA
:10FED00046FA07F2734602F00102002A42440CBFC0
:10FEE0004FF00A094FF0190917F0010F5FFA82F875
:10FEF0000EEB090C14BF284600201FFA8CFC591C7D
:10FF000004EB83028BB250616345F8D1013FF144A9
:10FF10007B1C1FFA89FEDBD118F0010F734614BF5A
:10FF200019200A200EEB0006B6B2591C04EB83021E
:10FF30008BB25561B342F8D1421E0EF101030EF1AE
:10FF40000200074992B2134402449BB292B20433B6
:10FF50008A80002104EB830359602261BDE8F883A5
:10FF6000CC79002470B5094CA36873B1054600260E
:10FF700006E099681A681E73A1609047A36823B1D0
:10FF80005A681846AA1A002AF3DA70BDCC79002400
:10FF9000064B10B5044618683AF0B4FD28B920465F
:10FFA0000349BDE81040FCF723BD10BD28490024DB
:10FFB00080F10B0870B50024144E96F82330651CB0
:10FFC0002341DB071CD5E4B229461148FCF7D8FCD5
:10FFD000752120462CF0E2F901460E48FCF7D0FCD2
:10FFE0001A2120462CF0DAF901460B48FCF7C8FC30
:10FFF0001B2120462CF0D2F901460848FCF7C0FC32
:020000040805ED
:10000000022D4FF00104D8D170BD00BF8C3C0024FC
:1000100096F10B08A2F10B08B5F10B08C8F10B081B
:1000200070B5054608461646FAF73CFE0D4B041E11
:100030001A780EDB944205DA21460B48FCF7A0FC47
:10004000204670BD2EB1FF2C03D10848FCF798FC68
:10005000F6E7013A064928464FF0FF34FCF7C8FCA2
:10006000EEE700BFD8210020DBF10B08ECF10B0814
:10007000FFF10B0810B5114B86B0114904460493EB
:10008000104B11480393114B114A0293114B0193EA
:10009000114B0093114BFCF7F3FBFCF7A5FB104948
:1000A0001048FCF76DFC3CB10F4A1049104806B0EF
:1000B000BDE81040FCF764BC06B010BD65F20B084B
:1000C0002FF20B086AF20B083AF20B0874F20B08D5
:1000D00025F20B087DF20B0889F20B08BF3C0024C7
:1000E00093F20B089BF20B08B7E80B0801E90B0829
:1000F000ACF20B080120BDE738B50B4D0C4605EB03
:10010000C00595F97C01FFF7B1FD01460748FCF7F2
:10011000B7FB95F8823133B1611C0548C9B2BDE81F
:100120003840FCF7ADBB38BDEC250B086CF30B0871
:1001300085090C082DE9F743804608460C46FDF773
:10014000D7F9054628B14046FDF7C0F903B0BDE830
:10015000F083204601AA2C492F465DF072FA2E4604
:100160000446DFF8A4907CB9022DECD1A7F57A7390
:10017000B3F57A7F21D94FF4FA634FF47A722349A9
:100180004046FDF7A9F9E1E74DB1012D10D001AAD4
:100190004946002001355DF054FA0446E3E70122A8
:1001A00021464046FFF73CFF431C0646EFD1CDE712
:1001B0002046FAF777FD0746E9E7154BB8B21B680A
:1001C0005B689847FCEEC07AFF2E17EE902A0BD1A1
:1001D000104BB6EEC00A19780F4BA14210DC114645
:1001E0000E48FCF7CDFBB1E70D4B31460D48B6EE9E
:1001F000C00A03EB860383ED030AFCF7C1FBA5E706
:100200000134A3EC010AE8E77FEE0B08F0FE0B08CF
:1002100090230020D8210020D8790024E6F20B0892
:10022000CC790024D9F20B08F8B5074608460C46ED
:10023000FDF75EF9C8B11F4B1E68013630463446E3
:1002400009F0C2FE0546F0B90134182CA8BF0024FD
:10025000204609F0B9FE0546A8B9B442F4D13846A3
:100260001549BDE8F840FCF7C3BB2046FAF71AFD74
:10027000044609F0A9FE054628B921460F48BDE805
:10028000F840FCF77DBB0B4B1C600AF0FBF92A46DB
:100290000B482146FCF774FB172C9BBF094B0C2223
:1002A000002002FB043398BF93F81403BDE8F84024
:1002B0000AF024BA9C050024F5F20B0809F30B0898
:1002C0001FF30B08EC250B0870B505460C46114EC4
:1002D0002046FDF70DF960B10F4B104893F900105F
:1002E0004B1C0ABF0E4BC9B21978BDE87040FCF731
:1002F00047BB2046FAF7D6FC032804D8C0B23446E0
:10030000FBF73AFFE4E7284603220649BDE87040C0
:10031000FCF76EBB58EC0B086405002438F30B089F
:10032000B83C002448F30B0870B505460C46114E46
:100330002046FDF7DDF860B10F4B104893F900102F
:100340004B1C0ABF0E4BC9B25978BDE87040FCF790
:1003500017BB2046FAF7A6FC032804D8C0B23446DF
:1003600017F0A4FBE4E7284603220649BDE87040E5
:10037000FCF73EBB58EC0B086505002434F30B0872
:10038000B83C002443F30B0802460846531C05D131
:10039000044B1A681B790A600B7170470249FAF71F
:1003A000E5BA00BF16F90B0886090C0810B5013133
:1003B0001446FFF781FC28B9064B1A681B792260A6
:1003C000237110BDC27920460349BDE81040FAF7F9
:1003D000CDBA00BF16F90B0847F10B080329F0B599
:1003E000054685B00C46164614D80B4F3970FCF7FD
:1003F000FBF90A492846FFF767FF2246084901A88A
:10040000FAF7B4FA01AB324608212846FCF722FF7E
:10041000FF233B7005B0F0BD6405002458EC0B08C9
:1004200038F30B080329F0B5054685B00C4616468F
:1004300014D80B4F3970FCF7D7F90A492846FFF753
:1004400073FF224608496846FAF790FA6B4632462F
:1004500010212846FCF7FEFEFF233B7005B0F0BDDF
:100460006505002458EC0B0834F30B082DE9F84F10
:10047000002607460C461D4DB046DFF87890DFF8A1
:1004800078A02046FDF734F8D5F800B048B92146E9
:100490005846FAF765FB20B921466868FAF760FB11
:1004A00080B15846FCF798F9696811B15046FCF7DD
:1004B000E7F9A96811B14846FCF7E2F94FF00108E5
:1004C000FCF792F901361035362EDAD12046FDF7C9
:1004D0000FF848B9B8F1000F06D122463846044952
:1004E000BDE8F84FFCF784BABDE8F88F202A0B0866
:1004F0006FF30B0869F30B0863F30B08434B2DE90B
:10050000F74F1A780546009141495B780A70414AD5
:100510001370414B1B780BB9FFF7FEFA3F4C0026D6
:1005200047F0E0FCB046A3460D23009973435BF807
:1005300003904846FAF714FB002840D0B8F1000FAA
:1005400001DDFCF751F949463548FCF799F90022DD
:1005500021462846FCF7F0FEFCF746F9237903F024
:100560001803082B44D0102B47D02046FCF7F2FE8E
:100570000D2303FB06B3B3F8090047F079FC82466C
:10058000D8B12046FCF718FE0746DAE902210244FA
:1005900001442046FCF79AFD78B94946019021486C
:1005A000FCF76EF9DAF80810019A28461346CA19C2
:1005B0002146FCF7A5FCFCF717F908F10108013604
:1005C00040F293230D349E42AED10020FCF7D2FDC1
:1005D000FF230F4A13700F4A1370B8F1000F11D1A7
:1005E000009A2846104903B0BDE8F04FFCF700BA66
:1005F0000E492846FFF768FEB7E70C492846FFF783
:1006000093FEB2E703B0BDE8F08F00BFB83C002412
:1006100064050024650500240149002474040B08C6
:1006200049EA0B0883F30B08DBE90B0858EC0B08CD
:100630002DE9F04F3B4C89B00A4600210546FCF7F6
:100640008CFD059094F90000FFF710FB814660884F
:1006500047F00EFC344BD0F808B01F7817B15F4656
:10066000D0F80CB0A3790026012B38BF01230693E4
:100670002279637906FB02331BF80380002F3AD0FE
:10068000FB5C4345059A2846079313BF01210021CF
:100690004FF0010A4FF0000AFCF75FFD079B01369F
:1006A000059053B303F00F021B095146284640330F
:1006B00002921E4ACDE900634B46FCF7C9F8B8F137
:1006C000000F24D008F00F034FEA1818174A5146BC
:1006D000029308F140032846CDE900634B46FCF73E
:1006E00087F8069BB342C3DC0834114BA342A9D15F
:1006F00009B0BDE8F08F3B46C3E7002FDFD04B4683
:100700000C4A514628460096FCF7A2F8D7E76B063C
:10071000E7D44B46074A514628460096FCF768F84E
:10072000DFE700BF68270B080149002493F30B089B
:1007300000290B08A9F30B082DE9F04F0C460746DA
:100740008BB040F2162047F093FB2246054600216D
:100750003846FCF702FD404B064615221B78002167
:1007600004A8002BD5E9024504BF25461C465CF0D1
:100770008BFF05F13F03039395F80090B9F1000F4B
:1007800030D095F801A0002C63D0224600231178C8
:10079000494557D1283392F8018001226B4403F870
:1007A000182CD0453246384613BF012100214FF0A6
:1007B000010B4FF0000BFCF7D0FC064654B1B8F12A
:1007C000000F07D0254B5A464146484600933B460A
:1007D000FFF796FA224B5A465146484600933B464D
:1007E000FFF78EFA0335039B9D42C5D13CB3651CD0
:1007F0000DF110084034DFF86490DFF864A018F8B9
:10080000013BCBB915F8013CB3B116B13046FCF74A
:1008100009F829783B4615F8010C0022CDF8009024
:100820000026FFF76DFA002215F8010C3B46114631
:10083000CDF800A0FFF764FA0335A542DFD10BB075
:10084000BDE8F08F01330332152BA0D14FF0000823
:10085000A7E7A046A5E700BF0149002451C8040846
:10086000F1C7040873B50E4610490546F7F7F4FEC4
:1008700018B93070012002B070BD2C78602C8CBF8C
:10088000613C413C082C0FD8013501230A2201A903
:100890002846FAF77DF9019BAB4205D00F2803D813
:1008A000013440EA0410E4E70020E4E716F90B08FD
:1008B000234870B5FBF790FF224B93F82C30002BA8
:1008C00038D0214B93ED010A5BF048FE01461F48EA
:1008D000FCF756F81E4C1F48FBF77EFF1E4B94F8A2
:1008E00021001E4A00280CBF10461846FBF794FF53
:1008F00094F8213013B31A4C1A48B4F89210FBF74D
:10090000BFFF194E94F89000184D00280CBF3046D8
:100910002846FBF781FFB4F894101548FBF7B0FFA9
:1009200094F8910000280CBF30462846BDE870407E
:10093000FBF772BF0F48FBF76FFFCBE770BD00BF3F
:10094000CDF30B08CC7900249C050024E7F30B08B9
:10095000E03C0024F6F30B08CAEA0B08960A0C08E0
:100960003035002007F40B08C6F30B08BDF30B0865
:100970002EF40B08ECF30B086B4B1B782DE9F04FB2
:1009800087B0002B00F0CA80684D4FF0000868481F
:10099000A968FBF7F5FF69686648FBF7F1FF664B4E
:1009A0006648D3E90031C91A654B1A68B1FBF2F207
:1009B000FBF7E6FFFBF718FF6248FBF72DFF6248E5
:1009C000FBF72AFF614B5FFA88F41B78A34221D81A
:1009D0005F4D00245F4EFBF707FF013455F8041FFD
:1009E0003046FBF74DFF162CF7D15B4D0124594ED5
:1009F000FBF7FAFE2B466968013430461B68043564
:100A0000C91AFBF73DFF162CF4D107B0BDE8F04F33
:100A1000FBF7EABE514B14264FF03C0B671C03EB6F
:100A2000840306FB045693ED280A5BF097FD96F8C5
:100A30001EA081B2B6F80E901AF0010F80B20CBF62
:100A40002D2252221AF0020F049045480CBF2D238C
:100A500054231AF0040FB1FBFBF10CBF4FF02D0C27
:100A60004FF0560C1AF0080F05914FF064010CBFBF
:100A70004FF02D0E4FF0430E1AF0800F01FB09F1DD
:100A80000CBF4FF02D0A4FF0530ACDE900CECDE94F
:100A900002A13946FBF7F4FEB37FDB073AD55C23AE
:100AA000304A6343D118D05891ED010A70B1B8EEC5
:100AB000400ADFED2D7A20EE270A07EE900AF8EEC5
:100AC000677A80EE270A5BF049FD00B2642290FB52
:100AD000F2F102FB11022548FBF7D2FE1421244853
:100AE00008F1010801FB075701FB0454F988628AE9
:100AF0000491218B02F0030392080391E18A029191
:100B0000A18B0191A18A009119214B43218AFBF706
:100B100037FF57E71748FBF75FFEDFE7164807B0D8
:100B2000BDE8F04FFBF778BE04000020101B00204A
:100B30004EF40B085EF40B083C1C002075F40B0807
:100B4000BC1D0024A2F40B08FEF40B08D8210020E1
:100B5000B81B0020AEF50B08BC1B00203035002070
:100B60005AF50B083018002000401C4677F50B089A
:100B70008CF50B0883F50B08B2F50B0808B5294B6B
:100B80001B68DB041ED5B5EE400AF1EE10FA26D044
:100B9000DFED257AB4EEE70AF1EE10FA1FD49FEDEF
:100BA000237AB4EEC70AF1EE10FA2AD870EE677A0B
:100BB0009FED1F7A9FED1F0AA7EE870A5BF0CEFC20
:100BC00080B208BDDFED187AB4EEE70AF1EE10FA54
:100BD0000BDA9FED190A5BF0C1FC80B208BD9FEDF6
:100BE000170A5BF0BBFC80B208BD70EE677A9FED20
:100BF000147A9FED140AA7EE870A5BF0AFFC80B26F
:100C000008BDDFED117ADFED116A70EE677A9FEDB6
:100C1000107AA7EEA67AB0EE470A5BF09FFC80B28E
:100C200008BD00BFE83D00240000404200E08244CF
:100C300066BEFFBE0060BB4400007A440080BB4437
:100C400038DFFF3E00407A440000834466BEFF3E2A
:100C500000A0BB44B94B42F201011A68B1EB124F3C
:100C60004FEA12432DE9F04F804691B000F0EF813A
:100C700042F20302934200F0EC8141F20302981A1F
:100C800043424341AE4A0024AE4E116806EBC30313
:100C9000AD4AAE4DAE48AF4FDFF88493BA46DFF8A9
:100CA00084B3B1FBF2F2D3F89817FBF7E9FDEA8DB4
:100CB0004FF47A730A20B2FBF3F103FB1122B5F96A
:100CC000303092B2B2FBF0F2A348FBF759FEA34AD0
:100CD000A349A448FBF7D4FDFBF786FDA24BA34A2A
:100CE000997BA34B06EB8101A248D31AA24AD1F803
:100CF000B4171288FBF744FEFBF776FD9F48FBF71D
:100D00006BFD95F832109E48FBF7BAFD9D48FBF746
:100D100063FD9D4B95F833101A889C4892B2FBF7FF
:100D2000AFFDFBF761FD9A499A48FBF7A9FD234601
:100D300099F81F202241D1072CD513B19648FBF713
:100D40004BFD611C9548FBF79BFD954B9548E35C7B
:100D50005BF82310FBF794FD9AF86A352341DA0714
:100D600002D59148FBF78CFD97F81831032B09D079
:100D70008E48FBF785FD97F81831012B02D18C487E
:100D8000FBF77EFDFB6C5B7B012B02D98948FBF7EF
:100D900077FD012307F5CE77002C00F05C81002B56
:100DA00040F05B818448FBF737FD844FD5F83890DD
:100DB000DFF874A207F1180B0123A34013EA090F0F
:100DC00015D01AF8042057F824305BF8241053F893
:100DD00022207B48FBF754FD012C06D1794B93F878
:100DE000DD1011B17848FBF74BFDFBF7FDFC01343A
:100DF000062CE1D17548FBF7EFFC754B1B681B0611
:100E000040F15B8195F85830724F032B8CBF7248CC
:100E10007248FBF7E1FC3B78022B40F021817048DF
:100E2000FBF7DAFC95F85830042B00F23E816D4850
:100E3000FBF7D2FC95F86830002B00F03C8106EB04
:100E4000C303D3F8F0176848FBF71AFDFBF7CCFC97
:100E5000664B67481C68674B1A78674B53F822103B
:100E6000FBF70EFD24B1227A617A6448FBF708FD96
:100E7000FBF7BAFC62494046FBF70FFDFBF7B4FCF9
:100E8000604B614819684FF47A73B1FBF3F1FBF7DB
:100E9000F7FC05A8FAF70AF838B105A908A859F02F
:100EA0005FF808A95948FBF7EBFCFBF79DFCD5F868
:100EB000F470002F00F0058107EE907ADFED546AA0
:100EC000B8EEE77AC6EE877AFDEEE77A17EE903A4B
:100ED00095F82C0030B14F4A039392ED010A5BF074
:100EE0003DFB039B6C6F5CB107EE904ADFED486AF7
:100EF000F8EEE77A86EEA77AFDEEC77A17EE904A0B
:100F0000304AB2F82C113A466429CDE90004A8BF52
:100F100064214148FBF734FDB5F86C2964233F4850
:100F2000B2FBF3F103FB112295F87D3906EB830642
:100F300092B2D6F824381B4E009377E00010005C84
:100F40000C030024EC250B0840420F00CC79002450
:100F5000D6F50B08481C0020E8F50B08F8FF012027
:100F6000000800000AF60B08B83C00240000040842
:100F7000000002081CF60B08A837002433F60B0803
:100F800045F60B0822EA0B08A42400244DF60B08B2
:100F900061F60B0866F60B08D6F60B086BF60B0825
:100FA000007A0024F5F60B08C5F50B0870F60B085F
:100FB00078F60B087DF60B0885F60B08A82D0B08B4
:100FC0008F000C08303500208AF60B088EF60B08CF
:100FD000E83D0024983D002494F60B08A0F60B0889
:100FE000B0F60B0806050C08E9F60B0800460024CD
:100FF00005F70B08FF45002444F70A080EF70B0815
:1010000058EC0B08B41D002418F70B0832F70B0836
:10101000002474499C05002445F70B088BF70B0846
:101020008C3C002410F80A08A405002495F87C39AB
:101030000125FBF7A5FC2B48FBF7CEFB2A4B1C68D0
:10104000002C40D1FBF7D0FB11B0BDE8F08F02239C
:1010500018E6032316E601246AE6FBF7C5FBA4E6BF
:10106000022009F03DFA044608B92048D8E690F974
:1010700004004DF0C7FDDFF898A0814639F0DEFD91
:101080005AF8202049461A48FBF7FAFBFB78012B57
:1010900004D11848FBF7A0FB1748C1E6A37917480D
:1010A0005AF82310FBF7ECFBF6E7BB780BB91448B2
:1010B000BEE61448BCE61449C5E61448FBF78CFBB1
:1010C000C4E63B4604E794FAA4F0B0FA80F005FACF
:1010D00000F024EA000408F04BFF01463046FBF71D
:1010E000CFFBADE7B0F70B08F8400024B6F60B08CD
:1010F000C0F60B08D0F60B08D5F60B0875ED0B08FB
:10110000D9F60B08CAE70B08CEF50B08F9F60B0861
:101110005CF60A082DE9F04FDFF8748199B098F871
:101120000330002B00F0978050480025504EDFF828
:1011300064B1FBF771FB2F46DFF85C91DFF85CA12F
:101140000BA9E8B216F018FA9DF83430002B53D0F2
:10115000139C54B107EE904A9FED460AF8EE677A69
:1011600080EE270A5BF0FAF904460B9A29465846A6
:10117000FBF786FB109A002A6FD002FB04F04FF4B5
:101180007A73B0FBF3F30993DDF848C0BCF1000FAC
:1011900065D00CFB04F142F21073B1FBF3F1082DA2
:1011A00098F8033018BF7F18002B5AD017984FF4C7
:1011B0007A7E0A2307901598069016980590119844
:1011C000B0FBFEFECDF810E00998B1FBF3FE03FB87
:1011D0001E11CDE902E10999B1FBF3F103FB110006
:1011E000BCFBF3F3CDE9001021465046FBF7C8FBEA
:1011F0000023B362C6E90D3301354036242D9FD15B
:1012000098F8033023B31C4C4FF47A731B48D4F87E
:101210008019D4F88429B1FBF3F3D208D4F88819E3
:10122000FBF7AEFB0A22164897FBF2F102FB1172A4
:10123000FBF7A6FB134B1B78432B06D1D4F88C2964
:10124000D4F890191048FBF79BFB0023C4F88839A9
:1012500019B0BDE8F08F0D4867E7099294E7614641
:101260009DE721464846FBF78BFBC1E7C6F70B0815
:10127000387A00248096184BCC7900246DF80B083E
:101280008DF80B08ED240024B1F80B0824F80B08A6
:10129000B83C00242EF80B0873F50B083DF80B083A
:1012A0002DE9FF47914604468A461E46FEF71EFC7E
:1012B000421CBDF830700546DDF834801FD0B9F10E
:1012C000FF3F1FD0154A3146CDE900093846236853
:1012D000C0474A465FFA8AF12079F0F72BFA0246B6
:1012E00000B10288D3B2314638460393C2F30323D8
:1012F000120B0293CDE90052094A2368C04704B09B
:10130000BDE8F0877B06FAD40C9031462368384656
:10131000044AC44604B0BDE8F0476047DBF80B0858
:10132000E8F80B080CF90B082DE9F043154685B0D9
:10133000894619466A1CBDF830600D9F28D04FEAD7
:10134000101800F00F04194A304608F14008CDE9A2
:1013500000454346B847C0B1EBB2D9F8000099F850
:1013600005100F2B11D82A46F0F72AFA68B1038826
:101370000021027830460392C3F303221B0B029232
:101380000B4ACDE900434346B84705B0BDE8F083BA
:101390007306FAD4030900F00F00064ABC460C900D
:1013A0004033304605B0BDE8F04360471BF90B08F9
:1013B0002DF90B0856F90B082DE9F04F714C8DB043
:1013C000DFF8CC910A4604F1B00A00218346FBF70E
:1013D000C4FE03900025A37A99F80060AB4200F3A5
:1013E000908010345445F5D140F216200DF1180AC2
:1013F00046F03EFD0027002E4FF015024FF0000191
:10140000D0E90245504604BF254634465CF03CF91D
:101410002E78002E3CD069783046FEF74DFC95F9C9
:101420000290049009F1010253425341002C00F054
:10143000A5800022A05CB04240F09C80224492F93A
:101440000280C14540F0948052788A4208BF01234F
:10145000012203F001030AF8072083F00101039A37
:1014600058460593FBF779FE059B039044B1464A25
:1014700030460499CDE900B24246FFF755FF059B7F
:10148000424A30460499CDE900B24A46FFF74CFF84
:1014900001370335152FBBD184B3564604F13F07FE
:1014A000DFF8E480DFF8E49016F801ABBAF1000F42
:1014B00021D12078F8B194F9023001331BD0617842
:1014C000FEF7FAFB0546039A01215846FBF745FE55
:1014D00094F902205346294603902078CDE900B8BC
:1014E000FFF722FF207853464FF0FF322946CDE91F
:1014F00000B9FFF719FF0334BC42D5D10DB0BDE8E8
:10150000F08FE08846F0B4FC002E627AD0E9023118
:10151000207A04BF1946334605FB00228F5623B3B9
:101520009E56B742039A5846049313BF01210021E7
:101530004FF001084FF00008FBF70FFE049B0390EB
:1015400043B1114B324629462046CDE900B343460C
:10155000FFF7A6FE0D4B29463A4620460135CDE958
:1015600000B34346FFF79CFE35E74FF0FF36D8E760
:1015700000236DE703323F2A7FF45CAF4FF0FF3862
:101580006BE700BFAC05002451C80408F1C704088C
:1015900001490024A84B1B68002B37D05B69F0B5CC
:1015A00085B0984780B3A54CD4F8D030002B01DD2E
:1015B000F8F782FD6378022B33D0032B24D194F803
:1015C000EC3113B19E48F9F7DDFE94F8D83013B131
:1015D0009C48F9F7D7FE94F81C3113B19A48F9F7F3
:1015E000D1FE94F860317BB1984805B0BDE8F04079
:1015F000F9F7C8BE96480321302305220090A17058
:101600009448954958F08AFD05B0F0BD7047A2682E
:1016100001209249F8F72AF8012840F06D8106234D
:10162000A370A378072BEFD801A252F823F000BFD4
:10163000F916050893160508F51505088716050817
:101640006D1605080F1605085716050851160508EA
:1016500003236370D8E700217E48F8F7CFF801280C
:1016600040F04A81A3780133A370DAE72378032B93
:1016700014BF4FF480758025207D002800F0C280C3
:1016800001284ED0FEE794F8A431002BBCD071485D
:10169000ABE70023092203A9D4F83002F7F72CFEA8
:1016A0000128B1D10022039B2270B3F80B20B2F5C0
:1016B000007F1BD11A7C022A18D193F8FE21552AEB
:1016C00014D193F8FF21AA2A10D1D889D4F8302256
:1016D0008618C4F834625F7B7A1EC4F844727F2A8D
:1016E00004D87A4237EA020200F00E810322012375
:1016F00084F8E821637087E70023092203A91846CC
:10170000F7F7FAFD01287FF47FAF039B93F8FE21E2
:10171000552A00F0A7800222012384F8E821637093
:1017200072E7D4F844224FF0FF3360680021520280
:10173000B3FBF2F31A18D4F83C3203F1020341EB85
:1017400001009342814146494FF0020038BF1A46DA
:10175000F7F700FF03288FD801A353F820F000BF4C
:1017600009160508711705080916050871170508F7
:10177000D4E9011326695A1AB24288BFC4E9031298
:1017800003280BD00133B3FBF5F205FB12320AB18B
:101790002B449B1A0022636022756DE723690622A1
:1017A000652BA2707FF63DAF2278653B032A15BFFB
:1017B0006FF0FF016FF07F014FF4807280220B40C9
:1017C00001339A422361BFF42CAFE268D4F83C1293
:1017D00098180231884207D394F8E81111B9012111
:1017E00084F8E81101216170D4F84412C4F8C821CA
:1017F00001FB03F3C4E901205B020522C4E96B335A
:10180000A2700EE7D4F83C2214490232F7F7A2FE88
:1018100003283FF631AF01A353F820F0091605085D
:101820002D180508091605089D170508012263688B
:1018300013442275A3601FE7542000245035002470
:101840003C370024283600246C360024B0360024AF
:1018500059850408F436002494B40B085435002448
:101860005835002493F8FF21AA2A7FF454AFD3F807
:10187000C6215AB193F8C2110639C9B2082905D850
:1018800040F2611020FA01F1CE0730D4D3F8D6210E
:101890005AB193F8D2110639C9B2082905D840F2D5
:1018A000611020FA01F1C80721D4D3F8E6215AB11A
:1018B00093F8E2110639C9B2082905D840F261103F
:1018C00020FA01F1C90712D4D3F8F621002A3FF417
:1018D00022AF93F8F231063BDBB2082B3FF61BAF89
:1018E00040F2611121FA03F3DB077FF514AF012306
:1018F000C4F83022A37094E602287FF485AE012359
:1019000084F8E83163707FE67A02013AC4F84C2229
:10191000DD8A05B95D6AC4F83852B3F81120520166
:1019200002F2FF125212C4F85422B3F8131001B994
:10193000196A104400EB45006D00091A40F6F47076
:10194000B1FBF7F18142C4F83C1213D94FF6F470A1
:10195000814212D903212170D96AB3180020C4F83A
